:020000040000fa
:08000000ba6b040001000000ce
:020000040000fa
:10020000409f04000000000096520400000000001f
:10021000b89e0400000000007c50040000000000b4
:10022000c67d040000000000429c040000000000a5
:10023000c0a0040000000000a8a10400000000000d
:10024000800078001106b100030035009101b10073
:1002500001003c000050a100000006001004b100a5
:10026000030035009001b10001003c0010000500c2
:1002700000000500800078001104b1000300350083
:100280009101b10001003c000050a00000000600f8
:100290001004b100070035009001b10004003400e3
:1002a0007000b100030035009001b10001003c0076
:1002b00010000500000005006900e10004003500a1
:1002c0006d00e100030034000002b10001003200c3
:1002d0000000050010000500889fbe008004780023
:1002e000900d81000000e00003003a009a00070032
:1002f0000000e0000a003500900d81000900e000d8
:1003000002003a000004780006003700000478007c
:1003100009004000900007000000e00001003d00df
:100320000084eb00080078004f04be0000000600c7
:100330000c02e20004003d000f42ab00020032005c
:100340000f02ab00feff32000040da00feff370074
:100350000a00fa0080017800e20f500028003e00f9
:10036000a00d8100e10f500008003200e0212000c4
:100370000000e000050032006421200085212000fb
:10038000a62120008001780004003700c42020004e
:10039000e520200006212000432120001440900089
:1003a0000004e000040035008009eb0014409000d8
:1003b0000074a00010429800154090000028a3008f
:1003c00003003a00154090000024a00090429800dd
:1003d0008001eb0007003700154090000008a300e3
:1003e000fdff320063c078000000fb00000b7800c6
:1003f0008301e800828f5100f7ff3a0008003700c0
:1004000030002000b0bf9f00c3bf9f00d1bf9f003e
:10041000e2bf9f006a80570000c0da006fb9970002
:10042000020078000080fa00000006000a00fa00ce
:1004300011002000b1bf9f00c0bf9f006a8057001d
:1004400000c0da004fb897000080fa0000000600f4
:100450000a00fa0051002000b1bf9f00c0bf9f00fa
:100460006a80570000c0da005fb897000080fa0089
:10047000000006000a00fa00881f7800800178005a
:100480000000e00029003a00a00d8100e10f5000bb
:1004900008003200e02120000000e00005003200ea
:1004a0006421200085212000c721200080017800e0
:1004b00004003700c4202000e52020002721200070
:1004c00043212000144090000004e00004003500a7
:1004d0008009eb00144090000074a00010429800c6
:1004e0000002eb000c003700130a200015447800ce
:1004f0006140640002003a008301e900fbff3a001a
:100500000402e8009541780061c0610005003200f6
:10051000170078008058780004035100820f5200c1
:10052000f1ff3a00060051000800370020002000cb
:10053000a0bf9f00b3bf9f00c1bf9f00d2bf9f005d
:100540006c80570000c0da005fb897004f04780055
:100550000080fa0000000600800078000000e00043
:1005600004003a00601b2200900d89000101780010
:10057000060037000081eb0060232200808f5000ce
:1005800002003e00910d89000001eb00020078009e
:1005900000000600020ab900001bb9000200b80002
:1005a000810042008100430000000600889fbe00d9
:1005b0008a9fbe00010578000100e00004003500bc
:1005c00008003c000000e000200032000500370079
:1005d00060001000e080180002003b0001f02c00d9
:1005e0001a0037000004be006011b8006b0920003b
:1005f0000982cf00020039000882cf000441b00018
:10060000694252000e00320008003b0082817100f6
:10061000610164008904d1000884d3008b05e800df
:100620000442e800f9ff3a000500370008044400de
:1006300089844c008b05e9000442e900fbff3a0085
:10064000840107000af0a70001f0a0004f05be00da
:100650004f04be0000000600889fbe008a9fbe00b7
:100660008c1f7800a10107001002200002003b004f
:1006700010458800a50137008a0062006408e10087
:1006800002003a0010458800ad0137006108e10022
:10069000fcff32000800be00030478000b000700d6
:1006a00001f0a100a901070008f0a600040037002e
:1006b0000001be0091042400b0fd20007900070075
:1006c00009f0a70001f0a20099013700889fbe0041
:1006d0008a9fbe008c1f7800840107008b013300c5
:1006e00003866c006450e1002e0032006420e100bb
:1006f000330032006150e1002f0032006120e10040
:100700003100320085855500eb07b000090020005c
:1007100008042000050037000804440089844c00c8
:100720000a0031000603430087834b000001530099
:1007300081815b00f8ff33000203be000800a000c7
:100740000804440089844c00f6ff3900c639dd00f6
:100750008301730001003200130020008904d100de
:100760000884d3000998a300050032000800a70000
:100770000300a0008904d1000884d3008b05e800a1
:100780008904d1000884d3000001eb000281d2006b
:100790003001070001f0a1000cf0a70001f0a0005b
:1007a000630137006420e100650132000801be00ea
:1007b0000200be00f7ff37006120e1006001320057
:1007c0006000b800f3ff37000000200001f82700a8
:1007d000f0ff3700889fbe008a9fbe008c1f780004
:1007e000420107004901330003866c006450e100b8
:1007f000240032006420e100270032006150e10053
:10080000220032006120e100210032008b8542008d
:10081000eb07b1000134b800003ab8000804420008
:1008200089844a00013ab8000030b800888040004e
:1008300009014a00040033000000400081804800a4
:10084000020149008b05e900c909dd008301700040
:100850000100320013002000c814de004814dd003f
:100860004709de001200b200c808de0008847000ec
:10087000f800070001f0a1000cf0a70001f0a000b3
:100880002b0137006120e1002d0132000801be007c
:100890000200be00f7ff37006150e100fcff3a00a4
:1008a0002701370003f0a200889fbe008a9fbe0088
:1008b0008c1f78000d010700140133006450e10023
:1008c0004f0032006420e1005200320003826c00cd
:1008d00007003b000905d0000306d000820f54003a
:1008e0000c065d0002003900020032008901780028
:1008f000030678008582550004003d000003fd00da
:100900008103fd008502ea008b854200840f72009e
:1009100002003b0060001000e08018006011b80089
:100920000005eb007a28e1000a0039000600780093
:10093000c75ddd00f707b200878075002d00370026
:10094000828171000a017800610560008180d10018
:100950000080d3008502e900f9ff3b000604400057
:100960008784480002003b0060041400e0841c00ff
:100970000988a300070032008a817100828171001a
:10098000610164008904d1000884d3008b05e8006c
:10099000170037000978a30013003a000b00e000ad
:1009a000130034008b05e9000804440089844c00de
:1009b0000a4474000978a3000d003a000b00e0001f
:1009c000070034008b05e9000804440089844c00ca
:1009d00001003a000b0020000978a300f7ff320065
:1009e0000001eb0002003700828171000a017800eb
:1009f000980007000cf0a70001f0a000cc00370021
:100a00006420e10002003a00838f6c00cc003300c8
:100a10000801be000200be00c50037000001eb0067
:100a20002f010700040032000200200003f8230019
:100a300001f0a7009bff0700000006000001be00b8
:100a40004e0107000470a70003f0a1006509b10082
:100a5000160032000d0035006828e1000600350060
:100a6000f0ff2f00f1ff27000300e00013003b0020
:100a700001002800000005000000400081804800bf
:100a80008502e900fcff3a0008003700f88f4200b9
:100a900002003c008000eb00000005008100d10056
:100aa0000080d3008502e800fcff3a000300e0006c
:100ab00002003b0060001000e0801800000006000b
:100ac0001400200042013700839f68000100e0000d
:100ad00002003d0060001000e08018000300e0000c
:100ae00002003d0060011100e08119005301070080
:100af0004f00e00002003b0060001000e0801800a2
:100b000000000600889fbe008a9fbe008c1f7800f0
:100b10000004be00190107000478a30026003a0073
:100b20006120e1002500320009f8a30025003a0009
:100b30006420e10021003200f507b1000508a300a0
:100b40000200320000004000818048006044b8008c
:100b500003102000020020000000400081804800b7
:100b60000805440089854c000a0541008b85490031
:100b70000a0550008b855800030033000a00be00b0
:100b800002047400838474008301d1000281d300c5
:100b9000830f7100f0ff3a008904d1000884d3006c
:100ba0006001490082017800c1adde00fb07b000a2
:100bb000280007005e0037000960a0000800be00a2
:100bc0005b0037001202200012458800f0ff2f0062
:100bd000f1ff270056003700f4ff2f00fc0037001c
:100be00004002000fa0037000001be00e300070007
:100bf0000470a70003f0a10003f8a30013003a005b
:100c00006509b10010003200090035006928e100d3
:100c1000020035000100280000000500000040002f
:100c2000818048008502e900fcff3a0000000600d0
:100c3000f88f4200050035008100d1000080d3000c
:100c40008502e800fcff3a00000006008000eb008f
:100c50000000050081002000618055000b003d0070
:100c60000b00200061fe2f000100e1001d00340098
:100c700082817100610164008904d1000884d3007d
:100c80000000e800faff3a007100200061006400f3
:100c9000030070000200600009003200610444009b
:100ca000e0844c000988a500050032008b05e800af
:100cb0006808e10002003a008904d1000884d300ea
:100cc000f20f20000258e10005003d00c75ddd0085
:100cd000f907b2008980750008007800000006005e
:100ce0000bf827008b007800000005000004be0010
:100cf000a20007000003be000405be000200be0003
:100d00009e000700844f7500000006000200be0030
:100d10006450e100050036006420e1000200360066
:100d20000968a30001003a000800be000160a000ad
:100d30004f0678004f05be004f04be0000000600bd
:100d4000f0ff2f00f1ff2700f9ff3700889fbe005a
:100d50008a9fbe008c9fbe000004be008700070073
:100d60000800be00890678006420e1000800390010
:100d7000040032000160a000120220001245880029
:100d80005300370091fc2300b0fd20004e003700d7
:100d90000006eb0009f0a10003f823000200200088
:100da0000800be0046ff07000600340001f82300db
:100db000000020000801be0044fe07000004be0041
:100dc0002c0020000800be0093e82300320a230014
:100dd0003bff0700120034000801be00d1fd2300d4
:100de000703d2b00b0fe07000005be00b3f32300ea
:100df000f27a26000800be0076fe070003f8230002
:100e000002002000a7fe07000801be00a6fe0700a2
:100e10000a01be002dfe07000004be000c06e8001b
:100e20000800be0001f0a10002002000039823008a
:100e300023ff07000800be00160035000801be00b1
:100e400064fe07000005be0032cd2c0043fb2300ea
:100e500095fe0700809fbe001269280003d52b0075
:100e60000a00be005bfe0700620f210013ef2b009b
:100e70008dfe07000a01be0056fe07004f01be00ae
:100e800012fe07000801be0052fe07000801be0066
:100e900085fe07000c00e0000b0032000c10a700dc
:100ea00001f0a200b2fd200093fc23006260e1008b
:100eb0000400320022a9200063f023000c10a700d8
:100ec00063f8230078fe07000df0a70001f0a200f0
:100ed0004f06be004f05be004f04be0000000600d6
:100ee000889fbe008a9fbe000003be00230007004b
:100ef0008505780082815200020020006220e10016
:100f000004003a00f307b100040035007718e1004f
:100f1000040035000600be00140037006000b80071
:100f20000f003700f50f2000faff2f008502d100d7
:100f30000a85d3008301e900fcff3b008184620045
:100f400000046500890f7400f2ff32008582ea0018
:100f50000a85ea0081846200000465003dff070005
:100f600007f0a70001f0a0000081eb000200e00004
:100f70004f05be004f04be0000000600c70ade0099
:100f8000f107b200f50fb20008003200e1cf4200d5
:100f9000020032000170a00024000500810f7000e3
:100fa000010032000408050044000500810f7000b4
:100fb00002003a00140005008502e900000040002c
:100fc00081c04800fcff3b000170a0002400050028
:100fd000889fbe008a9fbe00841f780043ff0700e1
:100fe0004f00780011003300f0ff2f00838f6c005a
:100ff00006003b00040565000a00a7000800370052
:1010000009f0a6001000200008003700820f5400ed
:10101000838f5c00030039001000200001003e00b7
:101020000000200009f0a7000000ea004f05be0004
:101030004f04be000000e000000006006022b8007f
:10104000060220000000d0008180d2000482d2007d
:101050008582d2000000a0000202520083825a0062
:10106000030031000202420083824a000000a10016
:101070000603e900f3ff3a0000000600881f78002d
:10108000000478005001be004000be000400400093
:10109000858048000601490087814900009cbe0008
:1010a0000294be000400e1000588e1000690e10022
:1010b0000798e10002003100680044001008e800d1
:1010c0004f04780000000600f4874700889fbe00a8
:1010d0008a9fbe008c9fbe008e1f78000205be0056
:1010e0000004be00d4b79f00e5b79f00f6b79f008d
:1010f00087bf9f000000eb00c0b79f00b0b79f0004
:10110000a0b79f0090b79f0080b79f000d042000fc
:10111000bfb097004fb09700000140000000e00012
:101120000f003d004f08de0000007100c0b79f00b7
:101130009e00070001003d0012002000a1000700f2
:1011400001003d0012002000a6000700b1000700ca
:10115000b60007000f004000c8ff0700220037005c
:101160004f08de0000067100ccb79f008f0007001b
:1011700001003d00120020009200070001003d0028
:101180001200200097000700a20007000fb297008e
:101190009fb297002fb39700bfb39700a900070035
:1011a0000000520081805a0002015b0083815b00d5
:1011b00080b79f0091b79f00a2b79f00b3b79f0071
:1011c0000007eb009f0007000020e10001a8e100fc
:1011d00002b0e10003b8e100010031001e00200070
:1011e0000e005600c0b79f004fb297000400e00009
:1011f0000700350010002000010020006011b80039
:1012000008047000898470000a0571008b857100e4
:101210008d06e900beff3a000400e00003003d0037
:10122000820007000f00400094ff07004fa89700be
:101230000000e00004003a000fb497009fb497004c
:101240002fb59700bfb59700940007004f077800af
:101250004f06be004f05be004f04be004f01b10057
:1012600000000600881f780018002000881f780002
:1012700095ff07008f87e9004f0478000000060003
:10128000801feb0090ff07008f87e9000000060039
:10129000889fbe008a9fbe008c1f78006e000700ea
:1012a00007003d0073000700e00f5b00e08f5b006c
:1012b00007003d00320007000006eb000400370085
:1012c0003400070002003d002a0007001c00200037
:1012d00072000700e3ff07000203be000002be0029
:1012e0000c00e00001003200220007000400be00f4
:1012f0000601be004f0678004f05be004f04be0039
:1013000000000600889fbe008a9fbe008c1f7800e8
:101310005100070005003d0056000700e00f5b008c
:10132000e08f5b0006003d00040037001900070055
:1013300003003d006000b8006011b8001000070015
:1013400056000700ceff07000203be000002be00e9
:101350000c00e00001003200060007000400be009f
:101360000601be004f0678004f05be004f04be00c8
:10137000000006006000b8006011b80000003700ef
:1013800004025000858258000603590087835900e3
:10139000000006000006eb00e00f5200e08f5a004c
:1013a000e00f5b00e08f5b00000006000180400062
:1013b00090b79f000001eb008fb097000100e000a4
:1013c000000006000200700090b79f0001804000fe
:1013d00080b79f000001eb00ffa897000100e0002c
:1013e000000006000200700080b79f0001804000ee
:1013f0006faa9700cf20de0001007000f0af9f00c1
:1014000004024200250007004f18de0000027200af
:1014100000000600e4af9f000804440089844c00eb
:101420000a054d008b854d00000006003fb2970075
:10143000cfb297005fb39700efb3970000fe2f0085
:10144000000006003fb09700cfb097005fb1970053
:10145000efb19700000006000205be000004be00c8
:10146000e00f5000e08f5800e00f5900e08f590066
:10147000000006006000b8006011b80008045000c9
:10148000898458000a0559008b8559001c002000ea
:10149000e00f5200e08f5a00000006000800be0076
:1014a0000a01be00000006002800fa00889fbe0066
:1014b0008a9fbe008c9fbe0003866b000c02070053
:1014c0000028a30064003a000128a30067003a0046
:1014d0000008a30062003a000108a30065003a007a
:1014e0001e009000be08900081064000ed3fb10054
:1014f000f4805700ee019000111ab8008e09900098
:10150000311bb8009e099000311cb800511db80075
:10151000f485570046000700fe0190003a000700de
:101520008b85e8003e0007008e0990004000070010
:10153000ee019000340007008b85e80038000700ba
:101540008e099000400007009e0990001b18b8000b
:10155000890440000a854800fe019000340007001d
:101560008b85e80038000700ee019000300007008e
:101570008e0990001b18b800890440000a854800b5
:101580000a98a30008003a000402420085824a003b
:1015900006034b0087834b0008044c0089844c00f1
:1015a0000a054d008d06e9008482720085027300f1
:1015b0004c3add0085027200010032001500200067
:1015c000443ade001400b2004538de00cb45dd00b1
:1015d0000b007000c540de00cb4ddd008b8070003d
:1015e0004549de00cb55dd000b017100c551de0021
:1015f0000d037800d701070003f0a1000cf0a7004d
:1016000003f0a000ce0137001b18b800850240008f
:1016100006834800e0834b0060044c00070037005d
:101620001b18b8000603400087834800faff370004
:101630001b18b8008703400008844800e0844c0071
:1016400060054d00000006001b18b80008044000ab
:1016500089844800faff37000108a300b5013a0069
:101660005800be005801be00e3ff37000008a30089
:10167000b0013a0009047800f9ff370081037800cf
:101680003efe07000001be006000b8000478a30021
:1016900013003a006220e10015003e000d00390001
:1016a0008301d1000281d3008180d3008301d10066
:1016b0000281d3008180d3008301d1000281d30055
:1016c0008180d3000538b000c42add00f300b200e9
:1016d0008381720007f0a70003f0a000000006005d
:1016e000f3ff2700f2ff2f006110b900fbff370066
:1016f00003ff2700f7ff37008f1fd100c10107004c
:101700008f87e9000000e00000000600801feb006a
:10171000bc0107008f87e9000000e0000000060020
:101720001400fa00889fbe008a9fbe008c9fbe00f6
:101730000005be000206be00680047000c90be0017
:101740000a90be00d80107006400e1001a003200d0
:1017500016003e006100e1001a0032006e049000a5
:10176000fe0490000e0b90009e0b90006011b800dc
:101770009e0590000b38b100d501200082817100d8
:10178000610164008703d1000683d3008984d300fc
:101790000884d3008502e900f8ff3a002dfd070018
:1017a0000df0a70001f0a00065013700f1ff270050
:1017b000f0ff2f006201370001f827000000200031
:1017c000f7ff37006000b800f5ff3700dd010700c4
:1017d0000509780000000600809feb0089010700e2
:1017e0008f87e9000000e000000006002800fa00f2
:1017f000889fbe008a9fbe008c9fbe0007067800af
:10180000878669000c003b00030478008704780099
:1018100008f0a10009f0a100840f5000858f580046
:10182000860f5900890f5c00030033000cf0a20002
:1018300001003a000cf0a1002d0107006400e10056
:101840005f003200780147006408e1006100320067
:101850006c014700748557003200be001201be00c3
:101860003a04be001a05be001e039000be0a900096
:101870008503530006003d000004fd008104fd00c7
:101880000205fd008305fd008703ea0005037800db
:101890000df8a3000400320060041400e0841c0072
:1018a00060051d00e0851d006022b8007d0320005a
:1018b0000d38e1008006eb000b0039004433dd00f9
:1018c000f300b20083017300390037008482720094
:1018d0000d027800e10664008b85d1000a85d300f3
:1018e0008984d3000884d3008703e900f7ff3b0015
:1018f00008004000898048000a0149008b814900a6
:1019000004003b0060001000e08018006001190036
:10191000e08119000358a300090032008d82720093
:1019200084827200610260008301d1000281d300d1
:101930008180d3000080d3000603e8001b0037003d
:101940000348a30017003a000600e0001700340027
:101950000603e9000d00a300000048008180480054
:1019600002014900838149000348a3000f003a00a7
:101970000600e000090034000603e9000000400012
:1019800081804800020149008381490001003a003a
:101990000003eb000348a300f5ff32006022b8000b
:1019a000020037008482720061826600e90007004d
:1019b00003f0a1000cf0a70003f0a000e000370046
:1019c000640147006408e10002003a000df8a3003a
:1019d000d8003a003200be001201be00d800370025
:1019e0001400fa00889fbe008a9fbe008c9fbe0034
:1019f0000004be000205be00680047000a90be0059
:101a00000890be00280107000070a7000bf0a1009d
:101a10000bf8a30020003a009e0990000e099000e8
:101a2000fe0090006e0090009e0290003443200063
:101a300084825200c20032000a003c00b4fc2f0035
:101a40000428e100140034008301d1000281d30096
:101a50008180d3000080d3008502e800faff3a00bd
:101a6000b7003700b40020000428e10007003c0064
:101a70000000400081804800020149008381490044
:101a80008502e900faff3a00ad00370003002800a4
:101a900002002000010037006011b8006000b800ab
:101aa000a70037002800fa00889fbe008a9fbe006a
:101ab0008c9fbe0003866b008d0007006400e10070
:101ac000440032006408e1004a0032006100e10095
:101ad000460032006108e10049003200ec06470090
:101ae0006000b8003d02be003d03be00f486570012
:101af0006011b8003d04be003d05be007d0320001e
:101b00000b0037000000a0008d06e9001300320032
:101b10000402420085824a0006034b0087834b0083
:101b20000000400081804800020149008381490093
:101b30000802520089825a000a035b008b835b0013
:101b4000f0ff3b000802420089824a000a034b0072
:101b50008b834b008d06e900edff3a008482720012
:101b600086827200f707b20087827200010032009d
:101b7000150020001e0490003e0b90000603540048
:101b8000e63fb0000368a300070032000000a70092
:101b90000500a0008301d1000281d3008180d30021
:101ba0000080d3000603e8008301d1000281d30046
:101bb0008180d3000080d3000002eb000482d200b9
:101bc0006400070003f0a1000cf0a70003f0a000e0
:101bd0005b003700640247006408e10055003200f2
:101be0003400be003401be00f6ff37006108e1009a
:101bf000500032006011b8006000b800f1ff3700fb
:101c000003ff270002002000fbff3700889fbe0073
:101c1000830478000300e0002c00350003003c0042
:101c2000008270000402710026003200364320005a
:101c3000c50020008383cf000a0039000541b100b0
:101c40008283cf00070039000541b1008183cf00b6
:101c5000040039000541b1008083cf000100390044
:101c60000541b10085c353006022b8001200320064
:101c70000a003b0084827200610260008301d1008f
:101c80000281d3008180d3000080d3000603e800e6
:101c90008743e800f7ff3a000700370000004000e4
:101ca0008180480002014900838149000603e90060
:101cb0008743e900f9ff3a002600070009f0a70072
:101cc00003f0a0004f04be000000060060001000fa
:101cd000e080180060011900e0811900d3ff3b008b
:101ce000033e2c00f7ff370007f0a200bffe3700cd
:101cf000680447000294be000094be00fc04470044
:101d00008694be008494be00090078006600070037
:101d1000080078006400070099007800814f700087
:101d20000b003b000800be00930007004f00b1000d
:101d300003003700f3ff2700f2ff2f006110b90006
:101d40004f06be004f05be004f04be000080fa00e3
:101d5000000006001800200057002000080453006f
:101d60000d003d000600200097fc2f000740e10019
:101d70001e00340084827200610260008301d10081
:101d80000281d3008180d3000080d3000804e800e2
:101d9000f8ff3a0047002000610460000504740069
:101da000040464000d00320061004000e08048003f
:101db00060014900e081490003b8a5000700320036
:101dc0000603e8006538e10004003a008301d10011
:101dd0000281d3008180d3000080d300f87f2000ef
:101de0000830e10003003500080378006000b80007
:101df0006011b8004433dd00f300b20083017300ca
:101e000000000600889fbe008a9fbe008c9fbe0017
:101e10000404be000605be00809fbe00829fbe0077
:101e200063000700040678000800be000a01be0037
:101e30005f000700840678004f03be004f02be001b
:101e40008d4f76007fb0970013003300f0ff2f0016
:101e50008b8f6b0006003b000d0666000c00a70090
:101e60000a00370007f0a600100020000a00370023
:101e7000880f5200898f5a008a0f5b008b8f5b009e
:101e8000030039001000200001003e000000200087
:101e900007f0a7000000ea004f06be004f05be0095
:101ea0004f04be0000000600800078005002be0013
:101eb0005003be004439de00f700b200f37f20007b
:101ec00003016100090032000218e10016003a0027
:101ed0008501720083017300838173000008200074
:101ee00015003a0040002000130037008501720001
:101ef000830173008381730005003a0004a8be00cb
:101f000006a8be00100020000b0037000201e90007
:101f10000402420085824a0006034b0087834b007f
:101f20000748a300f9ff32000740a00004a8be0044
:101f300006a8be00200020008000980092009800b3
:101f4000000006000003be000cfc07006220e10058
:101f5000020032000600be0005000500e507b100e2
:101f6000f107b20004f023008480700007f0a7009e
:101f700001f0a00024000500e48240001078a300d6
:101f800007003200640240001178a3003400be0054
:101f90001401be00040032000330a7000000060058
:101fa0003500be001501be000330a0000000060091
:101fb00005ff270005826100070032000428e100c8
:101fc00001003200240005000600070001003a006d
:101fd000440005000408050002000700f9ff3a006c
:101fe000140005006f82610081027000850271009b
:101ff0008502720000000600800078003004e000d6
:10200000feff3a00010050000000e9000000060059
:102010000c00fa00a0bf9f00c0bf9f00f6ff0700a2
:10202000b0bf9f00f0bf9f00100c2000d0bf9f00ea
:1020300074815700efb097006c805700470107008c
:102040000080fa00000006008001eb00020037006b
:10205000817178008301e800828f5100fcff3a0013
:10206000000006000c00fa00a0bf9f00c0bf9f0048
:10207000e1ff0700b0bf9f00f0bf9f00100c2000e1
:10208000d0bf9f0074815700efb097006c8057005d
:102090007f0207000080fa000000060000017800bf
:1020a00000c2b300010037000201e800924078004e
:1020b00080cf5000fcff3200e9cf5000faff320021
:1020c000d0c2b30080cf500003003a000201e80004
:1020d00014c0b300050037000042eb00b0c2b300eb
:1020e00080cf500001003a000201e8008000eb00c0
:1020f00005fd2f00040037006a08b9000080410088
:10210000850040000201e8009201fb0005804100cb
:10211000e90f5000f8ff36000404e000010032002f
:102120008100ea000100780000000600889fbe00e0
:102130008a9fbe008c9fbe0000017800e11422003f
:102140001100e0000b003a0020152200700a8900ff
:10215000500a8900910a8900610a89002140900093
:102160000004a000a0409800614090000004a0007e
:10217000e0409800e7004100c208de00c20cdd002c
:10218000640a81006d1b2200602322000d055000af
:1021900022002000811f7800110009000205d800ec
:1021a00000067800cf007800c308dd00e485400019
:1021b0008001eb00661b2200e514220001003700bd
:1021c00001027800244090000008a30002003200c1
:1021d0000a003700110a780094007800214090002e
:1021e0000008a300fbff320009014200828f50006b
:1021f00002003900840f510046003100940078003d
:10220000848f5000eeff3e00868f500002003900a0
:10221000858f5000eaff3900500a8100800f52007c
:102220004f003a00858f50004d003a008301e800ce
:10223000e18f5100e2ff36008c8f5400040036001d
:102240008a8f5400020031000b047800120037001e
:10225000614ab8006151b900b0ff2f0001002000b1
:102260000200500083805800800f5200818f5a0076
:102270000200350009047800070037000d80540083
:102280009223220002004000110009000a80d800b9
:102290000a80b90000047800080078000ef80700f2
:1022a00080017800e10f40002d003200500a8100cb
:1022b00003087800520a810064004100a2409000a7
:1022c000808f5100020032000104a000010037009d
:1022d0000104a100214198000880410064005000e1
:1022e00080097800500a8900e21422000208780070
:1022f000510a8100214090000004a000a0409800f5
:10230000234090000004a100a04198000202780040
:10231000a7ff3700620a8900828f5000090036004b
:102320009200780080142200a241900003487800b7
:10233000310a8900140978008040eb00600a8100ae
:1023400021409800600a8100000a78002440900033
:102350000004a00020429800640042000100370001
:102360000000eb004f06be004f05be004f04be004c
:102370000000060064005000600a8900a040900040
:102380000104a1002140980000000600889fbe00c3
:102390008a9fbe0000057800e40150001300100081
:1023a000c285de00234090000008a3000400320034
:1023b000630a8900234090000004a100a041980016
:1023c0000100780059ff0700000478000000e000d9
:1023d000170032008a0f50001500320060b89700d5
:1023e00008005000c284de00898f550001003600cd
:1023f000890578004259dd008a00780008007800dd
:10240000c40207008a0f5400090031004248dd0071
:10241000000044008a0f5000050036000a005000fa
:1024200000004400320a8100430a81000288be0095
:10243000080078004f05be004f04be0000000600f3
:1024400000047800ba02070008007800b8f7070017
:102450000c00fa00889fbe0000047800cfb09700ff
:10246000f0ff2700d0bf9f008004eb0099bf9f00c2
:1024700088bf9f00a8bf9f00200c2000b0bf9f0016
:1024800078815700708057000e0307000fb897003f
:10249000094878000fb89700080450000800780039
:1024a0004f04be000080fa0000000600889fbe00b6
:1024b000000478008144780000fd2f0000004400f3
:1024c000e90f500002003e00000178000d003700c7
:1024d0000800780061f707000000e0000300320008
:1024e0000800780063f7070000047800080078000f
:1024f00067f707000000e0000700320090fa2f00a5
:10250000000144000980fb00800f510002003d00e3
:102510000280fb0001003700f00f20004f04be00d6
:1025200000000600881f7800400d81002a0807007f
:102530000004780060f707000000e000faff3a00ae
:10254000e10f440003003200410d810008007800d3
:10255000550807004f04780000000600ec8747008c
:10256000889fbe008a9fbe008c9fbe008e1f780091
:1025700081bf9f0002077800400d89008046eb0074
:10258000040137008884fb00090078004af707003f
:10259000800078000000e00002003200e1ff070048
:1025a000fc00370050c2b300804f5400f0003a00e6
:1025b0000fbd970020c0b300c0ef9f00d1ef9f0078
:1025c00081ef9f000300370040c0b300c0ef9f00c1
:1025d0000fbd97000fb99700b240780082bf9f00ef
:1025e0008184fb0090c6b30080cf500035003200dc
:1025f00017003e006640500080cf5000620032005d
:102600000c003e007740500080cf50002800320080
:1026100006003e000104e0009b003200a0c2b300af
:1026200080cf50006e003a001d00370080c5b30017
:102630001600370040c6b30080cf500021003200a2
:102640006440400080cf500065003a00120037001f
:1026500030c7b30080cf50001e00320007003e009c
:102660006740500080cf50001100320063404000ae
:1026700080cf50005a003a001400370050c7b30012
:1026800080cf50000f0032006340400080cf5000e8
:1026900053003a006500370020c0b300cbff37007d
:1026a000dfe897008140e800d1ef9f00c8ff3700c6
:1026b0004fe9970080c0b300e24f5100c3ff3a00da
:1026c000c1ff3700acc0b300590037008cc0b30065
:1026d0005700370093ff0700dfe897000104e00090
:1026e00002003a004e017800d2b79f00400d8100f1
:1026f000b907070000047800e10f4000a200320093
:102700008fec9700120037000a85e8008abf9f000f
:10271000160037008fb897001100fb00800f54009f
:10272000f9ff32005fe997000204e00003003a007d
:102730005fb0970008587800d0b79f008944e9003f
:102740000a003200400d8100a30707000004780052
:102750000800e800e10f500004003600080078008f
:10276000d5f607000000e000eaff3200dfe897003e
:102770000104e00087003a008d46e8005fb1970051
:1027800001497800830037005fe897000004e0000b
:1027900003003a008d46e800ce007800d1b79f00d4
:1027a000400d81008c070700e10f400076003200e9
:1027b0005fe997000204e00003003a00dfb09700f1
:1027c00080587800d1b79f000fe997000241e900d7
:1027d00082ef9f004240a9006e003400f0ff3700f6
:1027e0000180fb0008fd2f0008004000e90f5000a9
:1027f0005f003e000a00780028fe070080ef9f007f
:1028000088007800030037000fb897000000e80048
:1028100080bf9f000fb997001200fb00010040002d
:10282000e90f5000f8ff360069ff37000cc1b30014
:102830003cff0700400d8100670707000005780096
:102840000040eb00e0ef9f00d0022000800f550019
:1028500005003a00400d81005f0707000005780081
:1028600011c0b300e1ef9f008c4078000a007800af
:102870000eff0700e14f40000a003a00410d8100c1
:102880000a007800880707000d04e0004b003a00ba
:10289000400d8100300090000048a300430032004a
:1028a000480037008fed97006044b8000c81fb00b2
:1028b000030020000800be0036f707000004be0039
:1028c0008c4078000a007800f8fe07000080fb00ca
:1028d0000100200008044000898448008b45e9007d
:1028e00007003200400d81003b070700000578001b
:1028f0008c407800edfe0700e14f4000ebff3a000e
:102900008c4078000a007800e8fe0700e14f4000a4
:1029100003003a00410d81000a00780062070700b9
:102920006fe997000204e000020032006004140026
:10293000e0841c005fe897000004e00015003a0006
:102940008d46e800cfe89700e4cf500003003a003e
:102950004e0078000888be000e0037000e81e900a6
:102960000207780012007800080878000900370094
:10297000400d810018070700808f540005003200c9
:10298000e10f40000b003a000d04e0000d003200a2
:102990000a0037008fb897003144780081bf9f004c
:1029a0000804e000f7fe3a00040037000000eb00e6
:1029b00005003700410d81003b0707000d80fb003b
:1029c000010037000080eb004f0778004f06be0083
:1029d0004f05be004f04be00cf00b100000006004e
:1029e000889fbe00000478008144780000fd2f001d
:1029f00000004400e90f500002003e000001780092
:102a00000d0037000800780014f607000000e00011
:102a1000030032000800780016f607000004780072
:102a2000080078001af607000000e00007003200f6
:102a300090fa2f00000144000980fb00800f510034
:102a400002003d000280fb0001003700f00f200073
:102a50004f04be0000000600881f7800500d810062
:102a6000dd0607000004780013f607000000e00010
:102a7000faff3a00e10f440003003200510d8100db
:102a800008007800080707004f04780000000600df
:102a9000ec874700889fbe008a9fbe008c9fbe00c7
:102aa0008e1f780081bf9f0002077800500d8900bb
:102ab0008046eb00040137008884fb0009007800a1
:102ac000fdf50700800078000000e0000200320001
:102ad000e1ff0700fc00370050c2b300804f5400f4
:102ae000f0003a000fbd970020c0b300c0ef9f0078
:102af000d1ef9f0081ef9f000300370040c0b3007b
:102b0000c0ef9f000fbd97000fb99700b24078004b
:102b100082bf9f008184fb0090c6b30080cf50002d
:102b20003500320017003e006640500080cf500054
:102b3000620032000c003e007740500080cf500011
:102b40002800320006003e000104e0009b00320035
:102b5000a0c2b30080cf50006e003a001d003700c5
:102b600080c5b3001600370040c6b30080cf5000c8
:102b7000210032006440400080cf500065003a00e0
:102b80001200370030c7b30080cf50001e00320063
:102b900007003e006740500080cf50001100320017
:102ba0006340400080cf50005a003a0014003700c4
:102bb00050c7b30080cf50000f0032006340400088
:102bc00080cf500053003a006500370020c0b300aa
:102bd000cbff3700dfe897008140e800d1ef9f008e
:102be000c8ff37004fe9970080c0b300e24f5100a3
:102bf000c3ff3a00c1ff3700acc0b3005900370033
:102c00008cc0b3005700370093ff0700dfe8970040
:102c10000104e00002003a004e017800d2b79f00a4
:102c2000500d81006c06070000047800e10f4000a1
:102c3000a20032008fec9700120037000a85e800ee
:102c40008abf9f00160037008fb897001100fb0065
:102c5000800f5400f9ff32005fe997000204e000a2
:102c600003003a005fb0970008587800d0b79f0083
:102c70008944e9000a003200500d81005606070021
:102c8000000478000800e800e10f5000040036005e
:102c90000800780088f507000000e000eaff320035
:102ca000dfe897000104e00087003a008d46e80065
:102cb0005fb1970001497800830037005fe8970013
:102cc0000004e00003003a008d46e800ce007800e2
:102cd000d1b79f00500d81003f060700e10f400073
:102ce000760032005fe997000204e00003003a003a
:102cf000dfb0970080587800d1b79f000fe99700a8
:102d00000241e90082ef9f004240a9006e003400ba
:102d1000f0ff37000180fb0008fd2f000800400095
:102d2000e90f50005f003e000a007800dbfc07005e
:102d300080ef9f0088007800030037000fb89700ed
:102d40000000e80080bf9f000fb997001200fb0051
:102d500001004000e90f5000f8ff360069ff37001e
:102d60000cc1b3003cff0700500d81001a0607009c
:102d7000000578000040eb00e0ef9f00d00220004b
:102d8000800f550005003a00500d81001206070023
:102d90000005780011c0b300e1ef9f008c4078007f
:102da0000a0078000eff0700e14f40000a003a00d9
:102db000510d81000a0078003b0607000d04e00079
:102dc0004b003a00500d8100300090000048a300f5
:102dd00043003200480037008fed97006044b80090
:102de0000c81fb00030020000800be00e9f507008d
:102df0000004be008c4078000a007800f8fe07004e
:102e00000080fb0001002000080440008984480085
:102e10008b45e90007003200500d8100ee050700e8
:102e2000000578008c407800edfe0700e14f40007f
:102e3000ebff3a008c4078000a007800e8fe0700bb
:102e4000e14f400003003a00510d81000a00780074
:102e5000150607006fe997000204e0000200320047
:102e600060041400e0841c005fe897000004e000a8
:102e700015003a008d46e800cfe89700e4cf5000f7
:102e800003003a004e0078000888be000e003700ac
:102e90000e81e90002077800120078000808780027
:102ea00009003700500d8100cb050700808f5400ca
:102eb00005003200e10f40000b003a000d04e00075
:102ec0000d0032000a0037008fb8970031447800b7
:102ed00081bf9f000804e000f7fe3a0004003700bd
:102ee0000000eb0005003700510d8100ee050700e2
:102ef0000d80fb00010037000080eb004f077800d9
:102f00004f06be004f05be004f04be00cf00b1000b
:102f1000000006008001eb000200370061f079003c
:102f20008301e800828f5100fcff3a000000060098
:102f3000881f7800600d81000000e0000100320071
:102f400000000100080b220008007800f3050700cc
:102f50006c044400400d2200800f5400faff3a0038
:102f60004f04780000000600889fbe008a1f78008a
:102f7000804078000004e00021003d008040ea002d
:102f8000d0c6b30080cf5000090034008104fb009c
:102f900042062000110009008204d80000017800d8
:102fa000010078004311dd002aba21001f0037001c
:102fb0000100fb0023ba210039003700a2002000e5
:102fc000110009000200d80000017800010078001b
:102fd0004311dd00030141004300dd000300400018
:102fe0003002be002003be0042209000d22090009c
:102ff000f2219000622190002bf907002e0037008b
:10300000d0c6b30080cf5000230034008104fb0001
:1030100042062000110009008204d8000001780057
:10302000010078004311dd002ac521000a0141009a
:10303000a8002000110009000800d8004300dd00ae
:103040000a00400040229000d022900060239000af
:10305000f02390000288900092889000b28990003e
:103060002289900010f90700801f78000102780083
:10307000110009008804d8000102fd004f0078000b
:103080000402fb004322dd000a0242005403be009a
:103090004402be00d8ff37000100fb0023c5210019
:1030a000eacf5000c5ff3c004300dd0003004000b4
:1030b0005001be004000be004f0578004f04be0026
:1030c000000006008f03b000889fbe008a9fbe00ec
:1030d0008c9fbe008e1f7800e0b79f00f1b79f0065
:1030e00082bf9f000000eb00a0b79f00e6043700fe
:1030f0008001eb0050c2b30080cf500009003200c5
:103100000100fb00efb09700ec040700e10f400066
:10311000dd043200afb097008100e800a1b79f0046
:10312000d90437007fb1970092407800d0c2b30035
:1031300080cf50000c00320007003c006d40500072
:1031400080cf50000d0032006b40400080cf500017
:1031500019003a000e00370000c3b30080cf5000c2
:1031600015003a000f0037000330a0007fb297002f
:103170000402e800f4b79f00eaff37000300a00054
:10318000ffb297008502e800f5b79f00e5ff370022
:103190000310a0007fb697000c06e800fcb79f0064
:1031a000e0ff37000320a0007fb097000000e80098
:1031b000f0b79f00dbff37000318a30001003200c7
:1031c0000300a1000338a300010032000320a10086
:1031d0000100fb0002fd2f0002004000e90f50003b
:1031e00010003e008000eb00c1b79f000202780093
:1031f0004fb197006a10b900ffb297001501fb00ac
:103200000001410004014100c2b79f005500fb00ce
:10321000f5b79f0004004000e90f50000d003e008c
:10322000f3ff37000006eb00ccb79f00a0c2b3004d
:1032300080cf500007003a000fb89700c000780018
:1032400080bf9f00c1b79f007fb197000201e800d7
:10325000f2b79f00e0c2b3007fb29700944f100016
:1032600021003a00830678000de0a0008400e80009
:1032700064405000914f100004003200f1b79f00ed
:103280008002eb00b5b79f00100037000fbe97001b
:103290004c0078008cbf9f00b0b79f00ffb0970034
:1032a0008180e800f1b79f00130037003fb297001c
:1032b0006a20b9000000410003004000b0b79f0041
:1032c000ffb297008502e800f5b79f007fb6970030
:1032d0001c01fb0003fd2f0003004100e90f50001b
:1032e000f2ff360004003700830678000dc0a0000e
:1032f0000000eb00b0b79f007fb19700b2407800ac
:10330000f2b79f00c17f9f00c0c6b30080cf5000be
:103310002700320014003c006840500080cf50006d
:103320009d00320009003c006c40500080cf5000ee
:10333000290032006b40400080cf50007200320004
:103340000104e000560432008e00370060c6b3006e
:1033500080cf50001c0032006340400080cf5000fe
:1033600088003a008c00370030c7b30080cf50008f
:103370001c00320007003c006440500080cf500029
:10338000130032000040e80080cf50007d003a007a
:103390001100370050c7b30080cf50007d003200cd
:1033a0006340400080cf500076003a000b003700a9
:1033b000000028000d48a30001003a000001200091
:1033c00080867600ccff37000da0a0007200370089
:1033d0000d60a000700037000d50a0000d70a0001f
:1033e0006d0037008fb997004300780083bf9f00be
:1033f000000478000000e00001003a0048082200c4
:103400008004eb00010037008104e80089007800a7
:10341000088044001004e000fbff3a003fb2970030
:103420000400e00003003200890f52000100310067
:10343000840478000007eb00cfb29700898f520018
:1034400001003600098752004368de00e106600093
:1034500019003a000d06780009003700efb0970018
:103460000002200015040700e10f400003003200b5
:103470002fb097000000e800a0b79f000c06e800fe
:103480008e0f5600f5ff3a000087eb000a00370068
:10349000880078003100fb0001047800efb097004d
:1034a00006040700e10f400003003200afb09700b0
:1034b0008100e800a1b79f000900e90080047800be
:1034c000e10f4000f2ff3a000006eb000d00e000c3
:1034d0000a003a00ec033700efb09700000220002a
:1034e000f6030700e10f4000030032002fb1970000
:1034f0000201e800a2b79f000c06e8008e0f5600fc
:10350000f5ff3a00e00337008fb9970043007800d9
:1035100083bf9f00cf80de00010178008201780028
:103520000205be000004be000203be000002be0091
:103530004822de00482edd0004027600c47f9f0092
:103540000d48a3000a0032000404e0000800320025
:10355000e14f420006003200d1fb2f0001804700fe
:103560000448780018409800290020000200370025
:10357000d07f9f0019002000d2fb2f00028447005b
:10358000a6ff3700c3fb2f0003844700190020006b
:10359000a2ff37000d0cb30000702000008266000f
:1035a000270232000dc8a300020032006400200090
:1035b000b4b79f000d48a300050032000fba970072
:1035c0004401be004400be0084bf9f0004003700d9
:1035d0008fba97004500be0085bf9f0027f80700ff
:1035e000e0af9f00f1af9f0082b79f0093b79f00ad
:1035f0006022b8006033b8006fa89700ffa897005a
:103600000fb197009fb197003bf807000000e00062
:103610000a003d006fa89700ffa897000fb1970020
:103620009fb1970003f0a200e0af9f00f1af9f00b1
:1036300082b79f0093b79f003d00b3000000eb00ee
:1036400080a79f006022b8006033b8006fa8970081
:10365000ffa897000fb197009fb197002bf80700c4
:103660000000e000340032006fa89700ffa8970028
:103670000fb197009fb1970029f8070003fc2f00b6
:103680000381470051f807000fa097000000e900f0
:103690006300b900a2002000110009000200d80058
:1036a0008000fd0081a79f000100e00002003d00b6
:1036b0000100e90080a79f000fa497000840ea00de
:1036c00029fe07006faa9700ffaa97000fb3970083
:1036d0009fb3970074f70700a0af9f00b1af9f00a2
:1036e000c2af9f00d3af9f006022b8000600200049
:1036f00007ff230000f807000000e00002003d0083
:103700000800e9000b0037006022b8000600200026
:10371000470224002fa89700bfa897004fa9970041
:10372000dfa997002cf807000000e0000200350038
:103730000800e80080a79f003fb29700f80f5200f2
:1037400057003c00d0c6b300804f5200290036001d
:103750000485fb0042062000110009000285d80004
:1037600000017800010478004311dd002bba21002c
:103770000b0141006022b8000600200007fe230074
:103780000288900092889000b2899000228990006f
:1037900045f70700a9002000809fbe001100090026
:1037a0000984d800000478004f00be004344dd00c7
:1037b0000b04440048229000d82290006823900017
:1037c000f823900038f70700801f78000102780086
:1037d000110009000985d8000102fd004f007800a2
:1037e0004322dd000b0242005403be004402be002f
:1037f0001f0037000480fb0029ba2100ea4f520065
:1038000014003600a2002000110009000280d80038
:1038100000017800010478004311dd000901410036
:103820006022b8000600200007fe2300422090001e
:10383000d2209000f2219000622190001af7070038
:103840004344dd00090444003802be002803be00e2
:10385000070037004300dd00090040006022b80087
:103860000600200007fe23005001be004000be00fd
:103870000df707000002be000203be006fa897000c
:10388000ffa897000fb197009fb19700d7f70700e7
:10389000e0af9f00f1af9f0082b79f0093b79f00fa
:1038a0000fa49700e90f540015003c006022b800f7
:1038b0006033b8006fa89700ffa897000fb197007a
:1038c0009fb1970091f707000000e000320032003e
:1038d0006fa89700ffa897000fb197009fb19700be
:1038e0003ff80700e00f5000e08f5800e00f59004c
:1038f000e08f590028003a00e10f54002600340000
:103900000400200005002e00b6e02200170124006c
:103910002fa89700bfa897004fa99700dfa997008d
:1039200075f707000000e00002003d00730054003e
:10393000010037007200540080a79f000fc097005d
:1039400089fd0700a0af9f00b1af9f00c2af9f00ed
:10395000d3af9f000002be000203be006fa8970015
:10396000ffa897000fb197009fb197004df807008f
:103970001bf807000205be000004be006000b8008e
:103980006011b800a0a79f00b1a79f00c2a79f0029
:10399000d3a79f002e0037006fa89700ffa89700bd
:1039a0000fb197009fb197000df807000205be0008
:1039b0000004be00e00f5000e08f5800e00f5900f7
:1039c000e08f59000200350090f80700130037001f
:1039d00010002000010020006011b8000800600005
:1039e000898060000a0161008b8161008b03d10036
:1039f0000a83d3008982d3000882d30000007200ba
:103a00008180720002017300838173007ff80700d8
:103a10000002be000203be0074f707000002be00f1
:103a20000203be006fa89700ffa897000fb1970090
:103a30009fb19700acf80700a0a79f00b1a79f0017
:103a4000c2a79f00d3a79f000000eb0080a79f00a4
:103a500014c0b300a5f221000b0037000400fb00e6
:103a60004300dd00050040005001be004000be00e4
:103a70000040e10001c8e10002d0e10003d8e1000c
:103a8000030039000442e800f44f5200f3ff3a000b
:103a9000c47f9f000400fb00bfb09700008040007f
:103aa0008fa09700010040004fb197000007510020
:103ab000bfb197000300e000010032000e07e900eb
:103ac00063806600010032000e07e9000d28a300a4
:103ad00026003200e18066000d18a3000c003200c1
:103ae000d00220000100e00001003a000080e9005f
:103af000efb0970071020700e10f4000180032009c
:103b00002fb297000402e800a4b79f00140037000a
:103b10000100e00012003200efb097000002200028
:103b200066020700e10f40000d003200afb29700bf
:103b30008502e800a5b79f0009003700efb09700a5
:103b4000000320005d020700e10f40000300320087
:103b50002fb697000c06e800acb79f000e07e900ef
:103b60000e00e000f5ff3c003d0037000d38a300db
:103b70000a0032000b003700efb09700000220006f
:103b80004e020700e10f4000030032002fb0970003
:103b90000000e800a0b79f000e07e9000e00e0005b
:103ba000f5ff3c00e18066000d18a3000c00320018
:103bb000d00220000100e00001003a000080e9008e
:103bc000efb097003d020700e10f400024003200f3
:103bd000afb097008100e800a1b79f002000370038
:103be0000100e0001e003200efb09700000220004c
:103bf00032020700e10f4000190032002fb1970098
:103c00000201e800a2b79f00150037000000fb008a
:103c10004300dd00a1f22100010040003002be009f
:103c20002003be000800be000a01be008df507009b
:103c3000a4002000050020006033b80090f50700c4
:103c40000003b000efb097001c020700e10f400036
:103c500003003200afb197008301e800a3b79f00d3
:103c60004f7a97000440e900c07f9f00e14f400079
:103c7000e6ff3a000b003700efb09700000320008a
:103c80000e020700e10f400003003200afb29700c0
:103c90008502e800a5b79f000fa097000000e9008b
:103ca00080a79f000fa097000000e000f2ff3c00fb
:103cb0003fb6970020c1b300f20f560001003c0050
:103cc0006fe09700c07f9f00cf7897000100fb0056
:103cd0003fb1970000005100e0a79f000104e00001
:103ce00008003200efb09700e0022000f301070067
:103cf000e10f400003003200afb197008301e800fc
:103d0000a3b79f004f78970097fc07000002be0002
:103d10000203be002fa09700bfa097004fa19700fd
:103d2000dfa19700e0f507002df707001e00370020
:103d30000000fb004300dd00acf221000c0040005d
:103d40003002be002003be000800be000a01be0013
:103d500044f50700a4002000050020006033b800ef
:103d600047f507000003b000efb09700d30107004c
:103d7000e10f4000030032002fb297000402e80078
:103d8000a4b79f00cf7a97000500fb004300dd0039
:103d90000c0040003002be002003be000800be0040
:103da0000a01be0036f507000205be000004be0091
:103db0004f7e97000c40e900c07f9f00e14f40001c
:103dc000dbff3a000006eb0009003700efb0970078
:103dd00000032000b9010700e10f4000030032009a
:103de0002fb097000000e800a0b79f000c06e80085
:103df000efa09700810f5600f4ff3a000d38a300a2
:103e0000a10132000e00e0009f0134000006eb002b
:103e1000efb0970000022000a8010700e10f40006a
:103e2000030032002fb197000201e800a2b79f0003
:103e30000c06e8008e0f560093013200f4ff3700a5
:103e40000d007800000cb20028003a000d00e000e0
:103e500005003d008fb997004305be004304be0036
:103e600083bf9f00140037000d48a3000b003200f1
:103e70000fba97004400be0084bf9f004f89de0048
:103e8000cf91de000002be000203780082037800ba
:103e90000605be000404be00070037008fba970075
:103ea0004500780085bf9f0000047800cfc4de0085
:103eb000090578008a057800e00f5400e08f5c0067
:103ec000e00f5d00e08f5d0020003d003d00b3008d
:103ed0006000b8006011b8000804500089845800e0
:103ee0000a0559008b855900180037000d00e000c5
:103ef00005003d000fbe97004c05be004c04be00ff
:103f00008cbf9f00110037000d48a300080032004d
:103f10008fba97004500be0085bf9f00040178005e
:103f2000840178000205be000004be0007003700cf
:103f30000fbe97004c0078008cbf9f0000047800f3
:103f4000090020000a0020000b0020003fb097006d
:103f50000000e00007003a00e00f5400e08f5c0032
:103f6000e00f5d00e08f5d0002003a0011002000cc
:103f7000b1b79f000d0778000e0cb20000042000be
:103f8000800f57002f00320003003c000e00e000bd
:103f9000070032003f00370000082000800f570064
:103fa00014003200000c2000800f570039003a0046
:103fb00014c0b300a5f221000b0037000400fb0081
:103fc0004300dd00050040005001be004000be007f
:103fd0000040e10001c8e10002d0e10003d8e100a7
:103fe0002b0039000442e800f44f5200f3ff3a007e
:103ff0002700370000012000010020006011b800f8
:1040000014c0b3000040e10001c8e10002d0e100ab
:1040100003d8e1001e003900450020000000d00058
:104020008180d2000281d2008381d2008502e90022
:10403000faff3a000442e800f04f5200f1ff3a0064
:104040001300370080002000010020006011b8003c
:1040500014c0b3000040e10001c8e10002d0e1005b
:1040600003d8e1000a0039003c0020000000d00025
:104070008180d2000281d2008381d2000c06e90047
:10408000faff3a000442e800f54f5200f1ff3a000f
:10409000c47f9f00cf7897000100fb003fb19700dd
:1040a000820f500002003d00c27f9f0004003700d5
:1040b000bfb19700808f510001003d00b0b79f0055
:1040c0004fb297000400e0000400320063806600f5
:1040d000020032000402e900c4b79f000de8a3000b
:1040e0000b003200cfb297003fb697008c8f520082
:1040f00003003c000000eb00c0b79f000400370045
:10410000cfb097003fb1970082805000c1b79f00a9
:10411000cf7997000300fb000002eb0094a79f00fb
:10412000cfb29700808f520002003400008052000e
:1041300090a79f000d28a30037003200e1806600a1
:104140000d18a3000c003200d00220000100e00096
:1041500001003a000080e900efb09700d7000700a7
:10416000e10f40000e0032002fb697000c06e80069
:10417000acb79f000a0037000100e00008003200e1
:10418000efb0970000022000cc000700e10f4000d4
:10419000030032002fb097000000e800a0b79f0096
:1041a0009fa097000100e0000f0032000006eb0026
:1041b000efb0970000032000c0000700e10f4000af
:1041c000030032002fb197000201e800a2b79f0060
:1041d0000c06e8009fa19700830f5600f4ff3a00f9
:1041e0000002eb0094a79f00bfb29700c328dd0038
:1041f00020f221008080400091af9f004228dd0026
:104200006400500080af9f006328b900f0a79f00b2
:1042100063065000820037001fa697000c00e000e4
:1042200011003200688066000f003a000006780036
:10423000efb0970000022000a0000700e10f40004f
:10424000030032002fb097000000e800a0b79f00e5
:104250000c06e8009fa09700810f5600f4ff3a007b
:104260000001eb0092a79f00e18066000d18a300fb
:104270000c003200d00220000100e00001003a00f2
:104280000080e900efb097008c000700e10f4000cc
:10429000d5ff3200afb197008301e800a3b79f00bc
:1042a000d1ff37000100e000cfff3200efb09700f0
:1042b0000002200081000700e10f4000caff320029
:1042c0002fb297000402e800a4b79f00c6ff370092
:1042d00000042000800f57003000320003003c0033
:1042e0000e00e000070032003d003700000820000b
:1042f000800f570011003200000c2000800f570083
:1043000037003a001fa897003002be002003be000d
:104310000800be000a01be00d2f30700a40020007e
:10432000050020006033b800d5f3070004c3b300d4
:1043300004424000c47f9f0029003700b5082200d6
:10434000d5b79f000d58a30002003a00c009220013
:10435000d0b79f0014002000050020006033b80093
:104360008fa897008100e900050033000402d00007
:104370008582d2000683d2008783d200f9ff3700fe
:104380000800be000a01be00b6f307006f0060001f
:104390005fb19700624078001000370014002000e1
:1043a000050020006033b8008c0178008301e9002b
:1043b000050033000402d0008582d2000683d200bb
:1043c0008783d200f9ff37000800be000a01be0053
:1043d000a4f30700674060000043b000c07f9f0067
:1043e0004f7a97000400fb00efb0970033000700fe
:1043f000e10f400003003200afb297008502e800f1
:10440000a5b79f001fa897006800500090af9f00bd
:104410008fa89700e480500081af9f00630656008c
:10442000d0ff2f003fb197000090b900ffa1970087
:104430000080410063005000800f5600a4ff3a0046
:104440000d38a300100032001fa297000400e00006
:104450000d0034000006eb00efb0970000022000d2
:1044600016000700e10f400003003200afb29700d2
:104470008502e800a5b79f000c06e8001fa0970082
:10448000800f5600f4ff3a007fb19700b2407800e9
:10449000f2b79f00c17f9f000104e00014fb3a00c7
:1044a0002fb097004f0778004f06be004f05be00a3
:1044b0004f04be008f03b10000000600889fbe00bd
:1044c0000001780001047800b10090000118a300f9
:1044d0003d0032000198a30003003a00180090004c
:1044e0000000e00038003a000190a000310498007c
:1044f00082047800f90fb200180090000000e0007c
:1045000002003a0028009000000c7800ea8f540066
:1045100006003a00380090000078a30003003a003b
:1045200088007800d0002000e4ff07009800900089
:1045300058009000808f50000b0032000100e8000e
:10454000100498001800780009587800000c7800d2
:1045500011c0b3004019220001487800ea8f5400ce
:104560000600320019003700880078000940780002
:10457000a200070080047800140037003800900083
:104580000088a3001100320018019000a8009000dc
:10459000480090006eef070098009000810f5000d7
:1045a00004003200380090000003b300300498008b
:1045b0008084eb000000eb001004980028009000bd
:1045c000000c7800010037008084eb0009007800bf
:1045d0004f04be0000000600881f78000004780029
:1045e000b00090000148a30007003a000108a300b2
:1045f000050032000198a30008003200100090006e
:104600000000e00005003200380090000040a000eb
:10461000300498008080eb00200037000190a1005a
:1046200031049800180090000000e00006003400fb
:104630000000e9001004980018007800b080fb002a
:10464000000c780006003700380090000068a300d6
:10465000edff3a0008007800ab000700800078000a
:10466000380090000078a3000c003a00fa8f500048
:1046700008003a00280090000000e000e2ff32004d
:10468000180090000000e80010049800180ce900e1
:10469000ddff3700ed8f5000e2ff320001007800af
:1046a0004f0478000000060080017800e10f400010
:1046b00017003200310090000008a30014003200ff
:1046c0000098a30012003a00210290000400e000cc
:1046d0000f0032001101900051009000800f510036
:1046e0000b00320011007800840f500002003a00e5
:1046f0008008e800020037000200e80090009800ff
:104700001100e900800878000348780001003700b4
:104710008081eb000300780000000600889fbe0047
:104720008a1f780000047800300090006300600069
:104730002400320008007800c1000700380590000e
:1047400080ef2f00000065003004980028009000e2
:104750000000e00004003200e804650002003a00b6
:10476000f000070029049800480090002fef070090
:10477000e10f400013003200b80090000102b200c7
:1047800010003a000ac8a30018003200800d810012
:104790000000e0001500320000017800810478007c
:1047a000012a200012289000880f500007003200d4
:1047b0004205b0004905b000818f54000b00320063
:1047c000f8ff37000080eb00090037000200780096
:1047d0001fef0700800d8100090040008000eb0002
:1047e0001128980001007800010037000000eb005c
:1047f0004f0578004f04be00000006000200fa00da
:10480000889fbe00a0ff9f0001047800b1009000c7
:10481000810478000904b200020032000000fb00ad
:10482000360037000118a30005003a000103b30069
:1048300031049800190498000080eb002f00370025
:10484000580090000000e00006003a004800900088
:1048500012002000e6805700bdee07001904980002
:1048600024003700280090000000e00008003a0013
:104870000019220020049800000c7800200020007d
:1048800050049800100498000130a00031049800f2
:1048900018019000a800900048009000acee0700be
:1048a00028009000000c78000080eb0010049800b5
:1048b00018007800aff8970001587800000c7800d5
:1048c0002ff89700ea4f50000a003a003800900095
:1048d0000088a3000700320018019000a800900093
:1048e000480090009aee070019049800a800900074
:1048f000010c7800aff897000100fb004f04be00e8
:104900000080fa00000006000200fa00889fbe0046
:104910008a1f7800000478000000eb001004980063
:10492000380090008080eb000008a3003f003200b8
:10493000401922001004e00010003200090b220090
:104940006a0b22001a0078006c0545002010b200a6
:1049500021102000810f500002003a000900780069
:1049600037000700ec844400400d2200808f540083
:10497000f4ff3a00401922000048eb004800900084
:10498000580190000200e0000d003a001204980067
:1049900012002000e8805700b6ee0700e10f50003b
:1049a00003003a000ff897008080fb001f003700db
:1049b000380090000040a00030049800120037003a
:1049c000a8009000abee0700100498000000e00083
:1049d00003003200e10f40000d003a0003003700f1
:1049e000380090000040a00002003700380090001e
:1049f0000003b30030049800a8009000010c780078
:104a00000000eb00100498008080eb0007003700e6
:104a1000a8009000010c78000000e9001004980044
:104a200001007800b080fb00000c780001007800e5
:104a30004f0578004f04be000080fa000000060019
:104a4000881f780000047800300090000008a30060
:104a500007003200800078000120b20004003a0014
:104a600011049800a8009000010c7800170037008e
:104a70000018a300190032000098a30017003200ac
:104a8000a80090000100e00014003200180190001e
:104a90000200e00011003200480090002cee0700f8
:104aa00098009000810f5000030032003800900001
:104ab0000003b300300498000000eb0010049800dd
:104ac00028009000000c7800380090000058a300e7
:104ad000020032000080eb00010037000000eb0014
:104ae0004f04780000000600710d81000100e00015
:104af0000300320011007800700d890003003700b8
:104b000020002000f4ed070080007800e18f4000d5
:104b100002003a00906e26001045880001007800df
:104b200000000600710d810001087800700d8900f9
:104b3000000006004a00fa00889fbe008a9fbe005f
:104b40008c9fbe000040eb00204f98000040eb001f
:104b5000104f98000040eb00004f98000000eb0061
:104b6000300798000000eb002007980090a2020098
:104b70000000000000b4020000000000e0ce880049
:104b8000e0ce8000ea0f500003003a000000eb0086
:104b9000300798000200370010002000300798000e
:104ba0003e0090000000e000020032004678020063
:104bb00000000000767d02000000000040c7bf003a
:104bc000614060000004e000020032004007a900dc
:104bd0000000fe0013002000e2192200e1ff2f0078
:104be000f0072000924402000000000010002000a6
:104bf00050ff88008002200040ff880080022000d3
:104c000030ff88008000200020ff880041ff8000e6
:104c100030ff80000088b9000000400010ff8800cd
:104c20003e0090000000e0002c003200786c020092
:104c30000000000053ff800020ff80000002780089
:104c400020ff80008003780031ff800020ff80007b
:104c50000088b9000004780041ff800020ff800038
:104c60000088b9008004780031ff800020ff8000b8
:104c70000088b90080007800001e2000010050006c
:104c800022002000110009000200d8000005780071
:104c900041ff800020ff80000088b900800078007c
:104ca000002820000100500022002000110009000f
:104cb0000200d8000303780084027800070278001d
:104cc00088017800090178008a007800a66b02004c
:104cd00000000000646c0200000000003e00900034
:104ce0000000e0000b003200a8820200000000007b
:104cf00081052000c02f2c00c479020000000000b4
:104d0000dc790200000000000000e000fcff3a0037
:104d10000f0037004e7b0200000000000004e0009e
:104d200002003a00a8820200000000008105200075
:104d3000c02f2c00667a0200000000007e7a02007c
:104d4000000000000000e000fcff3a000000370017
:104d50003e0090000000e000e700320070003700e5
:104d6000e87e020000000000204f9800dc7e020078
:104d700000000000104f98001e4890000004e00062
:104d8000030032001e489000e84f500064003a00d3
:104d9000ae4890000e48900080cf50006000320076
:104da0002e4890000000fb006101b900521f9800de
:104db000631f980090002000010020005e19900001
:104dc000ee199000800f5100818f590048003e007d
:104dd0005e189000ee189000006001003600370069
:104de000080037000c0037001000370014003700af
:104df000180037001c00370020003700240037005f
:104e0000280037008025200020008900c0122000e3
:104e1000100089003a00370080252000200089001a
:104e2000802520001000890035003700c0122000c6
:104e30002000890080252000100089003000370004
:104e4000802520002000890080da2f0010008900d2
:104e50002b0037000000eb00200089000000eb0071
:104e6000100089002600370080da2f00200089001a
:104e700080252000100089002100370080da2f00f3
:104e80002000890040ed2f00100089001c00370031
:104e900080da2f002000890080da2f0010008900be
:104ea0001700370040ed2f002000890080da2f0026
:104eb0001000890012003700c0fd2100104078006a
:104ec0000004e00005003a000c740200000000003d
:104ed000c1fd210010c0b3008048780001f5210019
:104ee00040b122002a7402000000000004003700d4
:104ef0000000eb00100089001000810020008900f4
:104f0000ae489000014f980010008100a6a2020058
:104f100000000000200081002aa302000000000021
:104f20008062210064790200000000000000e000bf
:104f30008bff320075003700e87e020000000000a1
:104f4000204f9800dc7e020000000000104f980007
:104f50001e4890000004e000030032001e4890004c
:104f6000e84f500064003a00ae4890000e489000b0
:104f700080cf5000600032002e4890000000fb00ff
:104f80006101b900721f980003279800900020006b
:104f9000010020007e1990008e219000800f5100aa
:104fa000818f590048003e007e1890008e209000ae
:104fb0000060010036003700080037000c003700a1
:104fc0001000370014003700180037001c003700ad
:104fd00020003700240037002800370080252000fb
:104fe00020008900c0122000100089003a0037001c
:104ff00080252000200089008025200010008900e5
:1050000035003700c01220002000890080252000d4
:105010001000890030003700802520002000890022
:1050200080da2f00100089002b0037000000eb0011
:10503000200089000000eb001000890026003700e6
:1050400080da2f00200089008025200010008900d0
:105050002100370080da2f002000890040ed2f006a
:10506000100089001c00370080da2f002000890022
:1050700080da2f00100089001700370040ed2f0064
:105080002000890080da2f0010008900120037000c
:10509000c0fd2100104078000004e00005003a0047
:1050a0000c74020000000000c1fd210010c0b3001c
:1050b0008048780001f5210040b122002a740200e6
:1050c00000000000040037000000eb001000890021
:1050d0001000810020008900ae489000014f980028
:1050e00010008100a6a20200000000002000810044
:1050f0002aa302000000000080622100067a02005c
:10510000000000000000e0008bff32008062210000
:10511000104078000004e0004b053d000000eb006b
:105120005000890080622100104078000000fb00e0
:105130000000ea006101b900f0fb2f00f1ff2f0031
:10514000020140008381480012279800232798001d
:1051500060032000010020001e219000ae2190007d
:10516000800f5100818f5900ff043e001e209000e7
:10517000ae2090000060010097003700fa0437006d
:10518000f904370064013700ac013700f60437003a
:10519000f5043700f404370030023700f20437001a
:1051a000f10437005902370096023700ed0237004c
:1051b0002d0337006d033700b5033700ea043700cd
:1051c000e9043700e804370031043700e60437000b
:1051d00049043700e4043700e3043700e2043700f1
:1051e000e1043700e0043700df043700de04370055
:1051f000dd043700dc043700160037001e013700dd
:10520000d9043700d8043700d7043700d604370054
:10521000ad013700d4043700d3043700d20437007f
:10522000d1043700d0043700cf043700ce04370054
:10523000cd043700cc043700cb043700ca04370054
:10524000c9043700bb033700d1033700c604370059
:10525000470437003e0090000000e00010003200dc
:10526000110020000000eb00e87f020000000000b9
:10527000c0ff88001100200010002000e87f02001d
:1052800000000000b0ff8800110020002000200076
:10529000e87f020000000000a0ff88001a0037002d
:1052a0004e7b0200000000000004e0000700320016
:1052b0000000eb00c0ff88000000eb00b0ff88009a
:1052c0000000eb00a0ff88000f0037001100200055
:1052d0000000eb00e87f020000000000c0ff880033
:1052e0001100200010002000e87f020000000000f4
:1052f000b0ff88001100200020002000e87f02009d
:1053000000000000a0ff880052008100c0ff800064
:105310008040780000c0eb0080c06000808a2000e0
:10532000017178000200e8005000890052008100fd
:10533000c0ff80004880de0080407800808a200026
:10534000017178000200e8005000890052008100dd
:10535000b0ff80008040780000c0eb0080c060009b
:10536000808a2000017178000200e8005000890066
:1053700052008100b0ff80004880de00804078004d
:10538000808a2000017178000200e8005000890046
:1053900052008100a0ff80008040780000c0eb0038
:1053a00080c06000808a2000017178000200e8005f
:1053b0005000890052008100a0ff80004880de007c
:1053c00080407800808a2000017178000200e800a7
:1053d00050008900640437003e0090000000e000a7
:1053e000110032006e004700ec8202000000000055
:1053f0006e00470080007800a0fc21001101be0073
:105400000288be0064004000e48040001101be003c
:105410000288be0064004000e48040001101be002c
:105420000288be001e0037004e7b02000000000014
:105430000004e0000a0032006000b80050fe88005e
:1054400061fe88006000b80090fe8800a1fe880020
:105450006000b80070fe880081fe880010003700f0
:105460007a004700ec820200000000007a0047004a
:1054700080007800a0fc21001101be000288be005f
:1054800064004000e48040001101be000288be00bc
:1054900064004000e48040001101be000288be00ac
:1054a000a0fc210060079800520081006e0090006f
:1054b00090407800808a2000017178000200e800a6
:1054c000500089006e0090000000e800600798001e
:1054d000520081006e00900090407800808a200089
:1054e000017178000200e800500089006e00900011
:1054f0000000e80060079800520081006e009000f4
:1055000090407800808a2000017178000200e80055
:10551000500089006e0090000000e80060079800cd
:10552000520081006e00900090407800808a200038
:10553000017178000200e80050008900e0fc2100c1
:1055400060079800520081006e0090009040780043
:10555000808a2000017178000200e8005000890074
:105560006e0090000000e800600798005200810083
:105570006e00900090407800808a200001717800d1
:105580000200e800500089006e0090000000e80072
:1055900060079800520081006e00900090407800f3
:1055a000808a2000017178000200e8005000890024
:1055b0006e0090000000e800600798005200810033
:1055c0006e00900090407800808a20000171780081
:1055d0000200e8005000890020fd210060079800cb
:1055e000520081006e00900090407800808a200078
:1055f000017178000200e800500089006e00900000
:105600000000e80060079800520081006e009000e2
:1056100090407800808a2000017178000200e80044
:10562000500089006e0090000000e80060079800bc
:10563000520081006e00900090407800808a200027
:10564000017178000200e800500089006e009000af
:105650000000e80060079800520081006e00900092
:1056600090407800808a2000017178000200e800f4
:1056700050008900bc0337004e7b02000000000090
:105680000004e0001300320038b402000000000003
:1056900020079800520081002e0090008040780082
:1056a000808a2000017178000200e8005000890023
:1056b000520081002e0090004800de0080407800fb
:1056c000808a2000017178000200e8005000890003
:1056d000a503370052008100e0c2bf000080fb003c
:1056e0000000d1006140600080407800808a200086
:1056f000017178000200e80050008900520081002a
:10570000818a20000040eb0000f178000200e800f0
:1057100050008900940337003e0090000000e00034
:105720000b003200e000220064790200000000005b
:105730000000e000fbff3200d0002200647902008c
:10574000000000000000e000fbff32000a0037000c
:10575000e0002200067a0200000000000000e000e5
:10576000fbff3200d0002200067a02000000000099
:105770000000e000fbff3200e00022001040780053
:105780008080fb00d0002200104078000000fb0069
:105790004800dd0000804000100089003e009000bd
:1057a0000000e0000b003200e000220064790200fb
:1057b000000000000000e000fbff3200d0002200eb
:1057c00064790200000000000000e000fbff3200ee
:1057d0000a003700e0002200067a02000000000004
:1057e0000000e000fbff3200d0002200067a020039
:1057f000000000000000e000fbff3200e00022009b
:10580000104078008080fb00d0002200104078001b
:105810000000fb004800dd000080400020008900ff
:1058200010008100a6a202000000000020008100fc
:105830002aa30200000000004b0337005200810041
:10584000100081008040780000c0eb0080c0600044
:10585000808a2000017178000200e8005000890071
:1058600052008100100081004880de0080407800f6
:10587000808a2000017178000200e8005000890051
:1058800052008100200081008040780000c0eb00c1
:1058900080c06000808a2000017178000200e8006a
:1058a0005000890052008100200081004880de0005
:1058b00080407800808a2000017178000200e800b2
:1058c00050008900280337003e0090000000e000ef
:1058d0003d0032004e7b0200000000000004e000aa
:1058e00039003200c2fe2100e1fe210000ff21004c
:1058f0006cb70200000000005200810080ff8000b1
:105900008040780000c0eb0080c06000808a2000ea
:10591000017178000200e800500089005200810007
:1059200080ff80004880de0080407800808a200070
:10593000017178000200e8005000890052008100e7
:1059400070ff80008040780000c0eb0080c06000e5
:10595000808a2000017178000200e8005000890070
:105960005200810070ff80004880de008040780097
:10597000808a2000017178000200e8005000890050
:105980005200810060ff80008040780000c0eb0082
:1059900080c06000808a2000017178000200e80069
:1059a000500089005200810060ff80004880de00c6
:1059b00080407800808a2000017178000200e800b1
:1059c00050008900e802370052008100818a2000df
:1059d0000040eb0000f178000200e8005000890070
:1059e00052008100818a20000040eb0000f1780025
:1059f0000200e8005000890052008100818a2000e6
:105a00000040eb0000f178000200e800500089003f
:105a100052008100818a20000040eb0000f17800f4
:105a20000200e8005000890052008100818a2000b5
:105a30000040eb0000f178000200e800500089000f
:105a400052008100818a20000040eb0000f17800c4
:105a50000200e80050008900c30237003e009000b9
:105a60000000e000c0023200500081008000780099
:105a7000b08a20000080400026b302000000000031
:105a8000c100220010c0b30080487800520081009d
:105a900050ff80008040780000c0eb0080c06000b4
:105aa000808a2000017178000200e800500089001f
:105ab0005200810040ff80008040780000c0eb0071
:105ac00080c06000808a2000017178000200e80038
:105ad000500089005200810030ff80008040780033
:105ae00000c0eb0080c06000808a20000171780057
:105af0000200e800500089005100810010ff800082
:105b00000080400050008900970237003e0090005e
:105b10000000e0000b003200e00022006479020087
:105b2000000000000000e000fbff3200d000220077
:105b300064790200000000000000e000fbff32007a
:105b40000a003700e0002200067a02000000000090
:105b50000000e000fbff3200d0002200067a0200c5
:105b6000000000000000e000fbff3200e000220027
:105b7000104078000000fb00401f9800ce199000f4
:105b8000e88f5100040032004e189000e90f5000d9
:105b90000a003200120037003e0090000000e000d2
:105ba00071023200d0002200104078000000fb009b
:105bb000c29b0200000000006b0237003e00900014
:105bc0000000e00068023200d0002200104078009f
:105bd0000000fb00029c020000000000620237008f
:105be000d0002200104078008000fb00e00022007e
:105bf000104078000000fb000a990200000000003d
:105c0000590237003e0090000000e00056023200ca
:105c100046780200000000005a78020000000000f0
:105c20008040eb0000ccb3006e7802000000000062
:105c30000000eb00400089001f0037004000810099
:105c40000000a200610060000004e0000c003200cf
:105c500058008100400081008040e80000ccb30083
:105c60006e7802000000000080407800808a2000ea
:105c7000017478000800e800500089000b0037002c
:105c800058008100400081008040e90000ccb30052
:105c90006e7802000000000080407800808a2000ba
:105ca000017478000800e80050008900400081007d
:105cb0000000e8004000890040008100e50f50002e
:105cc000deff3400d0002000400089001f003700b4
:105cd000400081000000a200610060000004e000bc
:105ce0000c00320058008100400081008040e90033
:105cf00000ccb3006e780200000000008040780005
:105d0000808a2000017478000800e80050008900b3
:105d10000b00370058008100400081008040e800ff
:105d200000ccb3006e7802000000000080407800d4
:105d3000808a2000017478000800e8005000890083
:105d4000400081000000e800400089004000810020
:105d5000f00f5000deff3400647802000000000005
:105d6000010237003e0090000000e0001f003200fa
:105d70000000eb004000890018003700400081005f
:105d800074b202000000000030008900520081005f
:105d9000300081008040780000c0eb0080c06000cf
:105da000808a2000017178000200e800500089001c
:105db00052008100300081004880de008040780081
:105dc000808a2000017178000200e80050008900fc
:105dd000400081000000e800400089004000810090
:105de000e70f5000e5ff3400df0137000000eb0053
:105df00040008900180037004000810074b20200a2
:105e00000000000030008900520081003000810055
:105e10008040780000c0eb0080c06000808a2000d5
:105e2000017178000200e8005000890052008100f2
:105e3000300081004880de0080407800808a2000a9
:105e4000017178000200e8005000890040008100e4
:105e50000000e8004000890040008100e90f500088
:105e6000e5ff3400c00137003e0090000000e00074
:105e70001f0032000000eb004000890018003700ce
:105e800040008100bab2020000000000300089002a
:105e900052008100300081008040780000c0eb009b
:105ea00080c06000808a2000017178000200e80054
:105eb0005000890052008100300081004880de00df
:105ec00080407800808a2000017178000200e8009c
:105ed00050008900400081000000e8004000890077
:105ee00040008100e70f5000e5ff34009e013700bd
:105ef0000000eb00400089001800370040008100de
:105f0000bab2020000000000300089005200810097
:105f1000300081008040780000c0eb0080c060004d
:105f2000808a2000017178000200e800500089009a
:105f300052008100300081004880de0080407800ff
:105f4000808a2000017178000200e800500089007a
:105f5000400081000000e80040008900400081000e
:105f6000e90f5000e5ff34007f0137003e0090004c
:105f70000000e0000b003200e00022006479020023
:105f8000000000000000e000fbff3200d000220013
:105f900064790200000000000000e000fbff320016
:105fa0000a003700e0002200067a0200000000002c
:105fb0000000e000fbff3200d0002200067a020061
:105fc000000000000000e000fbff3200e0002200c3
:105fd000104078008080fb00d00022001040780044
:105fe0000000fb004800dd0000804000f0ff88005a
:105ff0003e0090000000e0000b003200e0002200b4
:1060000064790200000000000000e000fbff3200a5
:10601000d000220064790200000000000000e000cf
:10602000fbff32000a003700e0002200067a02007f
:10603000000000000000e000fbff3200d000220062
:10604000067a0200000000000000e000fbff3200c2
:10605000e0002200104078008080fb00d000220089
:10606000104078000000fb004800dd000080400088
:1060700000008900f0ff8000f8a30200000000008b
:10608000000081000ca4020000000000360137006f
:10609000f0a30200000000003000890052008100df
:1060a000300081008040780000c0eb0080c06000bc
:1060b000808a2000017178000200e8005000890009
:1060c00052008100300081004880de00804078006e
:1060d000808a2000017178000200e80050008900e9
:1060e00004a402000000000030008900520081007a
:1060f000300081008040780000c0eb0080c060006c
:10610000808a2000017178000200e80050008900b8
:1061100052008100300081004880de00804078001d
:10612000808a2000017178000200e8005000890098
:106130000d0137003e0090000000e0000d0032002d
:106140004e7b0200000000000004e0000900320065
:10615000580081003eb80200000000008040780036
:10616000808a2000017478000800e800500089004f
:10617000fd00370052008100818a20000040eb00c2
:1061800000f178000200e80050008900f6003700b6
:106190000000eb00bab902000000000030008900e6
:1061a00052008100300081008040780000c0eb0088
:1061b00080c06000808a2000017178000200e80041
:1061c0005000890052008100300081004880de00cc
:1061d00080407800808a2000017178000200e80089
:1061e0005000890010002000bab902000000000031
:1061f000300089005200810030008100804078002a
:1062000000c0eb0080c06000808a2000017178002f
:106210000200e80050008900520081003000810037
:106220004880de0080407800808a2000017178007c
:106230000200e8005000890020002000bab90200e6
:106240000000000030008900520081003000810011
:106250008040780000c0eb0080c06000808a200091
:10626000017178000200e8005000890052008100ae
:10627000300081004880de0080407800808a200065
:10628000017178000200e80050008900b600370074
:1062900000632100600798003e0090000000e000cd
:1062a00005003200812520006e009000c4790200b4
:1062b0000000000004003700812520006e009000df
:1062c000667a020000000000500b81003000890057
:1062d00052008100300081008040780000c0eb0057
:1062e00080c06000808a2000017178000200e80010
:1062f000500089009c0037003e0090000000e00044
:1063000099003200a0fd2100647902000000000025
:106310000000e000fbff320080fd210064790200f4
:10632000000000000000e000fbff320060fd2100e3
:1063300064790200000000000000e000fbff320072
:106340005a78020000000000b0fe80000041780092
:10635000c0fe800080407800d0fe8000c878020037
:106360000000000064780200000000007e0037009a
:106370003e0090000000e0007b0032005a780200ee
:10638000000000000000eb00400089000b00370017
:106390004000810080007800808a2000008040005a
:1063a00064790200000000000000e000f8ff320005
:1063b000400081000000e8004000890040008100aa
:1063c000f70f5000f2ff3400200920004000890040
:1063d0000d0037004000810000017800818a200014
:1063e00060f82f0000804000000041006479020046
:1063f000000000000000e000f6ff320040008100d5
:106400000000e800400089004100810040092000b0
:10641000808f5000efff3400400a200040008900c8
:106420000d0037004000810000017800818a2000c3
:1064300070f72f00008040000000410064790200e6
:10644000000000000000e000f6ff32004000810084
:106450000000e8004000890041008100b00a2000ef
:10646000808f5000efff34000000eb0040008900f7
:106470000b00370041008100808a200061417800d4
:10648000400081008040780000cbb300c878020053
:1064900000000000400081000000e800400089008a
:1064a00040008100f70f5000f2ff34002009200067
:1064b000400089000d0037004100810060f82f0086
:1064c00080804000808a2000614178004000810087
:1064d0008040780000cbb300c878020000000000c4
:1064e000400081000000e800400089004100810078
:1064f00040092000808f5000efff3400400a200048
:10650000400089000d0037004100810070f72f0026
:1065100080804000808a2000614178004000810036
:106520008040780000cbb300c87802000000000073
:10653000400081000000e800400089004100810027
:10654000b00a2000808f5000efff340012c0b3006b
:1065500011c9b30000cbb300c878020000000000ee
:1065600064780200000000003e0090000000e0009f
:106570000600320080622100647902000000000001
:106580000000e000fbff32000500370080622100c0
:10659000067a0200000000000000e000fbff32006d
:1065a00080622100104078000004e000ddfa3a002b
:1065b000500081000000e000e5f932003e0090004c
:1065c0000000e0000b003200c00022001040780004
:1065d0000004e00007003200c10022000040eb0090
:1065e00080487800d6b30200000000000000e00000
:1065f000fcff32003e0090000000e0000900320085
:1066000051008100808a2000c4790200000000004f
:10661000dc790200000000000000e000fcff3a000e
:10662000cbf9370051008100808a2000667a020091
:10663000000000007e7a0200000000000000e00080
:10664000fcff3a00c2f93700806221001040780058
:106650000004e000bef934003e0090000000e000bd
:1066600010003200030037008062210064790200cc
:10667000000000008062210010407800ea4f5000c6
:10668000f9ff32008062210010407800ed4f500089
:10669000f5ff32000b00370080622100067a02000d
:1066a000000000008062210010407800ea4f500096
:1066b000f9ff32008062210010407800ed4f500059
:1066c000f5ff32008062210090407800808a20002f
:1066d0000148780010002000500089003e00900022
:1066e0000000e000150032008062210064790200a1
:1066f000000000000000e0000700320052008100ae
:106700008062210090407800808a2000017178002a
:106710000200e800500089008062210010407800eb
:10672000ea4f5000190032008062210010407800ca
:10673000ed4f5000ecff3a0014003700806221005a
:10674000067a0200000000000000e00007003200ae
:10675000520081008062210090407800808a2000f1
:10676000017178000200e800500089008062210079
:1067700010407800ea4f500004003200806221008f
:1067800010407800ed4f5000ecff3a0052008100bd
:10679000818a20000040eb0000f178000200e80050
:1067a00050008900808a20009040780020c6b30005
:1067b00080cf50000d003200808a20009040780089
:1067c00070c6b30080cf500008003200808a2000dd
:1067d000104078000000fb002001020000000000d3
:1067e00080407800808a200001487800808a20005c
:1067f000104078000000fb006101b900f0fb2f00a1
:10680000f1ff2f00020140008381480032279800e9
:106810004327980030032000010020003e21900013
:10682000ce219000800f5100818f590028083e0032
:106830003e209000ce209000006001003300370021
:10684000c1003700e00037001c013700400137006d
:106850006401370083013700db0137007d03370017
:106860009b0337000c0437005404370077043700cb
:106870000a0537008c0537000e0637003206370050
:10688000590637006e0637008c06370016073700aa
:10689000440737007a0737000d0837009b07370099
:1068a000db0737000a0837000908370008083700f7
:1068b00007083700060837000508370004083700c6
:1068c0006800370002083700010837000008370069
:1068d000ff07370084013700fd073700fc0737004a
:1068e000fb073700fa073700f9073700f8073700ca
:1068f000f7073700f6073700f5073700f4073700ca
:10690000f3073700f2073700c60637003e00900055
:106910000000e000180032001100200020002000dc
:10692000e87f020000000000000478001100200051
:1069300010002000e87f02000000000080047800c2
:10694000110020000000eb00e87f020000000000c2
:10695000881f7800891f7800801f780050352c0030
:10696000801f7800808a20002812020000000000aa
:10697000e8875700200037004e7b0200000000002f
:106980000004e00005003200818a200022362c003d
:1069900009000900b25878001700370011002000e4
:1069a00020002000e87f02000000000000047800c2
:1069b0001100200010002000e87f0200000000000d
:1069c00080047800110020000000eb00e87f020046
:1069d00000000000881f7800891f7800801f780061
:1069e00050352c00801f7800808a20002812020079
:1069f00000000000e88757003e0090000000e00023
:106a00000c003200808a2000fc0f02000000000011
:106a100080007800808a2000c47902000000000015
:106a2000dc790200000000000000e000fcff3a00fa
:106a3000c7f83700808a2000fc0f02000000000029
:106a400080007800808a2000667a02000000000042
:106a50007e7a0200000000000000e000fcff3a0027
:106a6000bbf837004e7b0200000000000004e0008d
:106a70000e0032005eb40200000000000004780046
:106a800038b4020000000000881f7800801f7800e2
:106a9000c0362c00801f7800808a20002812020057
:106aa00000000000e68757000c003700e0c2bf007e
:106ab0000080fb000000d100614060000080fb000e
:106ac000801f7800a0372c00801f7800808a20006b
:106ad0002812020000000000e48757003e009000ea
:106ae0000000e0000c003200808a2000fc0f020051
:106af0000000000080007800808a2000c479020035
:106b000000000000dc790200000000000000e0004e
:106b1000fcff3a008ef83700808a2000fc0f02004c
:106b20000000000080007800808a2000667a020061
:106b3000000000007e7a0200000000000000e0007b
:106b4000fcff3a0082f83700a0ff2100801f780088
:106b500010382c00801f7800808a20000810020066
:106b600000000000e48757003e0090000000e000b5
:106b70000c003200d0ff8000c29b02000000000029
:106b80003100200070382c00c479020000000000a1
:106b9000dc790200000000000000e000fcff3a0089
:106ba0006bf837003100200070382c00667a020044
:106bb000000000007e7a0200000000000000e000fb
:106bc000fcff3a0062f83700e6c2bf000080fb001d
:106bd0004600de00614060000081fb00e7c2bf00ac
:106be0000080fb000000d100614060000080fb00dd
:106bf0000000400080007800e7c2bf0061406000f4
:106c00000080fb0000804000000040008000780011
:106c1000e6c2bf000080fb004700de000080fb00f2
:106c2000008040000000400000004100e0ce8800ed
:106c3000e0ce8000801f7800b0382c00801f7800e4
:106c4000808a20002812020000000000e48757001c
:106c50003e0090000000e0000c003200808a20001e
:106c6000fc0f02000000000080007800808a2000f5
:106c7000c479020000000000dc790200000000007e
:106c80000000e000fcff3a0031f83700808a200065
:106c9000fc0f02000000000080007800808a2000c5
:106ca000667a0200000000007e7a02000000000008
:106cb0000000e000fcff3a0025f837004000220009
:106cc000801f780020002200801f780020392c00cf
:106cd000801f7800808a2000081002000000000059
:106ce000e687570010008100a6a202000000000005
:106cf000200081002aa30200000000003e00900056
:106d00000000e0000900320031002000b0392c0002
:106d1000c479020000000000dc79020000000000dd
:106d20000000e000fcff3a0009f8370031002000c5
:106d3000b0392c00667a0200000000007e7a020062
:106d4000000000000000e000fcff3a0000f83700ff
:106d50002000810011008100801f7800811f7800d1
:106d6000f0392c00801f7800808a20002812020051
:106d700000000000e68757003e0090000000e000a1
:106d80000c003200808a2000fc0f0200000000008e
:106d900080007800808a2000c47902000000000092
:106da000dc790200000000000000e000fcff3a0077
:106db000e7f73700808a2000fc0f02000000000087
:106dc00080007800808a2000667a020000000000bf
:106dd0007e7a0200000000000000e000fcff3a00a4
:106de000dbf73700a0ff2100801f7800903a2c00cd
:106df000801f7800808a2000081002000000000038
:106e0000e48757003e0090000000e0000c003200d4
:106e1000d0ff8000029c0200000000003100200032
:106e2000f03a2c00c479020000000000dc79020076
:106e3000000000000000e000fcff3a00c4f737004b
:106e400031002000f03a2c00667a020000000000b9
:106e50007e7a0200000000000000e000fcff3a0023
:106e6000bbf737003e0090000000e000b8f73200aa
:106e7000e87e0200000000008084fb00dc7e02004f
:106e8000000000000084fb00d07e02000000000033
:106e90000080fb00891f7800881f7800801f780021
:106ea000303b2c00801f7800808a200028120200ce
:106eb00000000000e8875700808a2000fc0f0200d5
:106ec0000000000080007800808a2000c479020061
:106ed00000000000dc790200000000000000e0007b
:106ee000fcff3a009af737003e0090000000e000f7
:106ef000160032004e7b0200000000000004e0009b
:106f00001200320016b802000000000000047800f1
:106f1000eeb702000000000080047800c6b702004f
:106f200000000000881f7800891f7800801f78000b
:106f3000403e2c00801f7800808a2000281202002a
:106f400000000000e887570004003700838a200013
:106f5000103f2c0009000900b05978003e00900055
:106f60000000e0000c003200808a2000fc0f0200cc
:106f70000000000080007800808a2000c4790200b0
:106f800000000000dc790200000000000000e000ca
:106f9000fcff3a006ef73700808a2000fc0f0200e9
:106fa0000000000080007800808a2000667a0200dd
:106fb000000000007e7a0200000000000000e000f7
:106fc000fcff3a0062f737003e0090000000e0004e
:106fd000f600320011002000b03f2c00c4790200fe
:106fe00000000000dc790200000000000000e0006a
:106ff000fcff3a0011022000d03f2c00c4790200af
:1070000000000000dc790200000000000000e00049
:10701000fcff3a0011032000f0412c00c47902006b
:1070200000000000dc790200000000000000e00029
:10703000fcff3a004e7b0200000000000004e0006c
:10704000090032001102200010452c00c479020012
:1070500000000000dc790200000000000000e000f9
:10706000fcff3a0008003700f102200030472c00f6
:10707000c479020000000000dc790200000000007a
:107080000000e000fcff3a0051022000304a2c00d2
:10709000c479020000000000dc790200000000005a
:1070a0000000e000fcff3a00e1022000904c2c00c0
:1070b000c479020000000000dc790200000000003a
:1070c0000000e000fcff3a00e1022000804f2c00ad
:1070d000c479020000000000dc790200000000001a
:1070e0000000e000fcff3a002103200070522c0059
:1070f000c479020000000000dc79020000000000fa
:107100000000e000fcff3a00f1012000a0552c0037
:10711000c479020000000000dc79020000000000d9
:107120000000e000fcff3a004e7b0200000000007f
:107130000004e0000800320081012000a0572c006c
:10714000c479020000000000dc79020000000000a9
:107150000000e000fcff3a008101200030592c00c3
:10716000c479020000000000dc7902000000000089
:107170000000e000fcff3a0081022000c05a2c0011
:10718000c479020000000000dc7902000000000069
:107190000000e000fcff3a00f1042000505d2c00ec
:1071a000c479020000000000dc7902000000000049
:1071b0000000e000fcff3a00f102200050622c00c9
:1071c000c479020000000000dc7902000000000029
:1071d0000000e000fcff3a003103200050652c0065
:1071e000c479020000000000dc7902000000000009
:1071f0000000e000fcff3a001102200090682c0023
:10720000c479020000000000dc79020000000000e8
:107210000000e000fcff3a00d1012000b06a2c0021
:10722000c479020000000000dc79020000000000c8
:107230000000e000fcff3a0011022000906c2c00de
:10724000c479020000000000dc79020000000000a8
:107250000000e000fcff3a0011032000b06e2c009b
:10726000c479020000000000dc7902000000000088
:107270000000e000fcff3a0011032000d0712c0058
:10728000c479020000000000dc7902000000000068
:107290000000e000fcff3a0001022000f0742c0026
:1072a000c479020000000000dc7902000000000048
:1072b0000000e000fcff3a001103200000772c00e2
:1072c000c479020000000000dc7902000000000028
:1072d0000000e000fcff3a0021032000207a2c008f
:1072e000c479020000000000dc7902000000000008
:1072f0000000e000fcff3a004e7b020000000000ae
:107300000004e00008003200f1012000507d2c0054
:10731000c479020000000000dc79020000000000d7
:107320000000e000fcff3a00c1022000507f2c006a
:10733000c479020000000000dc79020000000000b7
:107340000000e000fcff3a005102200020822c00e7
:10735000c479020000000000dc7902000000000097
:107360000000e000fcff3a00b102200080842c0005
:10737000c479020000000000dc7902000000000077
:107380000000e000fcff3a00a102200040872c0032
:10739000c479020000000000dc7902000000000057
:1073a0000000e000fcff3a0069f637001100200001
:1073b000b03f2c00667a0200000000007e7a0200d6
:1073c000000000000000e000fcff3a004e7b0200dd
:1073d000000000000004e00008003a0091012000d5
:1073e000f0892c00667a0200000000007e7a02001c
:1073f000000000000000e000fcff3a004e7b0200ad
:10740000000000000004e0000900320091012000ab
:10741000908b2c00667a0200000000007e7a020049
:10742000000000000000e000fcff3a000800370008
:1074300071022000308d2c00667a020000000000ee
:107440007e7a0200000000000000e000fcff3a002d
:10745000d1012000b08f2c00667a020000000000ed
:107460007e7a0200000000000000e000fcff3a000d
:107470006102200090912c00667a0200000000005a
:107480007e7a0200000000000000e000fcff3a00ed
:107490006102200000942c00667a020000000000c7
:1074a0007e7a0200000000000000e000fcff3a00cd
:1074b0007101200070962c00667a02000000000026
:1074c0007e7a0200000000000000e000fcff3a00ad
:1074d00001012000f0972c00667a020000000000f5
:1074e0007e7a0200000000000000e000fcff3a008d
:1074f0007102200000992c00667a02000000000052
:107500007e7a0200000000000000e000fcff3a006c
:10751000b1022000809b2c00667a0200000000006f
:107520007e7a0200000000000000e000fcff3a004c
:1075300091012000409e2c00667a020000000000ad
:107540007e7a0200000000000000e000fcff3a002c
:1075500051012000e09f2c00667a0200000000002c
:107560007e7a0200000000000000e000fcff3a000c
:107570009101200040a12c00667a0200000000006a
:107580007e7a0200000000000000e000fcff3a00ec
:1075900091022000e0a22c00667a020000000000a8
:1075a0007e7a0200000000000000e000fcff3a00cc
:1075b0009102200080a52c00667a020000000000e5
:1075c0007e7a0200000000000000e000fcff3a00ac
:1075d0008101200020a82c00667a02000000000033
:1075e0007e7a0200000000000000e000fcff3a008c
:1075f00091022000b0a92c00667a02000000000071
:107600007e7a0200000000000000e000fcff3a006b
:107610004102200050ac2c00667a020000000000fd
:107620007e7a0200000000000000e000fcff3a004b
:10763000d1012000a0ae2c00667a020000000000fc
:107640007e7a0200000000000000e000fcff3a002b
:10765000bff537003e0090000000e000bcf53200ae
:1076600010ff800021ff800032ff800043ff800078
:1076700054ff8000801f7800811f7800821f7800ef
:10768000831f7800841f780080b02c00801f780052
:10769000808a20002812020000000000ec875700ba
:1076a000808a2000fc0f02000000000080007800ab
:1076b000808a2000c479020000000000dc7902000a
:1076c000000000000000e000fcff3a00a0f53700d9
:1076d0003e0090000000e0009df532000080eb00cd
:1076e00000ff88000080eb00f0fe8800e0fd210034
:1076f000801f780000fe2100801f780040fe2100de
:10770000801f780060fe2100801f780080fe21002d
:10771000801f7800a0fe2100801f7800b0b12c00ef
:10772000801f7800808a20000810020000000000fe
:10773000ee87570050ff80000000e00005003a008f
:1077400041ff800030ff80000088b90010ff8800f2
:107750000500370041ff800030ff80000088b9003d
:107760000000400010ff880011ff800000d82000ba
:10777000808f50000b0034001000200050ff880064
:107780008002200040ff88008002200030ff880037
:1077900041ff800030ff80000088b90000004000f9
:1077a00010ff8800786c02000000000000ff8000dd
:1077b000e10f40000a003a0041ff800020ff8000f6
:1077c0000088b900800078000028200001005000e7
:1077d00022002000110009000200d80000ff8800ec
:1077e000f0fe8000e10f40000a003a0031ff800007
:1077f00020ff80000088b90080007800001e200073
:107800000100500022002000110009000200d800f1
:10781000f0fe880053ff800020ff80000002780007
:1078200020ff80008003780031ff800020ff80006f
:107830000088b9000004780041ff800020ff80002c
:107840000088b90000017800f0fe80008000780018
:1078500000ff8000030378008402780007027800ac
:1078600088017800a66b020000000000646c020032
:10787000000000003100200000b32c00c479020099
:1078800000000000dc790200000000000000e000c1
:10789000fcff3a002ef537003e0090000000e000ab
:1078a00009003200e103200040b32c00c47902003b
:1078b00000000000dc790200000000000000e00091
:1078c000fcff3a0008003700e103200040b32c0021
:1078d000667a0200000000007e7a020000000000cc
:1078e0000000e000fcff3a001100200080002000b2
:1078f0000a990200000000006000b800008fbe007e
:107900000400370012002000030020001e0f410079
:107910005e974900f0232400f1002000be0f100004
:10792000ae8f1800f7ff3400ac9b0200000000008f
:107930006000b800008fbe00040037001000200077
:10794000010020001e0f40005e974800f0702200ea
:1079500001002000be0f1000ae8f1800f7ff3400aa
:1079600070b10200000000003e0090000000e00046
:10797000090032009101200030b72c00c4790200c8
:1079800000000000dc790200000000000000e000c0
:10799000fcff3a00eef437009101200030b72c00d4
:1079a000667a0200000000007e7a020000000000fb
:1079b0000000e000fcff3a00e5f43700a0ff2100e2
:1079c000801f7800c0ff2100801f7800d0b82c00f5
:1079d000801f7800808a200008100200000000004c
:1079e000e6875700d0ff800080007800e0ff80002d
:1079f0000a990200000000003e0090000000e00034
:107a0000090032003100200060b92c00c479020066
:107a100000000000dc790200000000000000e0002f
:107a2000fcff3a00caf437003100200060b92c0096
:107a3000667a0200000000007e7a0200000000006a
:107a40000000e000fcff3a00c1f437003e00900067
:107a50000000e000bef432005a780200000000008e
:107a60000000eb00400089001b003700400081004f
:107a70000000a200610060000004e0000a00320083
:107a800048008100400081008040e80000ccb30045
:107a90006e7802000000000080407800808a20009c
:107aa000017478000900370048008100400081001f
:107ab0008040e90000ccb3006e78020000000000b6
:107ac00080407800808a20000174780040008100a6
:107ad0000000e8004000890040008100e50f5000f0
:107ae000e2ff3400d0002000400089001d00370074
:107af000400081000000a200610060000004e0007e
:107b00000b003200400081006704500040008100fb
:107b10008040e90000ccb3006e7802000000000055
:107b200080407800808a2000017478000a003700c5
:107b30004000810067045000400081008040e80060
:107b400000ccb3006e780200000000008040780096
:107b5000808a200001747800400081000000e80065
:107b60004000890040008100f00f5000e0ff340029
:107b70006478020000000000008b200010407800b4
:107b80008000fb00f00f200080806000108b200040
:107b9000104078000000fb004800dd00008140003c
:107ba000e08a2000104078008000fb00f00f2000e9
:107bb00080806000f08a2000104078000000fb0008
:107bc0004800dd0080814000c08a2000104078001d
:107bd0008000fb00f00f200080806000d08a200031
:107be000104078000000fb004800dd0000824000eb
:107bf000a08a2000104078008000fb00f00f2000d9
:107c000080806000b08a2000104078000000fb00f7
:107c10004800dd0080824000808a2000104078000b
:107c20008000fb00f00f200080806000908a200020
:107c3000104078000000fb004800dd00008040009c
:107c4000821f7800831f7800841f7800851f7800ca
:107c5000801f7800a0b92c00801f7800808a200047
:107c60002812020000000000ec875700808a2000e4
:107c7000fc0f02000000000080007800808a2000d5
:107c8000c479020000000000dc790200000000005e
:107c90000000e000fcff3a002df437003e009000a9
:107ca0000000e0003a0032007000200074b20200d0
:107cb00000000000800478006000200074b2020020
:107cc00000000000000578005000200074b202009f
:107cd00000000000800578004000200074b202001f
:107ce00000000000000678003000200074b202009e
:107cf00000000000800678002000200074b202001e
:107d000000000000301f98001000200074b2020034
:107d100000000000000478000000eb0074b20200d4
:107d200000000000891f78008a1f78008b1f7800f0
:107d30008c1f78008d1f7800be189000811f78007e
:107d4000881f7800801f7800d0ba2c00801f780030
:107d5000808a20002812020000000000f2875700ed
:107d6000808a2000fc0f02000000000080007800e4
:107d7000808a2000c479020000000000dc79020043
:107d8000000000000000e000fcff3a00f0f33700c4
:107d90009000200074b2020000000000000478008f
:107da0008000200074b2020000000000800478000f
:107db0007000200074b2020000000000000578008e
:107dc0006000200074b2020000000000800578000e
:107dd0005000200074b2020000000000000678008d
:107de0004000200074b2020000000000800678000d
:107df0003000200074b2020000000000201f980034
:107e00002000200074b2020000000000101f980043
:107e10001000200074b2020000000000001f980053
:107e20000000eb0074b2020000000000881f780020
:107e3000891f78008a1f78008b1f78008c1f7800bc
:107e40008d1f78002e199000821f78009e199000d7
:107e5000831f78008e189000811f7800801f7800a3
:107e600090bc2c00801f7800808a2000281202001d
:107e700000000000f6875700808a2000fc0f0200f7
:107e80000000000080007800808a2000667a0200ee
:107e9000000000007e7a0200000000000000e00008
:107ea000fcff3a00aaf337003e0090000000e0001b
:107eb0003a00320070002000bab202000000000058
:107ec0008004780060002000bab2020000000000c8
:107ed0000005780050002000bab202000000000047
:107ee0008005780040002000bab2020000000000c7
:107ef0000006780030002000bab202000000000046
:107f00008006780020002000bab2020000000000c5
:107f10007017980010002000bab2020000000000a4
:107f2000000478000000eb00bab20200000000007c
:107f3000891f78008a1f78008b1f78008c1f7800bb
:107f40008d1f78007e119000821f7800881f7800b6
:107f5000801f7800b0be2c00801f7800808a20002f
:107f60002812020000000000f2875700808a2000db
:107f7000fc0f02000000000080007800808a2000d2
:107f8000c479020000000000dc790200000000005b
:107f90000000e000fcff3a006df337009000200085
:107fa000bab2020000000000000478008000200047
:107fb000bab20200000000008004780070002000c7
:107fc000bab2020000000000000578006000200046
:107fd000bab20200000000008005780050002000c6
:107fe000bab2020000000000000678004000200045
:107ff000bab20200000000008006780030002000c5
:10800000bab20200000000006017980020002000b3
:10801000bab20200000000005017980010002000c3
:10802000bab2020000000000401798000000eb0008
:10803000bab2020000000000881f7800891f780093
:108040008a1f78008b1f78008c1f78008d1f7800a6
:10805000ee119000831f7800de109000811f7800e1
:108060004e119000821f7800801f780070c02c0095
:10807000801f7800808a2000281202000000000083
:10808000f6875700808a2000fc0f020000000000e5
:1080900080007800808a2000667a020000000000dc
:1080a0007e7a0200000000000000e000fcff3a00c1
:1080b00027f3370000002200801f7800e0ff210036
:1080c000801f780090c22c00801f7800808a2000da
:1080d0000810020000000000e6875700f0ff800053
:1080e000f8a3020000000000000081000ca40200c0
:1080f000000000003e0090000000e0000900320097
:108100003100200020c32c00c479020000000000d0
:10811000dc790200000000000000e000fcff3a00f3
:108120000bf337003100200020c32c00667a0200d8
:10813000000000007e7a0200000000000000e00065
:10814000fcff3a0002f3370004a402000000000024
:1081500000047800f0a3020000000000881f7800ef
:10816000801f780060c32c00801f7800808a200068
:108170002812020000000000e68757003e00900031
:108180000000e0000c003200808a2000fc0f02009a
:108190000000000080007800808a2000c47902007e
:1081a00000000000dc790200000000000000e00098
:1081b000fcff3a00e6f23700808a2000fc0f020044
:1081c0000000000080007800808a2000667a0200ab
:1081d000000000007e7a0200000000000000e000c5
:1081e000fcff3a00daf237003e0090000000e000a9
:1081f000090032003100200000c42c00c4790200c4
:1082000000000000dc790200000000000000e00037
:10821000fcff3a00080037003100200000c42c00a9
:10822000667a0200000000007e7a02000000000072
:108230000000e000fcff3a000000fe00c4f237003e
:108240000000eb00a6a20200000000000000eb000e
:108250002aa30200000000008000eb008000200044
:108260000a990200000000003e0090000000e000bb
:10827000090032003100200040c42c00c479020003
:1082800000000000dc790200000000000000e000b7
:10829000fcff3a00aef237003100200040c42c0051
:1082a000667a0200000000007e7a020000000000f2
:1082b0000000e000fcff3a00a5f237003e0090000d
:1082c0000000e0004e00320020ff2100801f7800f7
:1082d00080c42c00801f7800808a200008100200d3
:1082e00000000000e4875700c0fd21001040780026
:1082f0000004e00005003a000c74020000000000d9
:10830000c1fd210010c0b3008048780093ff8000b9
:10831000331798003e109000e30f50001b0032000e
:10832000be109000e38f500007003c003e1190000b
:10833000e10f51000b003200be119000e28f51009e
:108340000d003200200037003e109000e40f500076
:1083500013003200be109000e58f5000150032006f
:1083600019003700018420000000eb002a7402008d
:108370000000000019003700016e2000408420003a
:108380002a740200000000001400370041d52000cc
:1083900060f220002a740200000000000f00370085
:1083a00041e92000e0c721002a740200000000001b
:1083b0000a00370001f5210040b122002a740200b2
:1083c00000000000050037004074020000000000bb
:1083d000c1fd21000040eb00804878003100200002
:1083e000d0c42c00c479020000000000dc79020037
:1083f000000000000000e000fcff3a0054f23700eb
:1084000031002000d0c42c00667a02000000000079
:108410007e7a0200000000000000e000fcff3a004d
:108420004bf237003e0090000000e0000f003200e9
:108430004e7b0200000000000004e0000b00320050
:108440003eb80200000000000000fb00801f780022
:1084500010c52c00801f7800808a2000281202009e
:1084600000000000e487570004003700828a2000e3
:1084700083c52c0005000900335978003e009000a8
:108480000000e0000c003200808a2000fc0f020097
:108490000000000080007800808a2000c47902007b
:1084a00000000000dc790200000000000000e00095
:1084b000fcff3a0026f23700808a2000fc0f020001
:1084c0000000000080007800808a2000667a0200a8
:1084d000000000007e7a0200000000000000e000c2
:1084e000fcff3a001af2370020002000bab902005f
:1084f000000000008004780010002000bab90200db
:1085000000000000000478000000eb00bab902008f
:1085100000000000891f7800881f7800801f780005
:10852000e0c52c00801f7800808a200028120200fd
:1085300000000000e88757003e0090000000e000c7
:108540000c003200808a2000fc0f020000000000b6
:1085500080007800808a2000c479020000000000ba
:10856000dc790200000000000000e000fcff3a009f
:10857000f7f13700808a2000fc0f020000000000a5
:1085800080007800808a2000667a020000000000e7
:108590007e7a0200000000000000e000fcff3a00cc
:1085a000ebf137003e0090000000e00009003200cf
:1085b00061022000b0c62c00c47902000000000057
:1085c000dc790200000000000000e000fcff3a003f
:1085d0000800370061022000b0c62c00667a020055
:1085e000000000007e7a0200000000000000e000b1
:1085f000fcff3a00f00c8100801f780020c92c009d
:10860000801f7800808a20002812020000000000ed
:10861000e48757003e0090000000e0000c003200ac
:10862000808a2000fc0f020000000000800078001b
:10863000808a2000c479020000000000dc7902007a
:10864000000000000000e000fcff3a00c0f137002d
:10865000808a2000fc0f02000000000080007800eb
:10866000808a2000667a0200000000007e7a020004
:10867000000000000000e000fcff3a00b4f1370009
:108680003e0090000000e000b1f1320060fd2100ea
:10869000801f780080fd2100801f7800a0fd210050
:1086a000801f780030ca2c00801f7800808a20004c
:1086b0000810020000000000e88757005a78020006
:1086c00000000000b0fe800000417800c0fe800085
:1086d00080407800d0fe8000c878020000000000d2
:1086e000647802000000000031002000f0ca2c0075
:1086f000c479020000000000dc79020000000000e4
:108700000000e000fcff3a0091f137003e009000cd
:108710000000e0008ef1320080fd2100801f780013
:10872000a0fd2100801f780030cb2c00801f780036
:10873000808a20000810020000000000e687570031
:10874000c0fe8000d1fe8000801f7800811f78006d
:10875000c0cb2c00801f7800808a200028120200e5
:1087600000000000e6875700808a2000fc0f02000e
:108770000000000080007800808a2000c479020098
:1087800000000000dc790200000000000000e000b2
:10879000fcff3a005a78020000000000c0fe800092
:1087a00080407800d0fe80006e780200000000005b
:1087b0000000fb00b0fe88006478020000000000aa
:1087c000b0fe8000801f780060cc2c00801f7800f5
:1087d000808a20002812020000000000e487570071
:1087e000808a2000fc0f020000000000800078005a
:1087f000808a2000c479020000000000dc790200b9
:10880000000000000000e000fcff3a0050f13700db
:108810003e0090000000e0004df1320020002000fa
:1088200040008900250037005a780200000000004f
:10883000400081008040eb006e78020000000000e4
:108840000000fb00b0fe8800647802000000000019
:10885000b0fe80000000e00015003500b0fe800092
:1088600041008100801f7800811f7800d0cc2c004f
:10887000801f7800808a200028120200000000007b
:10888000e6875700808a2000fc0f020000000000ed
:1088900080007800808a2000c47902000000000077
:1088a000dc790200000000000000e000fcff3a005c
:1088b000400081000080e800400089004100810004
:1088c000e00f2000808f5000d7ff340020f13700e8
:1088d0003e0090000000e00009003200510120003d
:1088e00060cd2c00c479020000000000dc79020099
:1088f000000000000000e000fcff3a0014f1370027
:108900005101200060cd2c00667a020000000000ba
:108910007e7a0200000000000000e000fcff3a0048
:108920000bf137003200f800900188006118e10077
:10893000040032007018e10002003200f0ff2f0046
:10894000030037003119ba008301e900fdff3a0046
:108950003200f90000000600849fbe004220a900fa
:10896000440424006110e1000a0032005404240091
:108970007010e1000700320064042400f5ff2f00ae
:108980000510e10003003200f0ff2f004f02be008f
:10899000000006003200f800203b8800113b8800f0
:1089a000043b88004200f800000e20004220b7007f
:1089b00050052000303b8800a00a2000303b880092
:1089c00061e7a800000000000000000061e7af00c0
:1089d000feff37000000eb004200f9003200f90012
:1089e0004f02be0000000600841f78004220a9004c
:1089f000440024006118e100060032005400240005
:108a00007018e100030032004f027800f0ff2f00e1
:108a1000000006003200f80091018800821f7800f3
:108a20003019bb008301e900fdff3a00213b8800bb
:108a30004f017800123b8800043b88004200f80098
:108a4000000e20004220b70050052000303b880077
:108a5000a00a2000303b880061e7a8000000000069
:108a60000000000061e7af00feff37000000eb00f0
:108a70004200f9003200f9004f02780000000600c1
:108a80000600fa00889fbe008a9fbe008c9fbe0031
:108a9000b67a0200000000005a7b020000000000cd
:108aa00090a2020000000000107902000000000007
:108ab0007000200018b50200000000000040eb002c
:108ac000968602000000000040c7bf0061406000c1
:108ad0000004e000020032004007a9000000fe0090
:108ae00000b4020000000000e0ce8800e0ce80006c
:108af000801f7800c0ce2c00801f7800808a200064
:108b00002812020000000000e4875700808a20003d
:108b1000fc0f02000000000080007800808a200026
:108b2000c479020000000000dc79020000000000af
:108b30000000e000fcff3a00e0ce80000000e00012
:108b400003003a00ba4d020000000000a6033700ff
:108b5000e0ce8000e10f500003003a00e0c10200c7
:108b600000000000a0033700e0ce8000e20f5000bc
:108b700003003a00fa5a0200000000009a0337008e
:108b8000e0ce8000e30f500003003a009a25020077
:108b90000000000094033700e0ce8000e40f500096
:108ba00003003a0046c00200000000008e033700b8
:108bb000e0ce8000e50f500003003a00425502006d
:108bc0000000000088033700e0ce8000e60f500070
:108bd00003003a005e5302000000000082033700e9
:108be000e0ce8000e70f500003003a007c5c0200fa
:108bf000000000007c033700e0ce8000e80f50004a
:108c000003003a00485302000000000076033700da
:108c1000e0ce8000e90f500003003a00acbf020034
:108c20000000000070033700e0ce8000ea0f500023
:108c30000d003a004678020000000000786c020047
:108c40000000000007e2a900e442a800e462a800d6
:108c50003000200018b50200000000009a25020034
:108c60000000000060033700e0ce8000eb0f5000f2
:108c700073013a00808a2000e1cf2c003c000900fb
:108c800031587800808a2000fc0f020000000000ac
:108c900080007800808a2000667a020000000000d0
:108ca0007e7a0200000000000000e000fcff3a00b5
:108cb000808a2000820720008000eb002410020040
:108cc00000000000808a2000b1d32c001b000900a6
:108cd00031587800808a2000fc0f0200000000005c
:108ce00080007800808a2000667a02000000000080
:108cf0007e7a0200000000000000e000fcff3a0065
:108d0000808a2000820720008000eb0024100200ef
:108d1000000000000000eb00204588008162210077
:108d20000040eb00804878002045800080007800fb
:108d3000c090200000804000067a02000000000081
:108d40000000e0000a0032002045800041062000bb
:108d500080804000808a2000e1407800806221000d
:108d600001487800204580000000e8002045880088
:108d70008062210010407800ea4f50000400320069
:108d80008062210010407800ed4f5000e6ff3a006d
:108d9000204580004206200000014100818a200019
:108da0000040eb0000f17800808a2000420620009d
:108db0008000eb002410020000000000c0902000a2
:108dc000104078000000fb0020079800e00420001d
:108dd000ae009000808f5000ad003200e004200013
:108de000ae009000808f50000d003c0080042000f9
:108df000ae009000808f5000c1003200d0042000ef
:108e0000ae009000808f50003f00320060042000d0
:108e1000ae009000808f5000b6003200f70037009f
:108e200000052000ae009000808f50000d00320041
:108e300000052000ae009000808f50001500350026
:108e400020052000ae009000808f50009c00320072
:108e500030052000ae009000808f500047003200a7
:108e6000e6003700808a2000b260020000000000a7
:108e7000a08d2000818a2000811f780071d52c00f0
:108e8000811f78002812020000000000e4875700cc
:108e9000df003700c1902000808a2000801f78000a
:108ea00070d62c00801f780001007800321002007c
:108eb00000000000e4875700808a2000186202004a
:108ec000000000000004e00006003200a08d200039
:108ed000d1d62c0014000900315878005001b1009f
:108ee000cb003700a08d2000818a2000811f7800f0
:108ef00071d52c00811f78002812020000000000ac
:108f0000e4875700c2003700c1902000808a20000b
:108f1000801f780020d82c00801f78000100780086
:108f20003210020000000000e4875700808a200011
:108f3000f8620200000000000004e00006003200b9
:108f4000a08d200081d82c00150009003158780030
:108f50006001b100ae003700a08d2000818a2000a2
:108f6000811f7800e1d92c00811f780028120200af
:108f700000000000e4875700a5003700c1902000e2
:108f8000808a2000801f780030db2c00801f780052
:108f9000010078003210020000000000e487570052
:108fa000808a200018620200000000000004e00037
:108fb00006003200a08d2000d1d62c00140009003c
:108fc000315878005001b10008003700a08d200012
:108fd000818a2000811f780071d52c00811f7800c4
:108fe0002812020000000000e4875700a08d200036
:108ff000fc0f02000000000080007800a08d20001f
:10900000667a0200000000007e7a02000000000084
:109010000000e000fcff3a00c1902000808a2000a0
:10902000801f780090db2c00801f78000100780002
:109030002812020000000000e4875700c0902000c2
:10904000f8620200000000000004e00006003200a8
:10905000a08d200081d82c0015000900315878001f
:109060006001b1006a003700c0902000a18d20008f
:10907000801f7800e0d92c00801f78000100780064
:109080002812020000000000e4875700600037004b
:10909000808a20006c61020000000000a08d20008a
:1090a000818a2000811f7800e1d92c00811f78007f
:1090b0002812020000000000e48757005400370027
:1090c000bc5e020000000000304588003045800092
:1090d000a18d2000801f780030dc2c00801f7800dc
:1090e000010078002812020000000000e487570009
:1090f00047003700705f02000000000044003700a6
:1091000041012000c0dd2c00667a02000000000052
:109110007e7a0200000000000000e000fcff3a0040
:109120002103200010df2c00667a020000000000fe
:109130007e7a0200000000000000e000fcff3a0020
:10914000a102200040e22c00667a0200000000002c
:109150007e7a0200000000000000e000fcff3a0000
:10916000b1012000f0e42c00667a0200000000004b
:109170007e7a0200000000000000e000fcff3a00e0
:10918000d1012000b0e62c00667a02000000000049
:109190007e7a0200000000000000e000fcff3a00c0
:1091a0002102200090e82c00667a020000000000f6
:1091b0007e7a0200000000000000e000fcff3a00a0
:1091c00021032000c0ea2c00667a020000000000a3
:1091d0007e7a0200000000000000e000fcff3a0080
:1091e000a18d2000a0c0b30080487800b18d200080
:1091f0000040eb008048780005003700a08d20007b
:10920000f1ed2c0015000900315878006001b10023
:10921000a08d2000fc0f02000000000080007800fc
:10922000a08d2000667a0200000000007e7a020015
:10923000000000000000e000fcff3a00b5fe37002f
:10924000e0ce8000ec0f5000bb013a00c0022000cd
:10925000801f780050022000801f7800100020003e
:10926000801f7800b0052000801f7800b00120002a
:10927000801f780050ef2c00801f7800808a20002b
:109280002812020000000000ec875700808a2000ae
:10929000fc0f02000000000080007800808a20009f
:1092a000667a020000000000d103200030f02c009c
:1092b000667a0200000000007e7a020000000000d2
:1092c0000000e000fcff3a0070b102000000000066
:1092d0006101200010f42c00667a020000000000fa
:1092e0007e7a0200000000000000e000fcff3a006f
:1092f0000c7402000000000001f5210040b12200c2
:109300002a7402000000000000502300c100200069
:10931000deb302000000000040062000a6a202000a
:1093200000000000400620002aa302000000000008
:10933000786c02000000000016002000850020006c
:1093400084002000031420000214200001052000e6
:10935000000a2000a66b020000000000110020009f
:1093600010002000206c020000000000646c02006d
:1093700000000000a8820200000000001000200091
:10938000c29b02000000000010002000029c0200ae
:109390000000000011002000800020000a99020057
:1093a000000000002100200080f52c00667a0200f9
:1093b000000000007e7a0200000000000000e000d3
:1093c000fcff3a0020002000f47e020000000000b4
:1093d0008004780010002000f47e020000000000ed
:1093e000000478000000eb00f47e020000000000a2
:1093f000891f7800881f7800801f7800b005200042
:10940000801f7800b0012000801f7800b005200088
:10941000801f7800b0012000801f7800b0f52c007c
:10942000801f7800808a20002812020000000000bf
:10943000f0875700808a2000fc0f02000000000027
:1094400080007800808a2000667a02000000000018
:109450007e7a0200000000000000e000fcff3a00fd
:10946000e6c2bf000080fb004600de0061406000f5
:109470000081fb00e7c2bf000080fb000000d100bc
:10948000614060000080fb00000040008000780028
:10949000e7c2bf00614060000080fb000080400028
:1094a0000000400080007800e6c2bf000080fb00a2
:1094b0004700de000080fb0000804000000040000c
:1094c00000004100e0ce8800e0ce8000801f7800e0
:1094d000b0052000801f7800b0012000801f7800b8
:1094e00080f82c00801f7800808a2000281202005b
:1094f00000000000e8875700808a2000fc0f02006f
:109500000000000080007800808a2000667a020057
:10951000000000007e7a0200000000000000e00071
:10952000fcff3a00e87e0200000000008084fb009f
:10953000dc7e0200000000000084fb00d07e020000
:10954000000000000080fb00891f7800881f780061
:10955000801f7800b0052000801f7800b001200037
:10956000801f7800f0f92c00801f7800808a20008e
:109570002812020000000000ec875700808a2000bb
:10958000fc0f02000000000080007800808a2000ac
:10959000667a0200000000007e7a020000000000ef
:1095a0000000e000fcff3a007000200046b202001c
:1095b00000000000800478006000200046b2020035
:1095c00000000000000578005000200046b20200b4
:1095d00000000000800578004000200046b2020034
:1095e00000000000000678003000200046b20200b3
:1095f00000000000800678002000200046b2020033
:1096000000000000100798001000200046b2020081
:1096100000000000000478000000eb0046b20200e9
:1096200000000000891f78008a1f78008b1f7800d7
:109630008c1f78008d1f78009e009000811f78009d
:10964000881f7800801f7800b0052000801f7800f8
:10965000b0012000801f780060fd2c00801f780082
:10966000808a20002812020000000000f6875700c0
:10967000808a2000fc0f02000000000080007800bb
:10968000808a2000667a0200000000007e7a0200d4
:10969000000000000000e000fcff3a007000200025
:1096a000bab20200000000008004780060002000d0
:1096b000bab202000000000000057800500020004f
:1096c000bab20200000000008005780040002000cf
:1096d000bab202000000000000067800300020004e
:1096e000bab20200000000008006780020002000ce
:1096f000bab2020000000000000f78001000200045
:10970000bab2020000000000000478000000eb0084
:10971000bab2020000000000891f78008a1f78009a
:109720008b1f78008c1f78008d1f78009e007800ba
:10973000811f7800881f7800801f7800b005200006
:10974000801f7800b0012000801f780020012d00cc
:10975000801f7800808a200028120200000000008c
:10976000f6875700808a2000fc0f020000000000ee
:1097700080007800808a2000667a020000000000e5
:109780007e7a0200000000000000e000fcff3a00ca
:1097900020002000bab90200000000008004780018
:1097a00010002000bab90200000000000004780098
:1097b0000000eb00bab9020000000000891f780029
:1097c000881f7800801f7800b0052000801f780077
:1097d000b0012000801f780020052d00801f780038
:1097e000808a20002812020000000000ec87570049
:1097f000808a2000fc0f020000000000800078003a
:10980000808a2000667a0200000000007e7a020052
:10981000000000000000e000fcff3a00808a200009
:1098200026b3020000000000d6b3020000000000d2
:109830000000e000fcff3200808a20001040780029
:109840008000fb00800f200000806000b00b8900ca
:10985000808a2000104078000000fb006700600054
:109860004501dd00908a2000104078008000fb0058
:10987000000e2000008060004380de0000007100c8
:10988000a00b8900908a2000104078000000fb00a7
:109890007f0060004300dd00900b8900900b810089
:1098a000a10b8100b20b810083522100801f780040
:1098b000811f7800821f7800b0052000801f78008b
:1098c000b0012000801f780030072d00801f780035
:1098d000030078002812020000000000ec87570007
:1098e00080522100fc0f0200000000008000780080
:1098f00080522100667a0200000000007e7a020099
:10990000000000000000e000fcff3a000000eb0057
:109910002045880003003700204580000000e80053
:10992000204588002145800030062000808f5000af
:10993000f9ff3400a3fe3700e0ce8000ed0f5000a9
:109940001b003a00808a2000fc0f0200000000008b
:1099500080007800808a2000667a02000000000003
:1099600000003700806221006479020000000000de
:109970000000e0000400320011002000806221009d
:10998000667a02000000000080622100067a020070
:10999000000000000000e000f2ff32001100200093
:1099a00080622100c479020000000000edff370052
:1099b000e0ce8000ee0f500003003a00f4520200a7
:1099c0000000000008003700e0ce8000ef0f5000dc
:1099d00003003a001e57020000000000020037009a
:1099e0001e53020000000000ffff37001400fa00c1
:1099f0006000b80040079800510798006000b80068
:109a000020079800310798006000b800008fbe0062
:109a10000000eb00100f98003a0037000000eb0048
:109a2000f47e020000000000000f980010002000eb
:109a3000f47e020000000000700798002000200063
:109a4000f47e020000000000600798000e089000fd
:109a50006101b9004e009000de009000000041005e
:109a60008180490040079800510798007e009000cf
:109a70006101b9002e009000be009000000041007e
:109a80008180490020079800310798006e009000ff
:109a9000cf80de001e0f40005e9748006e009000f1
:109aa000801f78007e019000821f78000e089000d1
:109ab000801f780040142d00801f7800808a2000cd
:109ac0002812020000000000e8875700808a20006a
:109ad000fc0f02000000000080007800808a200057
:109ae000c47902000000000080bb200001002000bb
:109af000deb30200000000001e0890000000e80035
:109b0000100f98001e089000ff0f5000c3ff340094
:109b10004e009000de0090004b09dd004500de00a5
:109b200000007100c588de00c00b89002e00900087
:109b3000be0090004b09dd004500de000000710012
:109b4000c588de00d00b89001e00be004b09dd0079
:109b50004500de0000007100c588de00800078004e
:109b600080d12f0000804000e00b89000080fa00c7
:109b7000000006001800fa00889fbe008a9fbe0001
:109b80000c74020000000000110020008000200082
:109b90000a9902000000000094ff0700e00b81001a
:109ba000d10b8100c20b8100801f7800811f7800db
:109bb000821f780010152d00801f7800808a2000f9
:109bc0002812020000000000e8875700808a200069
:109bd000fc0f02000000000080007800808a200056
:109be000c4790200000000008000eb00800020002b
:109bf0000a990200000000000000eb0040079800f6
:109c0000803e200001002000500798006107980066
:109c1000000037000000eb00f47e020000000000ae
:109c2000300f980010002000f47e020000000000b9
:109c3000200f980020002000f47e020000000000a9
:109c4000100f9800c10b81003e08900001005000e9
:109c5000300f9800d10b81002e08900001005000b9
:109c6000200f9800e10b81001e08900001005000b9
:109c7000100f98001e0890000000e00006003d0054
:109c80009e08900080da2f00808f50000200340080
:109c90000000eb00100f98003e0890006103b9002f
:109ca0003e0890006102b900860078000400780048
:109cb000000db80005b0b9000b01780000014100ab
:109cc00007a0b90000014100820578002e0890002d
:109cd0006104b9002e0890006103b9008800780083
:109ce00006007800000ab80007c0b9000501780036
:109cf0000001410009b0b900000141008202780072
:109d00000a0542008b854a001e0890006104b900d4
:109d10001e0890006103b9008800780006007800f2
:109d2000000ab80007c0b900050178000001410031
:109d300009b0b90000014100820278000a00420027
:109d40008b804a0070079800010f98005e00900019
:109d5000ee009000c289de004e0add004201de0006
:109d6000020172007e0090008e0890000200400008
:109d70008380480050079800610798005044800095
:109d80000000e0000c003a004e0090000000e000ef
:109d9000090032000000eb00400798008000eb0053
:109da000800020000a990200000000000000eb0083
:109db000c29b0200000000005e019000ee019000d6
:109dc000703e200001002000800f5100818f59005b
:109dd0002f003c004e009000e10f50008dff32003c
:109de0001000200040079800100020004044880028
:109df000504480000000e000fdff3a007e0090002b
:109e00008e089000809fbe009e089000811f780001
:109e10002e0a9000841f78003e089000801f780072
:109e20005e009000ee009000809fbe0020172d0085
:109e3000801f7800808a20002812020000000000a5
:109e4000f0875700808a2000fc0f0200000000000d
:109e500080007800808a2000c479020000000000a1
:109e600001f5210040b122002a7402000000000028
:109e700010002000c29b0200000000008000eb00e8
:109e8000800020000a9902000000000061ff3700f6
:109e90005e019000ee01900000902000d1032000b0
:109ea000800f5100818f59005aff34004e009000fe
:109eb000e20f500057ff32002000200040079800ba
:109ec0001000200040448800504480000000e00062
:109ed000fdff3a007e0090008e089000809fbe003b
:109ee0009e089000811f78002e0a9000841f780041
:109ef0003e089000801f78005e009000ee00900009
:109f0000809fbe00a0192d00801f7800808a20004d
:109f10002812020000000000f0875700808a20000d
:109f2000fc0f02000000000080007800808a200002
:109f3000c4790200000000003e089000630f60003a
:109f40001e00e00005003a00018420000000eb0044
:109f50002a740200000000000c00370011002000ed
:109f60009e8f100005003a00016e20004084200002
:109f70002a740200000000000400370041d52000d0
:109f800060f220002a740200000000000000eb00d4
:109f9000c29b0200000000003e089000cf80de005f
:109fa000d6020200000000000004be002e0890004f
:109fb000cf80de00d6020200000000000801be00d3
:109fc0002c030200000000001007980021079800f1
:109fd0003e089000cf80de00d602020000000000a4
:109fe0000004be002e089000cf80de00d6020200e2
:109ff000000000000801be002c0302000000000069
:10a00000b2fd20009304240066030200000000005b
:10a010000200200003082400ea0302000000000000
:10a02000b2fd200093fc2300540402000000000055
:10a03000b2fd200093ec2300540402000000000055
:10a040000e050200000000001e05020000000000d6
:10a0500030079800030037003e0090006800500071
:10a06000300798003e009000e80f5000faff3c00d7
:10a07000030037003e009000680040003007980061
:10a080003e0090000000e000faff35003e02900024
:10a09000841f78001e009000ae009000809fbe00dc
:10a0a000ae089000811f78003e0a9000841f78005f
:10a0b000e01b2d00801f7800808a200028120200fb
:10a0c00000000000ec875700808a2000fc0f02008f
:10a0d0000000000080007800808a2000c47902001f
:10a0e000000000003e009000110020000a990200cc
:10a0f00000000000c7fe37000600fa00889fbe007f
:10a100008a9fbe000000eb00b00289004d003700be
:10a11000b0028100810522004200dd000101400003
:10a120006000b8000089be000000eb00a0028900ba
:10a130001c003700bb028100b002810081052200b3
:10a140004200dd00010040001004be00b0028100aa
:10a15000a10281004300dd000100400080004000ba
:10a16000200322000080400010057800a00281003a
:10a1700074b202000000000000d0b900cf80de0001
:10a180000801400089814800810522004258dd0015
:10a19000010040000288be00a00281000000e8002b
:10a1a000a0028900a0028100e70f5000e1ff340007
:10a1b000b0028100000f7800b0028100810522000a
:10a1c0004200dd00010040001000be0010079800b2
:10a1d000210798001e019000ae019000e00f510091
:10a1e000e08f590006003d001e009000ae00900078
:10a1f00063004000e08048001007980021079800a5
:10a200001e019000ae0190004e1add004210de00eb
:10a2100000007200c298de006222200000014100ae
:10a220001e0078001e00780080004000000622001a
:10a230000080400002087800b00281000000e800c1
:10a24000b0028900b0028100e10f5000b0ff34007d
:10a250001103810010032000808f500012003c0089
:10a2600011038100e0fc2f00808f50000e003400ad
:10a270000103810010032000808f50000a003c0081
:10a2800001038100e0fc2f00808f500006003400a5
:10a29000100381007400b9001003890000038100dd
:10a2a0007400b9000003890011038100803e200082
:10a2b000808f500003003400803e2000100389008e
:10a2c000060037001103810080c12f00808f5000ed
:10a2d00002003d0080c12f001003890001038100ae
:10a2e000803e2000808f500003003400803e20001c
:10a2f00000038900060037000103810080c12f00a0
:10a30000808f500002003d0080c12f0000038900b3
:10a3100010038100a6a202000000000000038100db
:10a320002aa30200000000004f05be004f04be003b
:10a330000080fa00000006001000fa00889fbe00ae
:10a340008a9fbe00600798007107980040062000b1
:10a3500050079800d0cc2c00c1d4230030079800bf
:10a36000410798003000200020079800de00900090
:10a370006e0090000080500010079800800081005f
:10a38000cf80de00d6020200000000000005be0003
:10a390001e009000cf80de00d60202000000000008
:10a3a0003e019000ce019000ea0302000000000090
:10a3b0000004be002e009000cf80de00d602020016
:10a3c000000000000001be000800be00660302009d
:10a3d000000000000001be000a00be00540402009c
:10a3e000000000001e05020000000000800089003f
:10a3f000810081001e009000808040007e0090005f
:10a400000088b900000f7800703e20009e0f1000f9
:10a4100011003400703e20007e0190001100090000
:10a420000200d800800078001e00900000805000dc
:10a430008000890081008100c0032000808f5000cf
:10a4400002003400c003200080008900703e20001c
:10a45000000f78001200370080c12f009e0f1000ff
:10a460000f003c0090c12f007e01900011000900f8
:10a470000200d800800078001e009000008040009c
:10a480008000890080008100ea0f400002003d004a
:10a4900060ff2f008000890090c12f00000f78001e
:10a4a0001e0078004f05be004f04be000080fa0079
:10a4b000000006000a00fa003007980041079800e3
:10a4c0000000eb00200798000000eb001007980048
:10a4d000ae0090003e009000008f50009e0078007b
:10a4e0004e0090000088b900100798009e00900070
:10a4f000703e2000808f500003003400703e20002a
:10a5000010079800060037009e00900080c12f00c1
:10a51000808f500002003c0090c12f00100798006f
:10a520001e0090000080fa00000006000400fa00ff
:10a53000889fbe007000200074b20200000000007e
:10a54000000478000000eb0074b20200000000007c
:10a550000000440022002000110009000200d80081
:10a560006100200074ff0700100798000000eb0056
:10a5700074b2020000000000000478001000200007
:10a5800074b202000000000080044400700020004b
:10a5900074b2020000000000000478006000200097
:10a5a00074b202000000000000004400008054006b
:10a5b00041002000bfff0700000f78001e00900040
:10a5c0001e005000a6a20200000000001e00900025
:10a5d0001e0040002aa30200000000004f04be003d
:10a5e0000080fa00000006000000fa00b67a0200bf
:10a5f0000000000090a20200000000000040eb00fc
:10a60000968602000000000070b102000000000009
:10a61000419c200000f42900847b0200000000001f
:10a62000a128200060292500847b02000000000092
:10a630005a7b020000000000ffff37000000fa0014
:10a64000b67a02000000000090a2020000000000a4
:10a650000040eb00968602000000000070b102008e
:10a66000000000004138200080eb2900847b0200bc
:10a6700000000000a1282000c0072500847b020004
:10a68000000000005a7b020000000000ffff3700be
:10a690000000fa00b67a0200000000000040eb0063
:10a6a0009686020000000000a88202000000000060
:10a6b0009083020000000000fdff37001a00fa003e
:10a6c000889fbe000080eb00400f98000000eb0068
:10a6d000000f78007801470013002000e1ff2f00f1
:10a6e000f00720009244020000000000000f7800f4
:10a6f0001e007800630f60000000eb00300f980030
:10a70000310020009e8f1000020032001e00e00089
:10a7100005003a0010002000200f9800c003200020
:10a72000100f980004003700c0032000200f98008d
:10a7300010002000100f980080002000000f9800eb
:10a74000ae0890001e0890000088b90070079800bd
:10a75000786c0200000000008e0990000e0a900044
:10a760009e0890000e0890000088b90080037800d1
:10a77000ae0890000e0890000088b9000004780030
:10a780009e0890000e0890000088b90080007800b4
:10a79000001e2000010050002200200011000900ce
:10a7a0000200d80080047800ae0890000e089000e7
:10a7b0000088b900800078000028200001005000c7
:10a7c00022002000110009000200d8003e0b90007a
:10a7d00083027800870178000801780089007800fa
:10a7e000a66b0200000000001100200010002000f5
:10a7f000206c020000000000646c020000000000f9
:10a80000808a200026b3020000000000ac9b0200fa
:10a81000000000000000eb00c29b020000000000ee
:10a820000000eb00029c020000000000d6b3020012
:10a83000000000000000e000fcff3200808a2000e1
:10a84000500798000000eb00300798000000eb0074
:10a85000200798000000eb00100798000040eb0074
:10a86000004f98000000eb006007980016003700ca
:10a870005e00900090407800114f98005e009000bc
:10a880000000e800500798001e4890008080fb0000
:10a890003e00900001004000300798009e48900064
:10a8a0000e48900080cf5000040036001e489000f3
:10a8b000004f9800ee009000110798006e00900085
:10a8c0000000e800600798006e009000fd0f500047
:10a8d000e7ff3400160037005e00900090407800db
:10a8e000114f98005e0090000000e80050079800ab
:10a8f0001e4890008080fb002e0090000100400068
:10a90000200798009e4890000e48900080cf50008d
:10a91000040036001e489000004f9800ee009000a2
:10a92000110798006e0090000000e8006007980092
:10a93000ee0090001e089000808f5000e6ff35006a
:10a940001e009000f30f500005003e001100200093
:10a95000700020000a990200000000000d0037007e
:10a960009e00900070022000808f500005003e0085
:10a97000110020000000eb000a9902000000000016
:10a980000400370011002000100020000a99020086
:10a9900000000000300020009e0f10000300320075
:10a9a000210020009e8f10000e003a001e00900033
:10a9b0006a00b9008000780040ed2f000080400060
:10a9c000a6a20200000000009e00900060ff2f0081
:10a9d0000088b900c012b0002aa3020000000000e5
:10a9e0000d0037009e00900060ff2f000088b90026
:10a9f000c012b000a6a20200000000001e009000dd
:10aa00006a00b9008000780040ed2f00008040000f
:10aa10002aa30200000000000e4890000080fb0006
:10aa20009e009000811f7800801f78002e0090000b
:10aa3000801f7800be009000811f7800201e2d002e
:10aa4000801f7800808a2000281202000000000089
:10aa5000ea875700808a2000fc0f020000000000f7
:10aa600080007800808a2000c47902000000000085
:10aa70008038210001002000deb302000000000049
:10aa80005fff37001200fa00889fbe000000eb0055
:10aa9000000f98004001200070079800400120003e
:10aaa000600798008000200050079800fe0090008a
:10aab0006e0090000088b90040079800786c020092
:10aac00000000000de0190005e029000ee009000a9
:10aad0005e0090000088b90080037800fe009000be
:10aae0005e0090000088b90000047800ee0090003d
:10aaf0005e0090000088b90080007800001e2000f1
:10ab00000100500022002000110009000200d800be
:10ab100080047800fe0090005e0090000088b9007c
:10ab20008000780000282000010050002200200052
:10ab3000110009000200d8000e0b9000830278007b
:10ab4000870178000801780089007800a66b020070
:10ab5000000000001100200010002000206c020006
:10ab600000000000646c020000000000a8820200e7
:10ab700000000000808a200026b3020000000000d0
:10ab8000ac9b0200000000000000eb00c29b020032
:10ab9000000000000000eb00029c0200000000002a
:10aba0000000eb00bab9020000000000fe0f5000e8
:10abb0000a003c0010002000bab9020000000000aa
:10abc000fe0f500005003c0020002000bab9020032
:10abd00000000000fe0f50000300340010002000b1
:10abe000c29b0200000000000000eb0046b2020021
:10abf000000000008000780000192000808f5000c5
:10ac000004003400110020000000eb000a9902004b
:10ac1000000000001000200046b20200000000000a
:10ac20008000780000192000808f5000040034005c
:10ac300011002000100020000a990200000000000e
:10ac40002000200046b202000000000080007800d2
:10ac500000192000808f50000400340011002000f3
:10ac6000200020000a9902000000000030002000af
:10ac700046b20200000000008000780000192000a9
:10ac8000808f5000040034001100200030002000ac
:10ac90000a990200000000004000200046b20200b5
:10aca000000000008000780000192000808f500014
:10acb0000400340011002000400020000a99020026
:10acc000000000005000200046b20200000000001a
:10acd0008000780000192000808f500004003400ac
:10ace00011002000500020000a990200000000001e
:10acf0006000200046b202000000000080007800e2
:10ad000000192000808f5000040034001100200042
:10ad1000600020000a99020000000000700020007e
:10ad200046b20200000000008000780000192000f8
:10ad3000808f5000040034001100200070002000bb
:10ad40000a99020000000000d6b3020000000000d3
:10ad50000000e000fcff32006000b800100798001f
:10ad600021079800808a2000000f78000000eb0087
:10ad7000300798000e0037001e0078001040780061
:10ad80000081fb00030020001e009000ae00900038
:10ad900000004100818049001007980021079800b9
:10ada0001e0fe8003e0090000000e8003007980009
:10adb000be0090004e009000808f5000eeff3500e6
:10adc0001e009000ae009000809fbe0000212d006c
:10add000801f7800808a20002812020000000000f6
:10ade000e6875700808a2000fc0f02000000000068
:10adf00080007800808a2000c479020000000000f2
:10ae00001e019000ae01900000b82b000100200050
:10ae1000800f5100818f5900030036001000200080
:10ae2000029c020000000000803821000100200088
:10ae3000deb30200000000004eff37002a00fa00d7
:10ae400040062000000f78006a00470001232d0013
:10ae500007000900311878000001b1007a004700ae
:10ae600001222d0007000900311878000001b1000f
:10ae7000ac9b0200000000000000eb00c29b02003f
:10ae8000000000000000eb00029c02000000000037
:10ae90000000eb0046b202000000000080007800d5
:10aea00080252000808f5000040034001100200015
:10aeb0000000eb000a9902000000000010002000d2
:10aec00046b20200000000008000780080252000cb
:10aed000808f50000400340011002000100020007a
:10aee0000a990200000000002000200046b2020083
:10aef000000000008000780080252000808f500036
:10af00000400340011002000200020000a990200f3
:10af1000000000003000200046b2020000000000e7
:10af20008000780080252000808f500004003400cd
:10af300011002000300020000a99020000000000eb
:10af40004000200046b202000000000080007800af
:10af500080252000808f5000040034001100200064
:10af6000400020000a99020000000000500020006c
:10af700046b202000000000080007800802520001a
:10af8000808f500004003400110020005000200089
:10af90000a990200000000006000200046b2020092
:10afa000000000008000780080252000808f500085
:10afb0000400340011002000600020000a99020003
:10afc000000000007000200046b2020000000000f7
:10afd0008000780080252000808f5000040034001d
:10afe00011002000700020000a99020000000000fb
:10aff0000000eb0046b20200000000008000780074
:10b00000a00f2000808f500023003c001000200083
:10b0100046b202000000000080007800a00f20006f
:10b02000808f50001c003c002000200046b202002f
:10b030000000000080007800a00f2000808f5000ea
:10b0400015003c005000200046b202000000000045
:10b0500080007800a00f2000808f50000e003c0080
:10b060006000200046b2020000000000800078006e
:10b07000a00f2000808f500007003c0070002000cf
:10b0800046b202000000000080007800a00f2000ff
:10b09000808f50006900340010002000c29b020025
:10b0a00000000000800c200020079800800c200089
:10b0b000100798000000eb00400798002c003700b4
:10b0c0004e00900046b202000000000030079800d9
:10b0d0003e009000801f780000242d00801f780023
:10b0e000808a20002812020000000000e487570038
:10b0f000808a2000fc0f0200000000008000780021
:10b10000808a2000c4790200000000004e009000f8
:10b11000ea00470000004000e08078003e00900018
:10b120004480de000088b900800078002e00900086
:10b1300001004000200798004e009000fa004700f0
:10b1400000004000e08078003e0090004480de0077
:10b150000088b900800078001e00900001004000c7
:10b16000100798004e0090000000e800400798008b
:10b170004e009000e70f5000d1ff34009e00900079
:10b18000811f78002e009000801f780050242d0031
:10b19000801f7800808a2000281202000000000032
:10b1a000e6875700808a2000fc0f020000000000a4
:10b1b00080007800808a2000c4790200000000002e
:10b1c000ae00900000322000808f5000020034005a
:10b1d00000322000200798009e00900000322000de
:10b1e000808f5000020034000032200010079800c9
:10b1f000ae00900000ce2f00808f500002003d0076
:10b2000000ce2f00200798009e00900000ce2f0057
:10b21000808f500002003d0000ce2f0010079800e4
:10b220002e009000a6a20200000000001e00900068
:10b230002aa30200000000001b003700c02b2000e2
:10b24000a6a20200000000001e0fe800c02b200094
:10b250009e0f10000200340040062000000f78000e
:10b260001e0078002aa30200000000009e00780063
:10b27000811f780060252d00801f7800808a2000c3
:10b280002812020000000000e4875700808a200096
:10b29000fc0f02000000000080007800808a20007f
:10b2a000c47902000000000000e224000100200038
:10b2b000deb3020000000000edfe37002400fa00bb
:10b2c000889fbe008a1f78000000eb0010079800de
:10b2d000090037001e009000e40047004200dd0036
:10b2e000010140006000b8000089be001e0090000f
:10b2f0000000e800100798001e009000e70f5000c3
:10b30000f4ff34000000eb00000f78001e0037004f
:10b310000000eb0010079800130037001e05900096
:10b320001e009000e40047004200dd0001004000e4
:10b330001004be001e00900046b202000000000093
:10b34000cf80de000801400089814800e40047000a
:10b350004250dd00010040000288be001e00900047
:10b360000000e800100798001e009000e70f500052
:10b37000eaff34000071220001002000deb3020069
:10b38000000000001e0fe800f00120009e0f1000da
:10b39000dfff34000000eb001007980025003700a5
:10b3a0009e0190001e009000e40047004200dd0076
:10b3b000010040001000be004b09dd004500de002a
:10b3c00000007100c588de00000178008380410024
:10b3d0006012220000804000020878001e009000e9
:10b3e00080004000601222000080400010007800c1
:10b3f000801f780020262d00801f7800808a200082
:10b400002812020000000000e4875700808a200014
:10b41000fc0f02000000000080007800808a2000fd
:10b42000c4790200000000001e0090000000e80047
:10b43000100798001e009000e70f5000d8ff34005e
:10b44000808a200071262d001300090031587800f1
:10b45000808a2000fc0f02000000000080007800bd
:10b46000808a2000c479020000000000006a2800e1
:10b4700011002000deb30200000000004f0578003c
:10b480004f04be000080fa00000006000000fa0031
:10b49000e6c2bf000080fb004600de0061406000a5
:10b4a0000081fb00e7c2bf000080fb000000d1006c
:10b4b000614060000080fb000000400080007800d8
:10b4c000e7c2bf00614060000080fb0000804000d8
:10b4d0000000400080007800e6c2bf000080fb0052
:10b4e0004700de000080fb000080400000004000bc
:10b4f000000041000080fa00000006000400fa008d
:10b50000881f7800100798000000eb00000f7800fb
:10b51000110037001e007800000040008000780015
:10b520001e009000008440001e00780046b2020019
:10b5300000000000000178001e007800800040003c
:10b5400060122200008040001000780000005100ce
:10b55000000c78001e0fe800700020009e0f100005
:10b56000ecff36004f0478000080fa00000006006f
:10b570000400fa00000f78001107980000ce2f0099
:10b580009e0f100002003d0000ce2f00000f78003b
:10b59000003220009e0f1000020034000032200014
:10b5a000000f78009e00900000ce2f00808f50008a
:10b5b00002003d0000ce2f00100798009e00900072
:10b5c00000322000808f5000020034000032200042
:10b5d000100798001e007800a6a2020000000000dc
:10b5e0001e0090002aa30200000000000080fa0064
:10b5f000000006001a00fa00b67a020000000000ff
:10b6000090a20200000000002cff07000000eb00e9
:10b61000000f78006a004700b8ff07000000eb0049
:10b620001007980099ff0700610060000004e00027
:10b630003e0032008000eb00600020000a9902000a
:10b640000000000011002000200020000a990200e4
:10b65000000000000000eb00200798000a003700ff
:10b660002e009000ea00470000004000e0807800d3
:10b6700020032000808f500006003c002e00900028
:10b680000000e800200798002e009000e70f50000f
:10b69000f3ff34002e009000e80f500003003a0042
:10b6a00010002000100798005d00370060ff2f0099
:10b6b000a006890060ff2f0010078900a00020006d
:10b6c00020078900a0002000900789006a00470039
:10b6d000a0009000c0122000808f50005000340065
:10b6e0006a0047009000900080f32f0080804000a7
:10b6f0006a004700110098006a004700a00090000f
:10b7000080da2f00808040006a0047002100980006
:10b710006a004700b0009000c0f92f008080400010
:10b720006a004700310098003d00370011002000fa
:10b73000600020000a990200000000008000eb0079
:10b74000200020000a990200000000000000eb0029
:10b75000200798000a0037002e009000ea004700fa
:10b7600000004000e080780020032000808f50001f
:10b7700006003c002e0090000000e8002007980022
:10b780002e009000e70f5000f3ff34002e009000d1
:10b79000e80f500003003a00100020001007980046
:10b7a0001f003700a0002000a0068900a000200094
:10b7b0001007890060ff2f002007890060ff2f001d
:10b7c000900789006a004700d0009000c012200056
:10b7d000808f5000120034006a004700c0009000c3
:10b7e000c0f92f00808040006a00470041009800a7
:10b7f0006a004700d000900080da2f00808040006f
:10b800006a004700510098006a004700e00090007d
:10b8100080f32f00808040006a004700610098009c
:10b82000800c200040079800800c20003007980012
:10b830001e0090000000e00027003a000000eb002e
:10b8400020079800210037002e0090008000400063
:10b85000400d220000804000100178002e00900072
:10b86000ea00470000004000608078004480de006d
:10b870000090b900800078004e0090000100400068
:10b88000400798002e00900080004000400e2200eb
:10b8900000804000100178002e009000ea00470070
:10b8a00000004000608078004480de000090b90015
:10b8b000800078003e0090000100400030079800b2
:10b8c0002e0090000000e800200798002e00900055
:10b8d000e70f5000dcff3400be0090004e009000e7
:10b8e00023ff070080a9230001002000deb302002f
:10b8f0000000000047ff37000400fa003105200077
:10b9000080092d00c479020000000000dc790200eb
:10b91000000000000000e000fcff3a004678020052
:10b9200000000000000037000e007800647902007b
:10b93000000000001e40780000404000004f7800ea
:10b940000e00e80064790200000000001e40900034
:10b950000004e00010003d005a78020000000000e2
:10b960001e409000804078000174a1001e407800c5
:10b970006e78020000000000204798006478020002
:10b98000000000000e80e80011002000c4790200d1
:10b9900000000000e4ff37000e80e8006479020038
:10b9a000000000005a780200000000002e409000c5
:10b9b000004178001e409000804078001e407800d2
:10b9c000c878020000000000647802000000000057
:10b9d000d5ff37000200fa0071052000c00e2d00cf
:10b9e000c479020000000000dc79020000000000c1
:10b9f0000000e000fcff3a00467802000000000072
:10ba00000e00780064790200000000000e00e800db
:10ba10006479020000000000f9ff37001800fa0006
:10ba20000000eb0020079800e0a021006103070060
:10ba3000300798000000eb0010079800b0003700b6
:10ba40001e0090007d00b900e6004000e0a021004b
:10ba5000614078008040eb00715798000004e000de
:10ba600002003a0012c0b300725798001e00900006
:10ba70007d00b900e7004000e0a0210061407800af
:10ba80008040eb00615798000004e00002003a009b
:10ba900012c0b30062579800fe5090006e519000a3
:10baa00002c060000080fb00200f98001e00900084
:10bab0007d00b900e8004000e0a02100614078006e
:10bac0008000eb00110f98000004e00002003a0033
:10bad00012002000120f98002e0890009e0890007f
:10bae00001006000000f98001e0090007d00b9006a
:10baf000e5004000e0a02100614078000001eb007b
:10bb000072079800e84f500002003a001000200031
:10bb1000700798008e0890007e01900002806000ff
:10bb20000000e000730032001e0090007d00b900ac
:10bb300080007800e0a0210000804000b2030700f0
:10bb40001e0090007d00b900e8004000f0a0210038
:10bb5000e14078000040eb00504f980050c6b30021
:10bb600080cf500002003a0011c0b300514f98003e
:10bb70001e0090007d00b900e9004000f0a0210007
:10bb8000e14078000041eb00424f9800d0c2b30082
:10bb900080cf500002003a0010c0b300404f980020
:10bba000de4890004e49900002c060000080fb001b
:10bbb000500798001e0090007d00b900ea00400088
:10bbc000f0a02100e14078000000eb004007980061
:10bbd00000c7b30080cf500002003a0011002000df
:10bbe000410798005e019000ce00900001006100c6
:10bbf0000000e0003f0032000000eb00000f780082
:10bc00001d003700ae0190001e0278001e0090005b
:10bc10001e0178007d00b90082004000e0a02100f4
:10bc2000614178006b18b9008400400000b3210026
:10bc300082707800ae0190001e0278001e00900015
:10bc40009e007800678140007d00b900020040003e
:10bc5000e8004000f0a02100614078000041780039
:10bc60006b18b90004004000e600400000b321005a
:10bc7000827078001e0fe800320020009e0f110035
:10bc8000e0ff34002e0090006b00b9006a01400014
:10bc900001b321000040eb0000f1780040002000db
:10bca000000f78000d003700ae0190001e027800f2
:10bcb0001e0090001e0178007d00b9008200400047
:10bcc000e0a02100614178006b18b90084004000b9
:10bcd00000b32100827078001e0fe80050002000a1
:10bce0009e0f1000f0ff34002e0090000000e800ce
:10bcf000200798001e0090000000e8001007980040
:10bd00009e0090003e009000808f50004cff350058
:10bd10002e0090000080fa00000006000600fa00e5
:10bd2000e0b921000f0107003cff07001007980051
:10bd30001e0090000000e0000a00320060b3210005
:10bd4000bb01070000b32100a7030700004f7800e4
:10bd5000e0b92100b60107001e00fb002007980093
:10bd60000200370030062000200798002e009000c7
:10bd70000080fa00000006002e00fa00e4004700f0
:10bd800020c0b30080487800e400470020c5b3001d
:10bd900090409800e400470060c2b300a0409800c3
:10bda000e40047000040eb00b0409800e40047008a
:10bdb0000040eb00c0409800e400470080c7b3009b
:10bdc000d0409800e400470030c0b300e040980045
:10bdd0006400470071002000c479020000000000e8
:10bde0000000eb00100798000040eb00004f7800c7
:10bdf000000037001e009000800078006b004700b4
:10be00000100400064790200000000000000e00032
:10be1000060032009e0090006b004700614f7800e2
:10be20001e0090000000e8001007980030c0b3002a
:10be30009e4f1000efff3a006b004700304090002b
:10be40000000fb00e60040001e009000808f5000c4
:10be5000e8ff3c001e019000eb0047000040eb00b3
:10be600000f178000000eb00100798000b0037008d
:10be70001e0190001e009000e70040006b0047008c
:10be8000e1407800900220000e004000017178002f
:10be90001e0090000000e800100798006b004700ab
:10bea000604090008000fb001e009000808f5000da
:10beb000efff3c001e019000910220008e804000a8
:10bec0000040eb0000f17800900220000e004000de
:10bed0004e100200000000000080fa000000060082
:10bee0001600fa00e400470020c0b3008048780044
:10bef000e400470020c5b30090409800e4004700ec
:10bf0000a0c1b300a0409800e40047000040eb004f
:10bf1000b0409800e40047000040eb00c0409800ab
:10bf2000e4004700c0c6b300d0409800e4004700da
:10bf300030c0b300e040980064004700710020006a
:10bf4000c4790200000000000000eb001007980018
:10bf50000040eb00004f7800000037001e0090000a
:10bf6000800078006c004700010040006479020006
:10bf7000000000000000e000070032009e0090007a
:10bf80006c00470000804000104f78001e009000b9
:10bf90000000e8001007980030c0b3009e4f10006a
:10bfa000eeff3a006c004700304090000000fb00bc
:10bfb000e60040001e009000808f5000e7ff3c002c
:10bfc0009e0090006c004700808040000040eb0025
:10bfd000804878006c004700604090000000fb0043
:10bfe0000080fa00000006001600fa00e400470096
:10bff00020c0b30080487800e400470020c5b300ab
:10c0000090409800e400470010c1b300a0409800a1
:10c01000e400470010c0b300b0409800e4004700bf
:10c020000040eb00c0409800e400470040c6b30069
:10c03000d0409800e400470010c0b300e0409800f2
:10c04000e400470030c0b300f040980064004700af
:10c0500081002000c4790200000000000000eb0015
:10c06000100798000040eb00004f780000003700f8
:10c070001e009000800078006c0047000100400026
:10c0800064790200000000000000e00007003200b8
:10c090009e0090006c00470000804000104f780028
:10c0a0001e0090000000e8001007980030c0b300a8
:10c0b0009e4f1000eeff3a006c00470030409000a9
:10c0c0000000fb00e60040001e009000808f500042
:10c0d000e7ff3c009e0090006c004700808040001d
:10c0e0000040eb00804878006c0047006040900002
:10c0f0000000fb000080fa00000006000400fa00c7
:10c100000de2a900de62a900e262a9006000b800a9
:10c11000008fbe0004003700100020000100200046
:10c120001e0f40005e9748001e00be00d6020200af
:10c1300000000000626626006366240060050200bd
:10c14000000000000000e000f3ff3500e262a800fc
:10c15000de62a80010790200000000000080fa00f2
:10c16000000006002c00fa0050179800e400470079
:10c1700020c0b30080487800e400470020c5b30029
:10c1800090409800e400470060c1b300a0409800d0
:10c19000e40047000040eb00b0409800e400470096
:10c1a0000040eb00c0409800e400470080c6b300a8
:10c1b000d0409800e400470030c0b300e040980051
:10c1c0006400470071002000c479020000000000f4
:10c1d0000000eb00100798000040eb00004f7800d3
:10c1e000000037001e009000800078006b004700c0
:10c1f0000100400064790200000000000000e0003f
:10c20000070032009e0090006b00470061407800fc
:10c21000004f78001e0090000000e8001007980012
:10c2200030c0b3009e4f1000eeff3a006b00470095
:10c23000304090000080fb00e60040001e009000af
:10c24000808f5000e7ff3c001e019000eb0047008c
:10c250000040eb0000f178000000eb0010079800b0
:10c260000c0037001e009000800078005e109000e7
:10c27000008140001e009000e80040006b00470075
:10c2800061407800004978001e0090000000e8003e
:10c29000100798006b004700704090008080fb0002
:10c2a0001e009000808f5000eeff3c001e009000aa
:10c2b000800078005e109000808040000040eb001d
:10c2c000804878006b004700604090000000fb0051
:10c2d0000080fa00000006003600fa00201f9800d7
:10c2e000e400470020c0b30080487800e400470025
:10c2f00020c5b30090409800e400470030c0b30070
:10c30000a0409800e40047000040eb00b0409800d7
:10c31000e40047000040eb00c0409800e400470004
:10c3200050c5b300d0409800e400470030c0b300cf
:10c33000e04098006400470071002000c4790200ca
:10c34000000000000000eb00100798000040eb0028
:10c35000004f7800000037001e0090008000780039
:10c360006b004700010040006479020000000000fb
:10c370000000e000060032009e0090006b004700c5
:10c38000614f78001e0090000000e8001007980040
:10c3900030c0b3009e4f1000efff3a006b00470023
:10c3a000304090000000fb00e60040001e009000be
:10c3b000808f5000e8ff3c001e019000eb0047001a
:10c3c0000040eb0000f178000000eb00100798003f
:10c3d0000c0037001e009000800078002e1890009e
:10c3e000008140001e009000e80040006b00470004
:10c3f00061407800004978001e0090000000e800cd
:10c40000100798006b004700704090008000fb0010
:10c410001e009000808f5000eeff3c006b00470034
:10c42000604090000000fb000080fa000000060061
:10c430003000fa00701798007e109000fc0f020088
:10c4400000000000000f7800e600470020c0b300a5
:10c4500080487800e600470020c5b300904098006f
:10c46000e600470070c1b300a04098001e007800ad
:10c470008040e8006600470031409800e600470031
:10c480000040eb00c04098006600470090409000dc
:10c49000660047002040900080c0400066004700d2
:10c4a0003040900080c04000660047005140980036
:10c4b0001e007800804078006600470061409800c8
:10c4c0000000eb00200798000d0037002e009000c0
:10c4d000670140002e009000800078007e109000e0
:10c4e0000080400090407800660047000000410056
:10c4f000014878002e0090000000e8002007980016
:10c500002e0090009e0f5000f0ff35001e007800b6
:10c51000e7004000660047008080400030c0b30064
:10c52000804878001e007800e80040006600470060
:10c53000c4790200000000000000eb002007980012
:10c540000040eb0020479800000037002e009000cc
:10c5500080007800400220000e00400001004000f2
:10c5600064790200000000000000e00009003200d1
:10c57000ae009000400220000e004000008040000d
:10c5800090407800214798002e0090000000e800bd
:10c59000200798002e409000e34f5000ebff3a0038
:10c5a000400220000e004000304090000000fb00e0
:10c5b000e60040002e009000808f5000e3ff3c001a
:10c5c000ae009000400220000e004000808040003d
:10c5d0000040eb0080487800400220000e00400040
:10c5e000604090000000fb000080fa0000000600a0
:10c5f0003a00fa00401f98004e189000fc0f02000d
:10c6000000000000000f78001e0fe800e600470061
:10c6100020c0b30080487800e600470020c5b30082
:10c6200090409800e600470040c0b300a04098004a
:10c630001e0078008040e800660047003140980006
:10c64000e60047000040eb00c0409800660047004d
:10c6500090409000660047002040900080c040005d
:10c66000660047003040900080c0400066004700f0
:10c67000514098001e007800804078006600470016
:10c68000614098000000eb00200798000d00370083
:10c690002e009000670140002e009000800078007e
:10c6a0004e189000008040009040780066004700df
:10c6b00000004100014878002e0090000000e800d2
:10c6c000200798002e0090009e0f5000f0ff3500cc
:10c6d0001e007800e70040006600470080804000b0
:10c6e00030c0b300804878001e007800e8004000a9
:10c6f00066004700c4790200000000000000eb0063
:10c70000200798000040eb00204798000000370009
:10c710002e00900080007800e00220000e00400013
:10c720000100400064790200000000000000e00009
:10c7300009003200ae009000e00220000e00400030
:10c740000080400090407800214798002e00900023
:10c750000000e800200798002e409000e34f5000b2
:10c76000ebff3a00e00220000e0040003040900055
:10c770000000fb00e60040002e009000808f50007b
:10c78000e3ff3c00ae009000e00220000e004000fd
:10c79000808040000040eb0080487800e0022000ec
:10c7a0000e004000604090000000fb000080fa0096
:10c7b000000006004800fa0020279800e800470023
:10c7c00020c0b30080487800e800470020c5b300cf
:10c7d00090409800e80047000040eb00a04098001f
:10c7e000e800470030c0b300b0409800e8004700c0
:10c7f0000040eb00c0409800e800470050c5b3007f
:10c80000d0409800e800470050c0b300e0409800d6
:10c81000e8004700a0c0b300f0409800e8004700df
:10c820000040eb0080489800e800470030c0b300ab
:10c830009048980068004700a1002000c4790200d9
:10c84000000000000000eb00300798000000eb0043
:10c85000100798001e009000200798000040eb0091
:10c86000004f78000000eb00200798000000370020
:10c870002e00900080007800720047000100400008
:10c8800064790200000000000000e00007003200b0
:10c89000ae0090007200470000804000104f78000a
:10c8a0002e0090000000e8002007980031c0b3007f
:10c8b0009ecf1000eeff3a0072004700304090001b
:10c8c0000000fb00e60040002e009000808f50002a
:10c8d000e7ff3c00720047009040900090c6b30014
:10c8e00080cf50002f003a000000eb002007980096
:10c8f0000f0037003e0090007d00b90080007800f6
:10c900002e20900000814000ae0190002e0090008b
:10c91000e6004000720047000080400010407800b0
:10c92000807179002e0090000000e8002007980038
:10c930002e009000e50f5000eeff34000000eb00e9
:10c9400020079800110037003e0090007d00b900dc
:10c95000800078002e20900000814000ae01900001
:10c960002e009000ec004000720047000080400064
:10c9700010407800804078006680410001707900a6
:10c980002e0090000000e800200798002e00900084
:10c99000e20f5000ecff34003e0090000000e80081
:10c9a0003007980072004700904090000040eb0074
:10c9b00060c7980030c4b30080cf5000020032003e
:10c9c00011c0b30061c7980072004700204090007a
:10c9d00070c798007ec090000004e00002003200a2
:10c9e00011c0b30071c798007ec09000eec09000e7
:10c9f00000c060000004e0009aff3a003e00900092
:10ca00000080fa00000006004600fa002027980087
:10ca1000e400470020c0b30080487800e4004700ed
:10ca200020c5b30090409800e400470020c0b30048
:10ca3000a0409800e400470060c0b300b0409800f8
:10ca4000e40047000040eb00c0409800e4004700cd
:10ca5000a0c5b300d04098002e2090001040780070
:10ca60008040780064004700614098002e209000cc
:10ca700010409000804078006400470071409800aa
:10ca80002e209000204090008040780064004700f5
:10ca9000014898002e20900030409000804078009f
:10caa00064004700114898002e20900040409000fc
:10cab0008040780064004700214898002e209000b4
:10cac0005040900080407800640047003148980052
:10cad000e400470030c0b300c0489800640047003d
:10cae000d1002000c4790200000000000000eb002b
:10caf000100798000040eb00004f7800000037005e
:10cb00001e00900080007800710047000100400086
:10cb100064790200000000000000e000060032001e
:10cb20009e00900071004700614f78001e00900049
:10cb30000000e8001007980030c0b3009e4f1000be
:10cb4000efff3a0071004700304090000000fb000a
:10cb5000e60040001e009000808f5000e8ff3c007f
:10cb60001e019000f10047000040eb0000f178004a
:10cb700071004700604090000004e00015003a009a
:10cb80000000eb00100798000c0037009e01900099
:10cb90001e009000ee0040007100470061417800e7
:10cba000ae209000688041000100400012409800d3
:10cbb0001e0090000000e800100798007100470078
:10cbc000504890008000fb001e009000808f5000b5
:10cbd000eeff3c0071004700604090000000fb0049
:10cbe0000080fa00000006004a00fa003027980092
:10cbf000e400470020c0b30080487800e40047000c
:10cc000020c5b30090409800e4004700a0c0b300e6
:10cc1000a0409800e400470080c0b300b0409800f6
:10cc2000e40047000040eb00c0409800e4004700eb
:10cc300040c6b300d0409800e400470010c0b300e5
:10cc4000e04098003e20900090407800640047004b
:10cc5000714098003e2090000000e800904078006d
:10cc600064004700014898003e2090000080e800e2
:10cc70009040780064004700114898003e209000e2
:10cc8000630040009040780064004700214898000d
:10cc90003e2090006400400090407800640047000f
:10cca000314898003e209000650040009040780098
:10ccb0006400470041489800e400470010c0b300fa
:10ccc000d0489800e400470030c0b300e048980026
:10ccd00064004700f1002000c47902000000000059
:10cce0000000eb00100798000040eb00004f7800b8
:10ccf0000000eb0010079800000037001e009000b5
:10cd00008000780073004700010040006479020051
:10cd1000000000000000e000060032009e009000cd
:10cd200073004700614f78001e0090000000e8008b
:10cd30001007980030c0b3009e4f1000efff3a007c
:10cd400073004700304090000000fb00e600400008
:10cd50001e009000808f5000e8ff3c0073004700e9
:10cd6000a04090000041eb0012cf980090c6b300a5
:10cd700080cf50000200320010c0b30010cf9800e6
:10cd800073004700204090008040eb0001cf9800e6
:10cd9000eb4f50000200320012c0b30002cf9800e7
:10cda0009ec890000ec9900002c060000004e00020
:10cdb000cfff3a0073004700604090000000fb0086
:10cdc0000080fa00000006001c00fa00e4004700a2
:10cdd00020c0b30080487800e400470020c5b300bd
:10cde00090409800e4004700d0c0b300a0409800f5
:10cdf000e400470010c0b300b0409800e4004700d2
:10ce00000040eb00c0409800e400470000c6b300bb
:10ce1000d0409800e400470010c0b300e040980004
:10ce2000e400470030c0b300f040980064004700c1
:10ce300081002000c4790200000000000000eb0027
:10ce4000100798000040eb00004f7800000037000a
:10ce50001e009000800078006c0047000100400038
:10ce600064790200000000000000e00007003200ca
:10ce70009e0090006c00470000804000104f78003a
:10ce80001e0090000000e8001007980030c0b300ba
:10ce90009e4f1000eeff3a006c00470030409000bb
:10cea0000000fb00e60040001e009000808f500054
:10ceb000e7ff3c009e0090006c004700808040002f
:10cec0000040eb00804878006c0047002040900054
:10ced0008040eb00215f9800ed4f500002003a00c7
:10cee00012c0b300225f98006c00470060409000c1
:10cef000305f98003e5890000004e00002003200cd
:10cf000011c0b300315f98003e5890002e59900038
:10cf1000004061000004e000050032006c004700a2
:10cf2000604090000000fb00400f98003700370081
:10cf30000000eb0010079800000037001e00900072
:10cf4000800078006c004700010040006479020016
:10cf5000000000000000e000070032009e0090008a
:10cf60006c00470000804000104f78001e009000c9
:10cf70000000e8001007980030c0b3009e4f10007a
:10cf8000eeff3a006c004700304090000000fb00cc
:10cf9000e60040001e009000808f5000e7ff3c003c
:10cfa0006c004700904090000041eb0072579800e1
:10cfb00090c6b30080cf50000200320010c0b30012
:10cfc000705798006c004700a04090000041eb00b3
:10cfd0006257980010c5b30080cf500002003200a5
:10cfe00010c0b30060579800fe5090006e51900042
:10cff00002c060000004e000cdff3a006c00470072
:10d00000604090000000fb00400f98004e08900028
:10d010000080fa00000006008a00fa0030879800bd
:10d02000014f9900e400470020c0b3008048780019
:10d03000e400470020c5b30090409800e40047009a
:10d04000f0c0b300a04098000e489100e3404000bb
:10d050006400470031409800e40047000040eb00c6
:10d06000c040980064004700904090006400470072
:10d070002040900080c04000640047003040900095
:10d0800080c040006400470051409800e400470021
:10d0900010c0b300e0409800640047008e48910043
:10d0a00071409800e40047000040eb008048980081
:10d0b0000000eb00100798000d0037001e009000e4
:10d0c000690140001e009000800078003e809000c2
:10d0d000008040009040780064004700000041005c
:10d0e000014878001e0090000000e800100798003a
:10d0f0000e4891008000fb001e009000808f5000c1
:10d10000eeff3c000e4891000000fb00e9004000eb
:10d11000640047008080400030c0b3008048780041
:10d120000e4891000000fb00ea0040006400470048
:10d13000c4790200000000000000eb001007980016
:10d140000040eb00004f7800000037001e00900008
:10d1500080007800c00720000e0040000100400061
:10d1600064790200000000000000e00008003200c6
:10d170009e009000c00720000e004000008040008c
:10d18000104f78001e0090000000e8001007980083
:10d1900030c0b3009e4f1000ecff3a00c0072000e3
:10d1a0000e004000304090000000fb00e600400010
:10d1b0001e009000808f5000e4ff3c009e00900015
:10d1c000c00720000e004000808040000040eb00bf
:10d1d00080487800c00720000e00400060409000aa
:10d1e0000000fb000080fa00000006004800fa0082
:10d1f000e600470020c0b30080487800e600470002
:10d2000020c5b30090409800e6004700c0c1b300bd
:10d21000a0409800e60047000040eb00b0409800b6
:10d22000e60047000040eb00c0409800e6004700e1
:10d23000e0c6b300d0409800e600470030c0b3001d
:10d24000e04098006600470071002000c4790200a9
:10d25000000000000000eb00200798000000eb0039
:10d26000100798000040eb00004f780000003700e6
:10d270001e009000800078006d0047000100400013
:10d2800064790200000000000000e00006003200a7
:10d290009e0090006d004700614f78001e009000d6
:10d2a0000000e8001007980030c0b3009e4f100047
:10d2b000efff3a006d004700304090000000fb0097
:10d2c000e60040001e009000808f5000e8ff3c0008
:10d2d0006d004700704090000000fb0020079800a0
:10d2e0002e0090000000e000140032000000eb006f
:10d2f000100798000b0037001e0190001e009000e0
:10d30000e80040006d0047006140780080407800f0
:10d31000e09d2100017178001e0090000000e800ef
:10d32000100798002e0090006600b9008000780079
:10d330001e009000808f5000efff3c002e009000f8
:10d340000000fb000080fa00000006001e00fa004a
:10d35000600f9800e400470020c0b30080487800c8
:10d36000e400470020c5b30090409800e400470067
:10d37000b0c1b300a0409800e400470060c0b30013
:10d38000b0409800e40047000040eb00c040980027
:10d39000e400470030c7b300d04098006e0890000a
:10d3a0006600b90080007800e09d210061407800af
:10d3b0008040780064004700614098006e0890004b
:10d3c0006600b9008000e800e09d2100614078001f
:10d3d0008040780064004700714098006e0890001b
:10d3e0006600b9008080e800e09d2100614078007f
:10d3f0008040780064004700014898006e08900063
:10d400006600b900e3004000e09d21006140780023
:10d410008040780064004700114898006e08900032
:10d420006600b900e4004000e09d21006140780002
:10d430008040780064004700214898006e08900002
:10d440006600b900e5004000e09d210061407800e1
:10d45000804078006400470031489800e4004700ad
:10d4600030c0b300c048980064004700d1002000dd
:10d47000c4790200000000000000eb0010079800d3
:10d480000040eb00004f7800000037001e009000c5
:10d4900080007800710047000100400064790200bc
:10d4a000000000000000e000060032009e00900036
:10d4b00071004700614f78001e0090000000e800f6
:10d4c0001007980030c0b3009e4f1000efff3a00e5
:10d4d00071004700304090000000fb00e600400073
:10d4e0001e009000808f5000e8ff3c001e0190005d
:10d4f000f10047000040eb0000f1780071004700a8
:10d50000604090000000fb000080fa000000060070
:10d510001a00fa0060579800e400470020c0b300ea
:10d5200080487800e400470020c5b3009040980090
:10d53000e4004700e0c4b300a0409800e4004700c6
:10d5400010c0b300b0409800e40047000040eb007a
:10d55000c0409800e400470010cab300d0409800d3
:10d5600064004700ee50900061409800e4004700de
:10d5700030c0b300f04098006400470081002000f4
:10d58000c4790200000000000000eb0010079800c2
:10d590000040eb00004f78006e509000e14f5000cb
:10d5a000030034000000eb00400f98002200370019
:10d5b0001e009000800078006c00470001004000d1
:10d5c00064790200000000000000e0000700320063
:10d5d0009e0090006c00470000804000104f7800d3
:10d5e0001e0090000000e8001007980031c0b30052
:10d5f0009ecf1000eeff3a006c00470030409000d4
:10d600000000fb00e60040001e009000808f5000ec
:10d61000e7ff3c009e0090006c00470080804000c7
:10d620000040eb00804878006c00470060409000ac
:10d630000000fb00400f98004e0890000080fa00a8
:10d64000000006001600fa00e400470020c0b30006
:10d6500080487800e400470020c5b300904098005f
:10d66000e4004700f0c4b300a0409800e400470085
:10d670000040eb00b0409800e40047000040eb00a1
:10d68000c0409800e400470010cab300d0409800a2
:10d69000e400470030c0b300e04098006400470059
:10d6a00071002000c4790200000000000000eb00bf
:10d6b000100798000040eb00004f78000000370092
:10d6c0001e009000800078006c00470001004000c0
:10d6d00064790200000000000000e0000700320052
:10d6e0009e0090006c00470000804000104f7800c2
:10d6f0001e0090000000e8001007980030c0b30042
:10d700009e4f1000eeff3a006c0047003040900042
:10d710000000fb00e60040001e009000808f5000db
:10d72000e7ff3c009e0090006c00470080804000b6
:10d730000040eb00804878006c004700604090009b
:10d740000000fb000080fa00000006001200fa0052
:10d75000000f7800110798002207980033079800ff
:10d76000440798005507980066079800000d81004f
:10d77000000f9800000326008e089000808f500054
:10d7800014003200000328008e089000808f5000a3
:10d790001b003200000323008e089000808f500091
:10d7a00001003200210037006e039000de0290007d
:10d7b0004e029000be0190002e0190009e0090004d
:10d7c0001e007800968c0200000000007007980090
:10d7d000180037006e039000de0290004e029000a9
:10d7e000be0190002e0190009e0090001e00780067
:10d7f000228f020000000000700798000d00370023
:10d800006e039000de0290004e029000be01900078
:10d810002e0190009e0090001e007800e291020010
:10d82000000000007007980002003700b0002000e0
:10d83000700798007e0090000080fa00000006004b
:10d840000600fa00000f780011079800000d810013
:10d850002007980000032600ae009000808f500043
:10d860000e00320000032800ae009000808f5000b0
:10d870000f00320000032300ae009000808f5000a4
:10d88000010032000e0037009e0090001e0078005c
:10d890006ea6020000000000090037009e00900004
:10d8a0001e007800c671020000000000040037006e
:10d8b0009e0090001e0078007ab002000000000078
:10d8c0000080fa00000006000000fa00010d81004f
:10d8d00000032300808f5000010032000200370057
:10d8e00018a40200000000000080fa0000000600fa
:10d8f0000400fa00b67a0200000000004678020038
:10d9000000000000d1a2a9004006200010079800e6
:10d9100004003700000000001e0090000000e90035
:10d92000100798001e0090000000e000f9ff3a0088
:10d93000d1a2a8004006200010079800040037007c
:10d94000000000001e0090000000e9001007980091
:10d950001e0090000000e000f9ff3a0081e0a900fd
:10d96000f1048000f0002f0080806000006620003d
:10d9700000804000f00488008040eb00c0cdb30080
:10d980006e780200000000001047980011c0b3003c
:10d99000c0cdb3006e78020000000000004f780098
:10d9a0001e4090000080fb00c800dd001e80fb00d0
:10d9b00000807000000d8900010d8100000323002c
:10d9c000808f500004003a008000eb000000eb0064
:10d9d0009bff070011003700010d810000032600a6
:10d9e000808f500004003a00110020001000200039
:10d9f00093ff070009003700010d81000003280094
:10da0000808f500005003a008000eb000000eb0022
:10da10008bff070008ae020000000000aaff07000d
:10da2000000d81000080fa00000006000800fa00e6
:10da3000200798003107980032c0bf000080fb002b
:10da4000000f78002e00900032e0b7003e009000fa
:10da50001000ba00100798001e00780032e0b700ee
:10da60001e0090000080fa00000006000600fa0088
:10da7000000d81002007980000032600ae009000f2
:10da8000808f50002100320000032800ae0090007b
:10da9000808f50002000320000032300ae00900071
:10daa000808f5000010032001e003700e1ff2f0080
:10dab000f0072000ddff07006300600010079800fa
:10dac0001e009000e20f50000a0032009e009000fd
:10dad000e38f50000a0032001e009000e10f50005a
:10dae000010032000900370011002000010f78000a
:10daf0000e00370020002000000f78000b003700d8
:10db00008000eb00010f78000800370010002000b3
:10db1000000f78000500370011002000010f780089
:10db2000020037000080eb00000f78001e00780034
:10db30000080fa00000006000600fa00000f7800de
:10db400011079800000d81002007980000032600af
:10db5000ae009000808f50000e00320000032800bd
:10db6000ae009000808f50000f00320000032300b1
:10db7000ae009000808f5000010032000e00370090
:10db80009e0090001e007800ecaa02000000000039
:10db9000090037009e0090001e007800007202000d
:10dba00000000000040037009e0090001e00780076
:10dbb000b4b00200000000000080fa00000006007f
:10dbc0000600fa00004f780011479800224798009d
:10dbd000000d81002007980000032600ae00900091
:10dbe000808f50001100320000032800ae0090002a
:10dbf000808f50001300320000032300ae0090001d
:10dc0000808f500001003200130037002e42900038
:10dc10009e4190001e4190009e40780080c2b3005b
:10dc200036a70200000000000b0037002e419000d4
:10dc30009e4090001e4078004872020000000000e4
:10dc4000050037002e4190009e4090001e40780055
:10dc5000fcb00200000000000080fa000000060096
:10dc60000600fa00008fbe00000d8100200798001a
:10dc700000032600ae009000808f50000d0032009f
:10dc800000032800ae009000808f50000d0032008d
:10dc900000032300ae009000808f5000010032008e
:10dca0000b0037001e00be008ca90200000000001f
:10dcb000070037001e00be006c720200000000006a
:10dcc000030037001e00be0020b10200000000006b
:10dcd0000080fa00000006000000fa00000d81003c
:10dce0000080fa000000060000a0fe0086a0a90047
:10dcf0001421ef000000000021e8800082d0210004
:10dd000013002000321ce10005003200080035003d
:10dd1000000000000000000000000000f9ff3700d4
:10dd2000a01680004800de0080587800f5ff37001c
:10dd300021e888009c28ec00e04480009e08e30075
:10dd400003003a001000200030e888001fe1a9001d
:10dd50000080fe00004006000200fa00004f78003c
:10dd60005a780200000000001e41780031c0b30064
:10dd7000c0cdb300c8780200000000006478020043
:10dd8000000000000080fa00000006000400fa0015
:10dd9000004f780011479800224798001e407800f5
:10dda000edff07005a780200000000002e419000ad
:10ddb0009e409000c0cdb300c87802000000000073
:10ddc00064780200000000000080fa0000000600f5
:10ddd0000400fa0020479800314798002e40900038
:10dde000ddff07005a78020000000000be409000ee
:10ddf000c0cdb3006e78020000000000004f780034
:10de000064780200000000001e80fb000080fa0021
:10de1000000006000200fa00004f78001e41780062
:10de200011c9b3000040eb00d8ff07000080fa00e2
:10de3000000006000200fa00004f78001e41780042
:10de400081c6b30010c0b300d0ff07000080fa0005
:10de5000000006000600fa00004f78001e80fb005c
:10de60002007980000042000ae009000808f500032
:10de70001a00320000082000ae009000808f500091
:10de80002700320000022000ae009000808f50007a
:10de9000010032003300370010c0b300e5ff070077
:10dea0001e41780001c8b30010c0b300b7ff0700df
:10deb0001e41780011c8b30010c0b300b3ff0700c3
:10dec00012c0b30021c8b30010c0b300afff0700f9
:10ded0000000eb00100798002400370030c0b300aa
:10dee000d4ff07001e41780001c8b30010c0b30082
:10def000a6ff07001e41780011c8b30010c0b30090
:10df0000a2ff070012c0b30021c8b30010c0b300c5
:10df10009eff07008000eb001107980013003700f8
:10df200070c0b300c3ff07001e41780001c8b300f2
:10df300010c0b30095ff07001e41780011c8b30060
:10df400010c0b30091ff070012c0b30021c8b30096
:10df500010c0b3008dff07000000eb001007980011
:10df6000020037008080eb00110798001e0090002f
:10df70000080fa00000006000600fa00004f78005a
:10df80001e80fb002007980000042000ae009000d7
:10df9000808f50001a00320000082000ae00900070
:10dfa000808f50002700320000022000ae00900059
:10dfb000808f500001003200330037000040eb003a
:10dfc0009cff07001e41780001c8b30010c0b300d9
:10dfd0006eff07001e41780011c8b30010c0b300e7
:10dfe0006aff070012c0b30021c8b30010c0b3001d
:10dff00066ff07000000eb001007980024003700c0
:10e0000010c0b3008bff07001e41780001c8b300a9
:10e0100010c0b3005dff07001e41780011c8b300b7
:10e0200010c0b30059ff070012c0b30021c8b300ed
:10e0300010c0b30055ff07008000eb0011079800e7
:10e040001300370030c0b3007aff07001e4178008c
:10e0500001c8b30010c0b3004cff07001e41780098
:10e0600011c8b30010c0b30048ff070012c0b300ce
:10e0700021c8b30010c0b30044ff07000000eb004c
:10e0800010079800020037008080eb00110798000d
:10e090001e0090000080fa00000006000600fa0052
:10e0a000004f7800114798001e80fb002007980061
:10e0b0002e009000e10f50000f0032002e00900063
:10e0c000e20f5000140032002e0090000000e0002b
:10e0d0000100320018003700d2c0b30081c3b30082
:10e0e00010c0b30029ff07001e40900059ff070031
:10e0f000100798001200370082c0b30081c3b3003c
:10e1000010c0b30021ff07001e4090009aff0700d7
:10e11000100798000a00370022c0b30081c3b30083
:10e1200010c0b30019ff07001e40900092ff0700c7
:10e1300010079800020037000080eb0010079800dd
:10e140001e0090000080fa00000006000a00fa009d
:10e150002007980031079800ae0090003e00900024
:10e16000808f5000030039000080eb0040079800ca
:10e170001e003700be009000f0312000808f50005c
:10e18000030036000080eb004007980017003700be
:10e190002e0090000000e900200798002e0090005b
:10e1a000204798002e0090004800de00304798007d
:10e1b0003e009000004f78003e0090004800de00d6
:10e1c000104798002e41900011c5b30010c0b30055
:10e1d000eefe07003e41900001c5b30010c0b30041
:10e1e000eafe07000000eb00400798004e00900098
:10e1f0000080fa00000006000800fa0020079800de
:10e20000310798000000eb000080fa0000000600d3
:10e210000a00fa002007980031079800ae0090002d
:10e220003e009000808f5000030039000080eb001a
:10e230004007980023003700be009000301f2000e8
:10e24000808f5000030036000080eb0040079800ec
:10e250001c0037002e009000204798002e009000f0
:10e260004800de00304798003e009000004f7800e4
:10e270003e0090004800de00104798003e419000ac
:10e2800001c6b30010c0b300c0fe07002e419000cd
:10e2900011c6b30010c0b300bcfe07001e419000c1
:10e2a00021c6b30010c0b300b8fe07001e417800bd
:10e2b00031c6b30010c0b300b4fe07000000eb008d
:10e2c000400798004e0090000080fa000000060011
:10e2d0000200fa00000f780012c0b300a1c5b3001d
:10e2e00020c0b300a9fe070012c4b30021c3b300cd
:10e2f00010c0b300a5fe07001e00e00011003a00a8
:10e3000000c1eb0081c8b30010c0b3009ffe07003e
:10e3100000c1eb0091c8b30010c0b3009bfe070022
:10e3200082c0b300a1c8b30010c0b30097fe0700bd
:10e3300000c1eb00b1c8b30010c0b30093fe0700ea
:10e340001000370002c2b30081c8b30010c0b30090
:10e350008efe070002c8b30091c8b30010c0b3001e
:10e360008afe070082c0b300a1c8b30010c0b3008a
:10e3700086fe070000c1eb00b1c8b30010c0b300b7
:10e3800082fe07000080fa00000006000600fa0086
:10e39000100798002107980001c9b3000040eb0066
:10e3a0008bfe0700004f78001e0090000000e00088
:10e3b0000300320000c8b3001e4f70000200370097
:10e3c000f0c7b3001e4f60002e0090000000e00078
:10e3d0000300320000c4b3001e4f7000020037007b
:10e3e000f0cbb3001e4f60001e41780001c9b3009e
:10e3f0000040eb0065fe07000080fa000000060008
:10e400000600fa00100798002107980080c9b300a1
:10e41000004f78001e0090000000e00001003a006c
:10e420001e24a0002e0090000000e0000a003a0028
:10e430001e04a0000041eb0051c5b30020c0b30092
:10e4400052fe07000041eb0061c5b30020c0b300dd
:10e450004efe07000800370082c0b30051c5b3006c
:10e4600020c0b30049fe0700c2c0b30061c5b300bd
:10e4700020c0b30045fe07001e41780041c0b30034
:10e4800020c0b30041fe07000080fa000000060033
:10e490000400fa00004f78001147980022479800c6
:10e4a0001e41780041cab30020c0b30037fe070008
:10e4b0001e41900051cab30020c0b30033fe0700d4
:10e4c0002e41900061cab30020c0b3002ffe0700a8
:10e4d0000080fa00000006000400fa00008fbe0071
:10e4e0001e00be004808de00010020000041780048
:10e4f000c1c2b30020c0b30024fe07001e00be004e
:10e500004008de000100200000417800d1c2b300c5
:10e5100020c0b3001dfe07001e00be004809dd003c
:10e520004800de0000007100c808de0000417800ed
:10e53000e1c2b30020c0b30014fe07001e00780043
:10e5400000417800f1c2b30020c0b3000ffe070005
:10e550000080fa0000000600811f7800801f78000c
:10e56000f0ff2700c0128800003020000000b30038
:10e57000d0128800de02a90000000000e002a9001d
:10e580009001090000000000e002a80041e2a8009c
:10e590004602ae00feff3700f0ff2700c0128800e1
:10e5a000004020003001b300d01288004602ae00c7
:10e5b000feff3700f0ff2700c01288000010200087
:10e5c0000030a0000040a000d01288004602ae003b
:10e5d000feff3700f0ff2700c01288000020200057
:10e5e000d01288004602ae00feff3700f0ff270081
:10e5f000c0128800006020000010a000d012880027
:10e600004602ae00feff3700f0ff2700c012880070
:10e6100000702000f005b300d01288004602ae0062
:10e62000feff370001f02000301280000100600082
:10e630000000e000fcff3a003012800001006000a2
:10e640000000e000fcff320030128000010060009a
:10e650000000e000fcff3a00301280000100600082
:10e660000000e000fcff32004662ae00020037000e
:10e67000801280009012800041e2a900f01e20006c
:10e68000101288004362a8004342a8008920a90014
:10e69000a8c0a800a8a0a900a880a9009120a8004f
:10e6a00041e2a8004f007800cf007800000006008b
:10e6b000801f78004022ef004222ef004422ef004a
:10e6c0004822ef004c22ef00c6e2a800e5a2a90014
:10e6d000e582a800e5e2a900e5c2a9004002a90080
:10e6e0004022a90040a2a9004122a90040c2a800de
:10e6f0004102a9004142a900f00e2000101288003a
:10e700004362a9004342a800300020002012880084
:10e710004c02a8004802a8008920a9009120a90065
:10e7200041e2a9004f007800000006008920a900fe
:10e73000809fbe00829fbe008012800090128000e9
:10e74000a0128000b01280008808e20026003a0083
:10e750008c08e200240032003400f8004400f80085
:10e760004440a80070448000a0018800014580005a
:10e77000fe73020000000000110078000000a100fc
:10e78000c0128800fe730200000000001100780033
:10e790000000a100d0128800fe73020000000000fb
:10e7a000110078000000a100e0128800fe73020052
:10e7b00000000000110078000000a100f0128800a5
:10e7c0008ca8ed008ca8ed0001458800a101800017
:10e7d000714488004400f9003400f9004f01be0084
:10e7e0004f00be00004006008a28ef0088a8ef0016
:10e7f0004f01be004f00be0000400600e280400016
:10e8000004003900a1018000e1804000a1018800de
:10e8100001002800000006000200fa00e202a80041
:10e820000000eb00000f7800010037001e0fe80029
:10e83000f07022009e0f1000fcff3400587302009d
:10e8400000000000ac720200000000000080fa002e
:10e85000000006000400fa00000f7800110798007d
:10e860008aa8ef008828ef009e0090001e00780024
:10e8700048740200000000000080fa00000006005a
:10e880000000fa00e202a9000080fa000000060081
:10e89000811f7800821f78004100dd0003003700ef
:10e8a0004f017800cf007800000006006144880026
:10e8b0000001eb00c1272d0081004000030039005a
:10e8c0000200280082804000120020004400f8006e
:10e8d0003400f8004440a80010002000020040006e
:10e8e000a001880000000000b074020000000000d9
:10e8f000110078000000a100c0128800b07402006e
:10e9000000000000110078000000a100d012880073
:10e91000b074020000000000110078000000a100a7
:10e92000e0128800b07402000000000011007800be
:10e930000000a100f01288008ca8ed008ca8ed006a
:10e9400001458800a1018000714488003400f9006d
:10e95000000000004400f9008920a900d0ff370022
:10e96000e280400004003900a1018000e180400005
:10e97000a101880001002800000006000000fa0044
:10e980000000370006c2bf00614060000004e000e4
:10e99000fcff3a0006c2bf00644060000004e000d3
:10e9a000f8ff3a0006c2bf00684060000004e000c3
:10e9b000f4ff3a0006c2bf00704060000004e000af
:10e9c000f0ff3a0009c2bf000044b2000004e000ba
:10e9d000ecff3a000080fa00000006000400fa0094
:10e9e000600920002010880007e2a90007e2a800c3
:10e9f00085c0a90085a0a900b10920009140780038
:10ea000080cfb30000c060005040b3009be0b7006f
:10ea10008da0a9000071220001002000008fbe001f
:10ea2000040037000080eb008080eb001e0f4000e8
:10ea30005e9748001e00be00e00f5000e08f5800b7
:10ea4000f8ff3a00100020000080fa0000000600e5
:10ea50000000fa0007e2a90085c0a90085a0a9006e
:10ea60008dc0a9008da0a900100020000080fa0030
:10ea7000000006000400fa006000b800008fbe002d
:10ea800007e2a90085c0a90085a0a9008da0a90062
:10ea90000000eb00401088000071220001002000ff
:10eaa000008fbe00040037000080eb008080eb0088
:10eab0001e0f40005e9748001e00be00e00f500091
:10eac000e08f5800f8ff3a00c4ff07000f0007006e
:10ead0000071220001002000008fbe0004003700fa
:10eae0000080eb008080eb001e0f40005e97480026
:10eaf0001e00be00e00f5000e08f5800f8ff3a0003
:10eb0000100020000080fa00000006000000fa005b
:10eb100085c0a9008dc0a800100020000080fa0068
:10eb2000000006000000fa0085c0a9008dc0a90001
:10eb3000100020000080fa00000006000600fa0025
:10eb40002116220010c0b3008048780008c2bf0020
:10eb5000704060000004e000170032000602a800c8
:10eb60000071220001002000008fbe000b00370062
:10eb700020162200104078000004e00003003a0054
:10eb800010002000200798000d0037000080eb00e7
:10eb90008080eb001e0f40005e9748001e00be0004
:10eba000e00f5000e08f5800f1ff3a008000eb00ca
:10ebb00021079800020037000000eb0020079800b2
:10ebc0002e0090000080fa00000006000600fa0007
:10ebd0002116220060c0b3008048780008c2bf0040
:10ebe000684060000004e000170032000622a80020
:10ebf0000071220001002000008fbe000b003700d2
:10ec000020162200104078000004e00003003a00c3
:10ec100010002000200798000d0037000080eb0056
:10ec20008080eb001e0f40005e9748001e00be0073
:10ec3000e00f5000e08f5800f1ff3a008000eb0039
:10ec400021079800020037000000eb002007980021
:10ec50002e0090000080fa00000006000600fa0076
:10ec60002116220050c0b300804878000642a80058
:10ec70000071220001002000008fbe000b00370051
:10ec800020162200104078000004e00003003a0043
:10ec900010002000200798000a0037000080eb00d9
:10eca0008080eb001e0f40005e9748001e00be00f3
:10ecb000e00f5000e08f5800f1ff3a008000eb00b9
:10ecc000210798002e0090000080fa000000060046
:10ecd0000600fa002116220030c0b30080487800f8
:10ece00006c2bf00614060000004e00010003a006e
:10ecf00006c2bf00644060000004e0000c003a005f
:10ed000006c2bf00684060000004e00008003a004e
:10ed100006c2bf00704060000004e00004003a003a
:10ed200006c2bf00624060000004e0000300320041
:10ed30000000eb00200798001700370006a2a9008a
:10ed40000682a8000071220001002000008fbe0092
:10ed50000b00370020162200104078000004e0006d
:10ed600003003a0011002000210798000a00370034
:10ed70000080eb008080eb001e0f40005e97480093
:10ed80001e00be00e00f5000e08f5800f1ff3a0077
:10ed90008000eb00210798002e0090000080fa0010
:10eda000000006000600fa002116220030c0b30061
:10edb0008048780006c2bf00614060000004e000a7
:10edc00010003a0006c2bf00644060000004e0008a
:10edd0000c003a0006c2bf00684060000004e0007a
:10ede00008003a0006c2bf00704060000004e00066
:10edf00004003a0006c2bf00624060000004e00068
:10ee0000030032000000eb002007980017003700d5
:10ee100006a2a8000682a8000071220001002000be
:10ee2000008fbe000b003700201622001040780033
:10ee30000004e00003003a001100200021079800c0
:10ee40000a0037000080eb008080eb001e0f4000be
:10ee50005e9748001e00be00e00f5000e08f580093
:10ee6000f1ff3a008000eb00210798002e0090008f
:10ee70000080fa00000006000a00fa00300798003f
:10ee8000007122000100200010079800210798005f
:10ee90000040eb00004f78002116220040c0b30074
:10eea00080487800007122000100200010079800bf
:10eeb000210798001d00370006c2bf0061406000b6
:10eec0000004e00013003a0006c2bf006440600086
:10eed0000004e0000f003a0006c2bf006840600076
:10eee0000004e0000b003a0006c2bf007040600062
:10eef0000004e00007003a0009c2bf000044b2006d
:10ef00000004e00003003a0010c0b300004f780096
:10ef10000b0037001e009000ae0090006100500012
:10ef2000e080580010079800210798001e0090000c
:10ef3000ae009000e00f5000e08f5800deff3a0076
:10ef40001e04e00003003a000000eb0040079800b8
:10ef50001e0037000662a800006a28001100200089
:10ef60001007980021079800110037002016220092
:10ef7000104078000004e00007003a000010800014
:10ef8000804078003e00900001487800100020008a
:10ef9000400798000d0037001e009000ae00900062
:10efa00061005000e0805800100798002107980089
:10efb0001e009000ae009000e00f5000e08f58005f
:10efc000eaff3a000000eb00400798004e00900076
:10efd0000080fa00000006000800fa004047980090
:10efe0002116220020c0b300804878004e409000d7
:10eff0000000fb00101088000071220001002000ba
:10f00000008fbe000b003700201622001040780051
:10f010000004e00003003a001000200030079800d0
:10f020000a0037000080eb008080eb001e0f4000dc
:10f030005e9748001e00be00e00f5000e08f5800b1
:10f04000f1ff3a008000eb00310798003e0090008d
:10f050000080fa0000000600809fbe003400f80027
:10f0600010002000a00188000000fa0085c0a9005f
:10f07000211622000040eb00804878000080fa0052
:10f080003400f9004f00be00004006000000fa0006
:10f09000ee740200000000000080fa00000006008c
:10f0a0000000fa0028750200000000000080fa004d
:10f0b000000006000000fa00867502000000000053
:10f0c0000080fa00000006000000fa0092750200bd
:10f0d000000000000080fa00000006000400fa00b2
:10f0e00020479800314798000040eb00004f78001f
:10f0f0002100370010c0b300004f78009e75020059
:10f10000000000001e4f60002e409000ec770200cf
:10f11000000000001e4f60003e409000ec770200af
:10f12000000000001e4f6000e675020000000000b5
:10f130001e4f60002e4090000040e800ec77020077
:10f14000000000001e4f60000e00e8003c77020047
:10f15000000000001e4f6000d27602000000000098
:10f160002e760200000000001e04e00004003a00b9
:10f170003a750200000000001e04e000ddff3200ce
:10f180001e4090000000fb000080fa000000060016
:10f190000600fa002047980031479800424798003f
:10f1a0000040eb00004f78001800370010c0b3009b
:10f1b000004f78009e750200000000001e4f6000a6
:10f1c0002e409000ec770200000000001e4f60000f
:10f1d0003e409000ec770200000000001e4f6000ef
:10f1e0004e409000ec770200000000001e4f6000cf
:10f1f0002e760200000000001e4f60001e04e0009a
:10f2000004003a003a750200000000001e04e0000d
:10f21000e6ff32001e00fb000080fa00000006003e
:10f220000c22ef000e22ef000ee2a9000ec2a90090
:10f230008520a9008d20a8000de2a8007000200004
:10f24000a01088008540a9008d40a80081e0a90099
:10f25000c0048000f1002f000080600001552000f4
:10f2600000804000c00488000fe2a8000f42a80000
:10f270004028ef004228ef0000000600809fbe00fb
:10f280008520a9000e22a9000e02ab000800320062
:10f2900000428000f003b2000180200081004000a5
:10f2a00012c2bf00804878004028ec00f6ff37000b
:10f2b0004f00be0000400600004280001142800066
:10f2c0000100500000000600014280001242800050
:10f2d0000208e10008003200f203b20001802000c1
:10f2e0000281400092407800014878004228ec00fa
:10f2f00010002000000006000000eb0000000600e7
:10f300008540a900809fbe00821f78009408e2001b
:10f31000150032009008e200160032009208e20068
:10f320001400320081448000420020000f22af0010
:10f33000feff3700904480000000e000070032002c
:10f340000000e90092a8b7003140780010e2b70051
:10f350000201e900f5ff3a00020037009028ef00b3
:10f3600001003700814488004f0178004f00be0043
:10f370000040060000002000a04488004f017800f3
:10f380004f00be00004006009408e200feff3a0075
:10f390008d40a9008100e90091448800b0407800c8
:10f3a000811088008044880011002000a14488005a
:10f3b0008d40a80000000600a04480000000060068
:10f3c000809fbe008700a9001822a9001802ab0088
:10f3d0000800320020448000f003b2004184200085
:10f3e000810040001cc2bf00804878008428ec00e7
:10f3f000f6ff37004f00be000040060020448000aa
:10f4000031448000010050000000060021448000cb
:10f41000324480000208e10008003200f203b2002a
:10f420004184200002814000924078000148780029
:10f430008628ec0010002000000006000000eb0011
:10f44000000006008720a900809fbe00821f780070
:10f450009a08e200150032009608e2001600320019
:10f460009808e20014003200b144800042002000fd
:10f470001922af00feff3700c04480000000e0000a
:10f48000070032000000e90098a8b700314078007a
:10f490001ae2b7000201e900f5ff3a000200370066
:10f4a0009628ef0001003700b14488004f01780032
:10f4b0004f00be000040060000002000d04488003d
:10f4c0004f0178004f00be00004006009a08e2009d
:10f4d000feff3a008f20a9008100e900c1448800a6
:10f4e000b0407800d1108800b0448800110020009e
:10f4f000d14488008f20a80000000600d04480007e
:10f50000000006000200fa00467802000000000039
:10f510003a750200000000005a7802000000000066
:10f52000f1c0b300c0c3b3006e7802000000000059
:10f53000004f7800647802000000000000c4b300af
:10f540009e4f100004003a00211a220010c0b300a0
:10f550008048780003003700211a22000040eb00a9
:10f56000804878000080fa00000006000000fa00e1
:10f57000c4c2a900c4e2a900c522a900c582a9008d
:10f58000c542a900c5a2a900c5c2a900c5e2a9003b
:10f59000c0c2a900c0e2a900c122a900c182a9007d
:10f5a000c142a900c1a2a900c1c2a900c1e2a9002b
:10f5b000d022a900cc22a900d042a900cc42a900a7
:10f5c000e2e2a900e302a900e802a900e822a900fa
:10f5d000dee2a900df02a900e402a900e422a900fa
:10f5e000e202a900de02a900d602a900d622a900e3
:10f5f000d642a900d662a900d682a900d6a2a90047
:10f60000d6c2a900d6e2a900d202a900d222a9003e
:10f61000d242a900d262a900d282a900d2a2a90036
:10f62000d2c2a900d2e2a900d1a2a900cda2a9000c
:10f63000e842a900e862a900e442a900e462a90046
:10f64000de22a800dec2a800e4c2a800e4e2a8000e
:10f65000e502a800e522a800d302a800d322a80052
:10f66000d342a800d362a800d382a800d3a2a800e6
:10f67000d3c2a800d3e2a800a2ff0700201a2200ec
:10f68000104078000004e000020032003eb60200a4
:10f69000000000000080fa00000006000000fa00f0
:10f6a000201a2200104078000080fb000080fa0041
:10f6b000000006000000fa000000eb00800888004f
:10f6c0000111200091407800f0ccb30000c0600030
:10f6d00010e1b7000000eb0030088800205c20003b
:10f6e0006008880084c0a9008cc0a80011e1a800af
:10f6f0000080fa00000006000000fa0011e1a900f5
:10f700000080fa00000006000800fa0010079800c8
:10f7100021079800200d8100000f78000b003700b2
:10f720001e007800b00090001e009000808f5000f6
:10f7300003003a0011002000310798002100370033
:10f740001e007800c0009000010f78001e00e0004d
:10f75000f3ff3a00a0002000961002000000000015
:10f76000000f78001e00e00003003a0010002000a7
:10f770002012020000000000ae0090001e00780081
:10f78000010878009e0078000000eb0090009800cf
:10f790009e00780010c0b300c04098001e007800a2
:10f7a0009e00900031009800210d81001e0078001d
:10f7b000410098001e007800200d890011002000f3
:10f7c000310798003e0090000080fa00000006001b
:10f7d0000800fa00200798000000eb0010079800ce
:10f7e000200d8100000f78001b0037001e007800fc
:10f7f000b00090002e009000808f500011003a0061
:10f800001e0090000000e000050032001e0078009d
:10f81000c00090001e0090004100980003003700d7
:10f820001e00780040009000200d89001e00780026
:10f83000ba110200000000001100200031079800fa
:10f84000090037001e007800100798001e0078009d
:10f85000c0009000010f78001e00e000e3ff3a00b6
:10f8600020002000300798003e0090000080fa0041
:10f87000000006000800fa00100798002107980011
:10f88000200d8100000f78000e0037001e00780068
:10f89000b00090001e009000808f500006003a00db
:10f8a000ae0090001e0078000108780011002000d2
:10f8b00031079800070037001e007800c000900054
:10f8c000010f78001e00e000f0ff3a002000200049
:10f8d000300798003e0090000080fa00000006000b
:10f8e0000600fa0010079800200d8100000f780034
:10f8f0000e0037001e007800b00090001e0090003f
:10f90000808f500006003a009e0078000000eb0057
:10f910009000980011002000210798000700370090
:10f920001e007800c0009000010f78001e00e0006b
:10f93000f0ff3a0020002000200798002e009000e1
:10f940000080fa00000006000600fa001007980088
:10f95000200d8100000f78000e0037001e00780097
:10f96000b00090001e009000808f500006003a000a
:10f970009e0078000040eb00c0409800110020007d
:10f9800021079800070037001e007800c000900093
:10f99000010f78001e00e000f0ff3a002000200078
:10f9a000200798002e0090000080fa00000006005a
:10f9b0000600fa0010079800200d8100000f780063
:10f9c0000e0037001e007800b00090001e0090006e
:10f9d000808f500006003a009e00780010c0b300ef
:10f9e000c040980011002000210798000700370050
:10f9f0001e007800c0009000010f78001e00e0009b
:10fa0000f0ff3a0020002000200798002e00900010
:10fa10000080fa00000006003600f800809fbe005b
:10fa2000829fbe00849fbe00869fbe003400f80007
:10fa300010002000a00188000200fa00200d8100c3
:10fa4000000f780084c0a9001e0037001e00780057
:10fa500040409000e14f500017003a001e0078002f
:10fa6000100078000000e000130032001e00780053
:10fa7000100090008000e8001e007800110098003f
:10fa80001e00780010009000800078001e007800b2
:10fa9000100078000000e900808f5000060036005a
:10faa0001e00780030009000000001009e007800e9
:10fab0000000eb00900098001e007800c00090004d
:10fac000010f78001e00e000e0ff3a000080fa001d
:10fad0003400f9004f03be004f02be004f01be00cc
:10fae0004f00be003600f900004006000000fa009a
:10faf000dec2a8008200a8008400a9008c00a80033
:10fb00000080fa00000006003600f800809fbe006a
:10fb1000829fbe00849fbe00869fbe003400f80016
:10fb200010002000a00188000000fa008c00a9004d
:10fb30005101200060dc2700847b020000000000ef
:10fb4000f11722000040eb0080487800f0172200f7
:10fb500090407800e017220001487800e01722006a
:10fb60009040780000182200014878000080fa00d8
:10fb70003400f9004f03be004f02be004f01be002b
:10fb80004f00be003600f900004006000200fa00f7
:10fb9000c00c8100e10f40001e003a00e0c2bf002f
:10fba0000044b2000004e000080032008c00a8000d
:10fbb0008400a90060dc2700e87b02000000000050
:10fbc0000080eb00c00c89006d0037009100200020
:10fbd00060dc27003a7c020000000000f1172200e0
:10fbe0000040eb0080487800f01722009040780039
:10fbf000e017220001487800e017220090407800ca
:10fc000000182200014878000000eb00c00c8900b9
:10fc10005b003700c00c8100e10f500010003a007b
:10fc2000e0c2bf000080fb004600de0061406000d3
:10fc3000804078000018220001487800210120004f
:10fc400060dc27003a7c0200000000001100200068
:10fc5000100020000a990200000000004800370050
:10fc6000c00c8100e10f500015003400c00c810071
:10fc7000e60f500012003c00e0c2bf000080fb0015
:10fc80004600de0061406000104798001e40900072
:10fc90008080fb00c00c8100660010000008dd00c1
:10fca00010479800e0172200904078001e40900016
:10fcb00080c04000e0172200014878003000370083
:10fcc000c00c8100e60f500013003400c00c81000e
:10fcd000ec0f500010003c00e0c2bf000080fb00b1
:10fce0004600de0061406000004f78009e80fb000f
:10fcf000c00c81006c0010000008dd00004f78008f
:10fd0000f0172200104078009e404000f0172200bb
:10fd1000014878001a003700c00c8100ed0f500038
:10fd200017003a008000eb00100020000a99020042
:10fd3000000000008c00a8008400a90060dc2700ff
:10fd4000e87b0200000000000080eb00c00c89008e
:10fd500000182200904078006019220001487800c5
:10fd6000e017220090407800101822000148780027
:10fd7000f0172200904078002018220001487800f7
:10fd8000c00c8100e10f400003003200c00c810074
:10fd90000000e800c00c89000080fa0000000600a6
:10fda0000000fa0060192200104078000080fb007b
:10fdb0000080fa00000006000000fa00101822007f
:10fdc000104078000080fb000080fa000000060070
:10fdd0000000fa0020182200104078000080fb008c
:10fde0000080fa00000006000a00fa0010079800e0
:10fdf0000000eb00000f78004e7b020000000000c6
:10fe00000004e0003a003200e01622009040780042
:10fe100000c4b30080cf500008003a000211220055
:10fe2000e1102200c010220098b60200000000007d
:10fe3000e11622000040eb00804878001e00900090
:10fe4000300798003e009000e10f50001100320092
:10fe50003e009000e10f5000040039003e00900089
:10fe6000e20f5000150032001e00370071088100bb
:10fe7000c0078100008f50001e007800c480de00a3
:10fe80001e0078004680de00808050002107980028
:10fe90004c00370061088100b0078100008f5000de
:10fea0001e007800c480de001e0078004680de0060
:10feb00080805000210798004200370081088100af
:10fec000e00c8100008f50001e007800c480de002e
:10fed0001e0078004680de008080500021079800d8
:10fee00038003700a029200020079800350037008f
:10fef0001e009000400798004e009000e10f500057
:10ff0000140032004e009000e10f50000400390050
:10ff10004e009000e20f50001b0032002700370017
:10ff20009e009000620b8100200320000088b90031
:10ff300002004000800040008088210000804000d6
:10ff400090007800b0078100808050002107980061
:10ff50001c0037009e009000620b810020032000ef
:10ff60000088b90002004000800040008088210025
:10ff70000080400090007800c00781008080500021
:10ff8000210798000f0037009e009000620b81004f
:10ff9000200320000088b9000200400080004000db
:10ffa000808821000080400090007800e00c8100f3
:10ffb000808050002107980002003700a02920000f
:10ffc000200798002e0090000080fa000000060034
:10ffd0001400fa0050079800610798006000b8000c
:10ffe00030079800410798004e7b02000000000097
:10fff0000004e0005c003200e0162200904078002f
:020000040001f9
:1000000000c4b30080cf500008003a000211220063
:10001000e1102200c010220098b60200000000008b
:10002000e11622000040eb0080487800a019220071
:10003000104078000004e0001b0032005e009000d9
:10004000000f98000e089000e10f50000b003200e6
:100050000e089000e10f5000040039000e089000d7
:10006000e20f5000090032000c0037000ab702000e
:10007000000000007007980076003700e6b6020026
:100080000000000070079800720037002eb70200d1
:1000900000000000700798006e003700a0292000c3
:1000a000700798006b0037005e009000100f9800fa
:1000b0001e089000e10f5000120032001e08900050
:1000c000e10f5000040039001e089000e20f5000bc
:1000d000170032002100370070088100000f7800ff
:1000e0001e007800c480de001e0078004680de001e
:1000f00080805000008020008080400071079800c0
:100100005400370060088100000f78001e0078005e
:10011000c480de001e0078004680de008080500033
:10012000008020008080400071079800490037005f
:1001300080088100000f78001e007800c480de0077
:100140001e0078004680de00808050000080200085
:1001500080804000710798003e003700a0292000f1
:10016000700798003b0037005e009000e20f5000df
:1001700031003e006e0090000000e0002e003200d2
:10018000ee00900020032000808f50002a003e00e7
:100190000000eb0020079800610b81006e009000ca
:1001a000008050003003b00022032000110009003d
:1001b0000280d8008000fd00100798001a00370068
:1001c000de0090001e019000200320000088b9008e
:1001d0000200400080004000808821000080400034
:1001e000100078006101b9003e009000ce00900040
:1001f00000004100818049003007980041079800c5
:100200002e0090000000e800200798001e009000db
:100210000000e80022032000110009000200d800bd
:100220008000fd0010079800ae0090006e00900066
:10023000808f5000e2ff39006e0090006101b8002d
:100240003e009000ce009000640502000000000017
:10025000700798007e0090000080fa000000060001
:100260000000fa004e7b0200000000000004e000e5
:100270000a0032000000eb00dbfe0700d007890017
:1002800010002000d8fe0700e007890020002000b1
:10029000d5fe0700f0078900150037005100200047
:1002a0000000eb004aff070080007800b0078100e3
:1002b00000805000d007890051002000100020006d
:1002c00043ff070080007800c007810000805000d5
:1002d000e007890051002000200020003cff0700bb
:1002e00080007800e00c810000805000f007890059
:1002f0000080fa00000006000000fa00889fbe009f
:100300008a9fbe00d6ff0700d00781006103b900b5
:10031000d00781006102b9008600780004007800ef
:10032000000db80005b0b9000b01780000014100d4
:1003300007a0b9000001410082057800e0078100b4
:100340006104b900e00781006103b900880078000a
:1003500006007800000ab80007c0b900050178005f
:100360000001410009b0b90000014100820278009b
:100370000a0542008b854a00f00781006104b9003c
:10038000f00781006103b90088007800060078005a
:10039000000ab80007c0b90005017800000141005b
:1003a00009b0b90000014100820278000a00420051
:1003b0008b804a00d6020200000000008205020085
:1003c000000000000008890011088900d0078100a2
:1003d0006103b900d00781006102b900860078008e
:1003e00004007800000db80005b0b9000b017800da
:1003f0000001410007a0b90000014100820578001a
:10040000e00781006104b900e00781006103b900e1
:100410008800780006007800000ab80007c0b9001c
:10042000050178000001410009b0b9000001410058
:10043000820278000a0042008b804a00d602020045
:100440000000000082050200000000000004be0061
:10045000f0078100cf80de00d6020200000000001d
:100460000801be002c03020000000000c2092300a6
:1004700053262c00ea0302000000000002002000c6
:10048000432b2400540402000000000040088900af
:1004900051088900400881005108810002002000b5
:1004a000030a240060050200000000000000e000d4
:1004b0000900350040088100510881000200200039
:1004c00003322400ec050200000000000000e00000
:1004d00001003c00040037006000b80020088900db
:1004e0003108890016003700e0078100cf80de0068
:1004f000d6020200000000000004be00d007810008
:10050000cf80de00d6020200000000000801be001d
:100510002c03020000000000c2092300532624001f
:10052000ea03020000000000020020004333240020
:1005300054040200000000002008890031088900ee
:100540004f05be004f04be000080fa000000060008
:100550000000fa00a119220010c0b3008048780002
:10056000210320000000eb0099fe0700b00789007e
:10057000210320001000200095fe0700c00789001d
:100580004e7b0200000000000004e0000700320083
:1005900021032000200020008dfe070001002c0018
:1005a00001004000e00c8900060037002103200014
:1005b0002000200086fe070001d02f00010040002f
:1005c000e00c8900a11922000040eb00804878006f
:1005d0000080fa00000006000c00fa00881f780076
:1005e0000004780044ff0700000881001108810022
:1005f000008fbe002008810031088100200798008c
:100600003107980040088100510881004007980098
:10061000510798008e007800080078001101be0094
:100620000288be0064004000e48040001101be006a
:100630000288be0064004000e48040001101be005a
:100640000288be00080078004f0478000080fa009d
:10065000000006000000fa0027ff070040088100a4
:10066000510881000080fa00000006000000fa0036
:1006700021ff070020088100310881000080fa0076
:10068000000006000000fa001bff070000088100c0
:10069000110881000080fa00000006000600fa0040
:1006a000881f780000047800edfe0700d007810065
:1006b000000f7800e007810010079800f007810024
:1006c000200798001e00be00008cbe00ae00900007
:1006d00021049800080078004f0478000080fa0098
:1006e000000006000000fa00ddfe0700d0078100d0
:1006f0000080fa00000006000000fa00d8fe0700a3
:10070000e00781000080fa00000006000000fa0007
:10071000d3fe0700f00781000080fa000000060009
:100720001600fa006000b800008fbe00cfff07007f
:10073000008fbe00a0078100cf80de00d60202003d
:10074000000000001e01be00520402000000000074
:100750001e05020000000000200f98002e089000e7
:100760000000e00003003d00ae0890008100ea00b8
:10077000210f98002e0990006110b900d6020200e6
:100780000000000002002000030a2400ec05020023
:10079000000000000000e00001003c0061013700a3
:1007a000c5e2a900c5c2bf000080fb004700de0013
:1007b000614060004601dd00512c2000914078002e
:1007c000f0cbb30000c0600002407000c5e2b7008b
:1007d000c5c2bf000080fb004600de006140600033
:1007e000614060004501dd00512c200091407800ff
:1007f000f0cdb30000c0600002407000c5e2b70059
:10080000c5c2bf000080fb004500de006140600003
:10081000614060004201dd00512c200091407800d1
:10082000b0cfb30000c0600002407000c5e2b70066
:10083000c5c2bf000080fb004200de0061406000d6
:10084000614060004401dd00512c2000914078009f
:10085000f0ceb30000c0600002407000c5e2b700f7
:10086000c5c2bf000080fb004400de0061406000a4
:100870006140600000414000512c20009140780010
:10088000d0cfb30000c0600002407000c5e2b700e6
:10089000c5c2bf000080fb000000d10061406000c5
:1008a000c700dd00c4c2bf000074a1000140700099
:1008b000c4e2b700c4c2bf000080fb004700de00f6
:1008c000614060004601dd00412c2000914078002d
:1008d000f0cbb30000c0600002407000c4e2b7007b
:1008e0000040eb002057980002002c00833a2400bf
:1008f0001e00be00ec050200000000000000e00049
:1009000001003c000200370011c0b30021579800dd
:100910000041eb001257980002002000431b240006
:100920001e00be0060050200000000000000e000a4
:10093000010034000200370010c0b30010579800c7
:10094000ae5090001e51900002c070000004a20042
:100950000004e00012003a000040eb00005798004d
:1009600002002800634224001e00be00f0050200c1
:10097000000000000000e00001003a000200370023
:1009800011c0b300015798000e5090000004a2005f
:100990000004e00002003a00c4c2a800dd003700f5
:1009a0000041eb00724f980002002000431b24001e
:1009b0001e00be00ec050200000000000000e00088
:1009c00001003c000200370010c0b300704f9800d7
:1009d0007e4890000004a2000004e00012003a00eb
:1009e0008040eb00614f9800020020007328240033
:1009f0001e00be0060050200000000000000e000d4
:100a0000010034000200370012c0b300624f9800aa
:100a10006e4890000004a2000004e00002003a00ca
:100a2000c5e2a800bb0037000040eb00504f980023
:100a300002002000732824001e00be00ec05020006
:100a4000000000000000e00001003c000200370050
:100a500011c0b300514f98005e4890000004a200fe
:100a60000004e00012003a000041eb00424f980001
:100a700002002000132e24001e00be0060050200ac
:100a8000000000000000e000010034000200370018
:100a900010c0b300404f98004e4890000004a200e0
:100aa0000004e00002003a00c5c2a8009900370027
:100ab0008040eb00314f980002002000132e2400ec
:100ac0001e00be00ec050200000000000000e00077
:100ad00001003c000200370012c0b300324f980002
:100ae0003e4890000004a2000004e00012003a001a
:100af0000040eb00204f980002002800d331240072
:100b00001e00be0060050200000000000000e000c2
:100b1000010034000200370011c0b300214f9800db
:100b20002e4890000004a2000004e00002003a00f9
:100b3000c5a2a800770037000041eb00124f9800d3
:100b400002002800d33124001e00be00ec05020084
:100b5000000000000000e00001003c00020037003f
:100b600010c0b300104f98001e4890000004a2006f
:100b70000004e00012003a008040eb00014f9800b2
:100b800002002800a33424001e00be0060050200fd
:100b9000000000000000e000010034000200370007
:100ba00012c0b300024f98000e4890000004a2004b
:100bb0000004e00002003a00c542a80055003700da
:100bc0000040eb007047980002002800a334240086
:100bd0001e00be00ec050200000000000000e00066
:100be00001003c000200370011c0b30071479800bb
:100bf0007e4090000004a2000004e00012003a00d1
:100c00000041eb006247980002002800733724007f
:100c10001e00be0060050200000000000000e000b1
:100c2000010034000200370010c0b3006047980094
:100c30006e4090000004a2000004e00002003a00b0
:100c4000c582a800330037008040eb005147980070
:100c500002002800733724001e00be00ec050200cd
:100c6000000000000000e00001003c00020037002e
:100c700012c0b300524798005e4090000004a200ea
:100c80000004e00012003a000040eb0040479800ea
:100c900002002400233924001e00be00600502006b
:100ca000000000000000e0000100340002003700f6
:100cb00011c0b300414798004e4090000004a200cc
:100cc0000004e00002003a00c522a800110037002d
:100cd00002002400233924001e00be00ec0502009f
:100ce000000000000000e00001003c0009003700a7
:100cf00002002c00833a24001e00be0060050200a2
:100d0000000000000000e000010034000100370096
:100d1000c4e2a8001e00be001e0502000000000084
:100d2000a00789000080fa00000006000200fa0017
:100d3000004f780000b4020000000000e0ce880000
:100d400010c0b3009e4f100004003a00c1622100a1
:100d500010c0b3008048780003003700c162210052
:100d60000040eb00804878000000eb000015880090
:100d70000000eb00101588000000eb002015880033
:100d80000000eb0030158800e0ce8000ea0f500034
:100d90000a003a009109200091407800f0c8b300a1
:100da00000c0600001c6b3000140700099e0b700c8
:100db000a802a900a822a90002003700a802a800e2
:100dc000a822a800a842a900a862a900a882a90098
:100dd000a8a2a900a8c2a900a8e2a900a902a90086
:100de000a922a900a942a900a962a900a982a90073
:100df000a9a2a900a9c2a900a9e2a900aa02a90062
:100e0000aa22a900aa42a800aa62a800aa82a80051
:100e1000aaa2a900aac2a900aae2a900ab02a9003d
:100e2000ab22a900ab42a900ab62a900ab82a9002a
:100e3000aba2a900abc2a900abe2a900112a200015
:100e400091407800c0cfb30000c06000a1e2b700bd
:100e5000a042a800012a20009140780000ceb300f3
:100e600000c07000a0e2b700212a20009140780065
:100e700030ccb30000c060000034a000a2e2b70094
:100e8000a342a800512a20009140780000ceb30070
:100e900000c060000004a000a5e2b700c06221000d
:100ea000104078000004e00007003200412a2000d2
:100eb0009140780000ccb30000c060003041b30026
:100ec000a4e2b70007003700412a200091407800d3
:100ed00000ccb30000c0600071c2b30001407000dc
:100ee000a4e2b7008560a9008d60a800a1e2a80077
:100ef000c0622100104078000004e00005003a00c4
:100f000000000000610b810000032000808f500072
:100f1000fbff36004e7b0200000000000004e000f2
:100f2000020032000000eb00e00c89000080fa00b3
:100f300000000600809fbe00821f78003400f80089
:100f400010002000a00188000c00fa00a16221001e
:100f50000040eb0080487800b16221000040eb00c7
:100f6000804878008560a900e01622009040780053
:100f7000f0c3b30080cf500005003e00e016220011
:100f8000104078008040e800e01622000148780018
:100f9000800b8100e10f400003003200800b8100d4
:100fa0000000e800800b8900c0622100104078003a
:100fb0000004e0002e00320000282000000f78001e
:100fc000510b81001e0078001000780000017800ad
:100fd000818040000063210000804000020878000a
:100fe0001e8fe800510b81001e0078001000780071
:100ff0000001780001804000810c200080804000ca
:101000000063210000804000020878001e8fe80085
:10101000510b81001e00780010007800000178005c
:101020000180400001192000808040000063210001
:1010300000804000020878001e8fe800500b8100fd
:101040000000e800500b8900510b810030062000a1
:10105000808f5000190236000000eb00500b890011
:10106000b162210010c0b30080487800130237003d
:10107000a1e2a900c001200050158800212a20000b
:101080009140780030ccb30000c060000034a00074
:10109000a2e2b700412a20009140780000ccb300c2
:1010a00000c0600071c2b30001407000a4e2b7004c
:1010b000e062210090407800d0c3b30080cf5000a0
:1010c0000f003a00c00f200050158800212a200090
:1010d0009140780030ccb30000c060004041b300c4
:1010e000a2e2b700412a20009140780000ccb30072
:1010f00000c060003041b300a4e2b7006e003700ca
:10110000e062210090407800e0c3b30080cf50003f
:1011100033003a00212a20009140780030ccb300ff
:1011200000c060000044a000a2e2b700412a2000f5
:101130009140780000ccb30000c060007041b30063
:10114000a4e2b700d0622100104078000080fb00cc
:10115000500798005e009000e20f50001700320028
:10116000de009000e28f500007003c005e0090001f
:101170000000e0000b003200de009000e18f500024
:101180000b0032004c0037005e009000e30f50006f
:101190000d003200de009000e48f50000d003200a0
:1011a00045003700c011210050158800420037006b
:1011b000c0212200501588003f003700c0412400a4
:1011c000501588003c003700c08128005015880069
:1011d00039003700f0012000501588003600370034
:1011e000e062210010407800e24f500032003a00e7
:1011f000212a20009140780030ccb30000c060006c
:101200000044a000a2e2b700412a200091407800eb
:1012100000ccb30000c060007041b300a4e2b7008e
:10122000d0622100104078000080fb004007980049
:101230004e009000e20f500017003200ce009000e8
:10124000e28f500007003c004e0090000000e000dc
:101250000b003200ce009000e18f50000b003200f6
:10126000150037004e009000e30f50000d003200d3
:10127000ce009000e48f50000d0032000e003700c9
:10128000c0112100501588000b003700c02122003a
:101290005015880008003700c04124005015880010
:1012a00005003700c0812800501588000200370073
:1012b000f001200050158800a1e2a80000282000bd
:1012c000000f7800e062210090407800f0c3b30086
:1012d00080cf500004003a00d06221001040780016
:1012e000e44f500033003200e062210010407800eb
:1012f000e34f500004003a00d06221001040780013
:10130000e44f50002b003200510b81001e0078008a
:101310001000780000017800818040000063210007
:1013200000804000020878001e8fe800510b810009
:101330001e00780010007800000178000180400055
:10134000810c20008080400000632100008040006c
:10135000020878001e8fe800510b81001e00780003
:101360001000780000017800018040000119200081
:101370008080400000632100008040000208780067
:101380001e8fe800500b81000000e800500b890020
:10139000510b810030062000808f50000500360080
:1013a0000000eb00500b8900b162210010c0b300b7
:1013b00080487800e062210090407800e0c3b300ec
:1013c00080cf500028003a00600b81000000e80048
:1013d000600b8900610b810010032000808f50009a
:1013e000020036000000eb00600b8900610b8100f9
:1013f0001e00780010007800000178008180400015
:101400008088210000804000020878001e8fe800dc
:10141000610b81001e007800100078000001780048
:10142000018040004106200080804000808821002b
:1014300000804000020878001e8fe800610b8100e8
:101440001e00780010007800000178000180400044
:10145000810c2000808040008088210000804000b6
:101460000208780000013700e06221009040780017
:10147000f0c3b30080cf500071003a00d062210069
:10148000104078000080fb00300798003e0090007c
:10149000e20f500023003200be009000e28f5000a7
:1014a00007003c003e0090000000e0000b0032000e
:1014b000be009000e18f500011003200ea003700ba
:1014c0003e009000e30f50001f003200be0090006d
:1014d000e48f500025003200e30037001e00780042
:1014e00010007800a0cd88001e8fe8001e00780054
:1014f00010007800e0cd8800e2e2a800da003700b2
:101500001e00780010007800b0cd88001e8fe80023
:101510001e00780010007800f0cd8800e302a800db
:10152000d10037001e00780010007800c0cd880080
:101530001e8fe8001e0078001000780000ce8800a2
:10154000e802a800c80037001e00780010007800ec
:10155000d0cd88001e8fe8001e00780010007800b3
:1015600010ce8800e822a800bf0037001e007800d7
:101570001000780030ce88001e8fe8001e00780032
:101580001000780020ce88001e8fe800510b8100eb
:101590001e00780010007800000178008180400073
:1015a0000063210000804000020878001e8fe800e0
:1015b000510b81001e0078001000780000017800b7
:1015c00001804000810c20008080400000632100e9
:1015d00000804000020878001e8fe800510b810057
:1015e0001e007800100078000001780001804000a3
:1015f000011920008080400000632100008040002d
:1016000002087800500b81000000e800500b8900b0
:10161000510b810030062000808f500005003600fd
:101620000000eb00500b8900b162210010c0b30034
:1016300080487800d042a800d022a8008a00370055
:10164000e062210010407800e34f500086003a002d
:10165000d0622100104078000080fb002007980035
:101660002e009000e20f500029003200ae009000e2
:10167000e28f500007003c002e0090000000e000c8
:101680000b003200ae009000e18f500014003200d9
:10169000750037002e009000e30f50002800320044
:1016a000ae009000e48f5000380032006e0037002a
:1016b0001e0078001000780040ce88001e8fe800e1
:1016c0001e0078001000780080ce8800e2e2a900b9
:1016d000d162210010c0b30080487800620037005a
:1016e0001e0078001000780050ce88001e8fe800a1
:1016f0001e0078001000780090ce8800e302a90058
:10170000d162210020c0b300804878005600370025
:101710001e0078001000780060ce88001e8fe80060
:101720001e00780010007800a0ce8800e802a90012
:10173000d162210030c0b300804878004a003700f1
:101740001e0078001000780070ce88001e8fe80020
:101750001e00780010007800b0ce8800e822a900b2
:10176000e0ce8000ea0f500004003a00d162210070
:1017700040c0b300804878003b003700d1622100b0
:101780000040eb0080487800370037001e007800ea
:1017900010007800d0ce88001e8fe8001e00780070
:1017a00010007800c0ce88001e8fe800d042a9004b
:1017b000d022a900d16221000040eb0080487800cf
:1017c000510b81001e0078001000780000017800a5
:1017d0008180400000632100008040000208780002
:1017e0001e8fe800510b81001e0078001000780069
:1017f0000001780001804000810c200080804000c2
:101800000063210000804000020878001e8fe8007d
:10181000510b81001e007800100078000001780054
:1018200001804000011920008080400000632100f9
:101830000080400002087800500b81000000e800a2
:10184000500b8900510b810030062000808f500022
:10185000050036000000eb00500b8900b16221004a
:1018600010c0b30080487800e0622100104078008a
:10187000304798000040eb0020479800f0c3b300c9
:10188000be40900080cf50000200360010c0b30070
:10189000204798003e4090008040e800e062210030
:1018a00001487800ae4090000104e00003003200df
:1018b000e16221000040eb0080487800a162210035
:1018c00010c0b300804878000080fa003400f900ae
:1018d0004f0178004f00be00004006000000fa00f3
:1018e000a0622100104078000080fb000080fa0018
:1018f000000006000000fa00b062210010407800ed
:101900000080fb000080fa00000006000000fa00e2
:10191000a1e2a8000080fa00000006000000fa0022
:10192000a1e2a9000080fa00000006002200fa00ef
:1019300070079800010f9800120f9800230f98006d
:10194000340f9800450f9800560f98007e009000c5
:10195000200db000700798000e089000670040004e
:10196000000f98004e0890000000e00003003200d5
:101970003e0890000000e00003003a000080eb0009
:10198000600f980010013700fe0090001e089000c4
:101990008080400020352000808f500003003600fa
:1019a0008080eb00610f9800070137008e089000df
:1019b0002e08900080804000701e2000808f500014
:1019c000030036000080eb00600f9800fe00370037
:1019d0001e0890003e099000110009000280d80006
:1019e0008000fd000000e000030032008080eb007a
:1019f000610f9800f40037002e0890004e09900007
:101a0000110009000280d8008000fd000000e00005
:101a1000030032000080eb00600f9800ea003700fe
:101a20004e089000630060000000e00033003a00c0
:101a30003e089000630060000000e0000f003a00e4
:101a400030032000000f78004e0890004200de00b6
:101a5000200798003e0890004200de001007980022
:101a60000e08900064005000000f98007e00900067
:101a70006400500070079800500037003e08900046
:101a8000610060000000e0000f003a00100120003b
:101a9000000f78004e0890000000d1002007980049
:101aa0003e0890000000d100100798000e0890003a
:101ab0000080e900000f98007e0090000080e9009f
:101ac000700798003d00370040042000000f7800a8
:101ad000ce089000210798003e089000100798005b
:101ae0000e0890000000e900000f98007e009000b2
:101af0000000e90070079800300037004e089000a1
:101b0000610060000000e00020003a003e08900004
:101b1000610060000000e0000f003a0010012000aa
:101b2000000f78004e0890000000d10020079800b8
:101b30003e0890000000d100100798000e089000a9
:101b40000080e900000f98007e0090000080e9000e
:101b5000700798001900370040042000000f78003b
:101b6000ce089000210798003e08900010079800ca
:101b70000e0890000000e900000f98007e00900021
:101b80000000e900700798000c00370040042000b6
:101b9000000f7800be089000110798004e089000d2
:101ba000200798000e0890000000e900000f980040
:101bb0007e0090000000e900700798001e00900071
:101bc0000000e900500798002e0090000000e90096
:101bd000600798001e0890003e099000110009005f
:101be0000280d800400798002e0890004e0990000f
:101bf000110009000280d800300798005e089000ac
:101c000084a40200000000000000e0000300320095
:101c10008080eb00610f98006b0037001e00780099
:101c2000c8a40200000000000000e0000300320031
:101c30000080eb00600f9800630037005e089000a2
:101c40000000e0001a003a009e007800710f980032
:101c500030032000fe089000808f500010003200fa
:101c600040042000fe089000808f500004003200e5
:101c70007e089000f10f500005003200250037006b
:101c800000032000f6a4020000000000210037003d
:101c900000022000f6a40200000000001d00370032
:101ca0000000eb00f6a4020000000000190037005d
:101cb0009e00780001179800300320008e109000dd
:101cc000808f500010003200400420008e109000e1
:101cd000808f5000040032000e109000f10f500071
:101ce000050032000b00370000042000f6a40200bb
:101cf000000000000700370000032000f6a40200e7
:101d0000000000000300370000022000f6a40200db
:101d100000000000313520007e00900040a5020048
:101d2000000000000000e000030032008080eb00b3
:101d3000610f980024003700811e20000e089000db
:101d40009ca50200000000000000e000030032003b
:101d50000080eb00600f98001b0037007e009000b1
:101d60000001e800711e20000e089000f2a502009c
:101d7000000000000000e000030032008080eb0063
:101d8000610f9800100037005e08900011000700f6
:101d9000000178006e029000de019000ce009000fd
:101da0003e0090003eb30200000000000000e00092
:101db000030032000080eb00600f98000200370043
:101dc0008000eb00610f98006e0890000080fa0020
:101dd000000006000600fa00000f78001e007800e0
:101de000200798002e009000e10f50000a003200fa
